:020000040800F2
:1000000000040020A51F0008F71F0008F71F0008C4
:10001000F71F0008F71F0008F71F00080000000086
:10002000000000000000000000000000F71F0008B2
:10003000F71F000800000000F71F0008B1BA010810
:1000400049BC01084BBC01084DBC010851BC01086A
:1000500071BC010873BC010875BC010899BC01089A
:10006000BDBC0108E1BC010805BD010829BD0108AE
:100070002BBD01082DBD01082FBD010831BD0108B0
:1000800033BD010835BD010837BD0108F71F000861
:10009000F71F0008F71F0008F71F000839BD010807
:1000A00085BD010887BD010889BD01088BBD010818
:1000B0008DBD010891BD0108BDBD01081DBE01082F
:1000C0001FBE010821BE010823BE010825BE01088C
:1000D00029BE010891BF0108C1BE010855C0010831
:1000E00019C10108DDC10108DFC10108E1C1010832
:1000F000E5C1010841C2010843C2010845C2010827
:1001000047C2010849C201084BC201084DC201089B
:1001100051C2010825C3010827C3010829C30108EA
:100120002BC301082DC301082FC3010831C30108E7
:1001300000000000000000000000000000000000BF
:1001400000000000000000000000000000000000AF
:10015000000000000000000000000000000000009F
:10016000000000000000000000000000000000008F
:10017000000000000000000000000000000000007F
:10018000000000000000000000000000000000006F
:10019000000000000000000000000000000000005F
:1001A000000000000000000000000000000000004F
:1001B000000000000000000000000000000000003F
:1001C000000000000000000000000000000000002F
:1001D000000000000000000000000000000000001F
:0401E0005FF8E0F1F3
:1001E800032A70B404460D4626D941EA000313F0E9
:1001F800030F13D020782B78984208BF294606D0E1
:100208001EE014F8010F11F8013F984218D1012A95
:1002180002F1FF32F5D1002070BC70470B4604464E
:1002280051F8045B50F8046BAE4204D1043A04461A
:10023800032A0B46F2D81D461046002ADAD1EBE70E
:10024800C01AE9E7032A2DE9F00109D82AB10023E9
:10025800CC5CC45401339342FAD1BDE8F001704735
:100268000B468218014603E02478013301F8014B5C
:1002780011F0030F1C46F7D113F003055DD06E4251
:10028800C5F1040CED009B594FEACC0C08E004348E
:10029800A7593B4607FA0CF748EA070741F8047BD9
:1002A800571A23FA05F8032FF1DC03E014F8013B91
:1002B80001F8013B8A42F9D8CFE753F8404C41F89E
:1002C800404C53F83C4C41F83C4C53F8384C41F8FE
:1002D800384C53F8344C41F8344C53F8304C41F80E
:1002E800304C53F82C4C41F82C4C53F8284C41F81E
:1002F800284C53F8244C41F8244C53F8204C41F82E
:10030800204C53F81C4C41F81C4C53F8184C41F83D
:10031800184C53F8144C41F8144C53F8104C41F84D
:10032800104C53F80C4C41F80C4C53F8084C41F85D
:10033800084C53F8044C41F8044C561A1D460C4618
:10034800403340313F2EB8DC2B460FE053F8101CE9
:1003580044F8101C53F80C1C44F80C1C53F8081CE7
:1003680044F8081C53F8041C44F8041C161B2146C6
:100378001D46103410330F2EE8DC2B4602E02468AB
:1003880041F8044B551A1C46032D03F10403F6DC0F
:1003980090E700BF032AC9B270B408D82AB103464F
:1003A800121803F8011B9342FBD170BC70478218E6
:1003B800044601E004F8011B14F0030FFAD14FF0D2
:1003C800013303FB01F31FE044F8403C44F83C3C94
:1003D80044F8383C44F8343C44F8303C44F82C3C6D
:1003E80044F8283C44F8243C44F8203C44F81C3C9D
:1003F80044F8183C44F8143C44F8103C44F80C3CCD
:1004080044F8083C44F8043C161B254640343F2E6B
:10041800DADC2C4607E044F8103C44F80C3C44F87D
:10042800083C44F8043C161B254610340F2EF2DC19
:1004380001E045F8043B541B032CFADC01E005F805
:10044800011B9542FBD3B0E710F0030F38B5044603
:1004580012D10368A3F1013222EA030313F0803FAB
:100468000AD1031D184653F8042BA2F1013525EAD9
:10047800020212F0803FF5D003782BB1431C1846D6
:1004880013F8012B002AFAD100F076F9204638BD7E
:10049800C9B2F0B4002950D010F0030F10D003787F
:1004A800002B79D0994246D0431C05E013F8012B64
:1004B800002A3FD091423ED013F0030F1846F5D1E1
:1004C800036841EA01270646A3F1013247EA0747D4
:1004D80022EA030212F0803F1DD187EA0303A3F149
:1004E800013222EA030313F0803F14D1043002E002
:1004F80012F0803F0FD1064650F8043BA3F10135B6
:1005080087EA030225EA0303A2F1013413F0803FCE
:1005180024EA0202ECD033783046002B3CD09942D2
:1005280009D0731C01E0914205D0184613F8012B3D
:10053800002AF8D11046F0BC704710F0030F0CD019
:100548000378002BF7D0431C03E013F8012B002A93
:10055800F1D013F0030F1846F7D102680346A2F151
:10056800013121EA020212F0803F0AD10430034629
:1005780050F8042BA2F1013121EA020212F0803F67
:10058800F5D01A781846002AD5D00133184613F842
:10059800012B002AFAD1CEE71846CCE780EA0102FF
:1005A80012F0030F3AD110F0030220F0030021F0FB
:1005B800030150F804CB08BF51F8043B0DD082F07A
:1005C80003024FEAC2026FF07F4323FA02F251F8A6
:1005D800043B4CEA020C43EA020300BFACF10132CF
:1005E8009C4501BF22EA0C0212F0803F50F804CB70
:1005F80051F8043BF2D04FEA0C604FEA1C2C01285A
:1006080028BFB0EB036F08BF1B0AF4D003F0FF0349
:100618004FEA1060A0EB0300704700BF10F0030F13
:100628000AD010F8012B11F8013B012A28BF9A4281
:10063800F4D0A2EB030070474DF8045D4DF8044D6B
:100648004FF0010242EA022242EA024201F0030CA0
:1006580021F0030150F8044B51F8045BBCF1020F80
:1006680026D04BD824F07F4CBCEB152FA4EB02030B
:1006780023EA04030DD113EAC21308BF51F8045B3F
:100688000AD18CEA040CBCEB056F0CD150F8044B72
:10069800E8E74FEA15255CE033F07F4352D10D7847
:1006A8004FEA146C55E04FEA146C05F0FF0550E072
:1006B8004FEA044CA4EB02034FEA1C4C23EA040360
:1006C800BCEB154F17D113EAC21308BF51F8045BEE
:1006D80007D18CEA040CBCEB054F08D150F8044B49
:1006E800E6E71B042ED10D884FEA144C31E04FEA9F
:1006F80005454FEA144C4FEA15452AE004F0FF0C73
:10070800BCEB156FA4EB020323EA04030DD113EA33
:10071800C21308BF51F8045B0AD18CEA040CBCEB85
:10072800052F0AD150F8044BE8E74FEA156510E0A9
:1007380014F0FF0F06D051F8045B4FEA142C25F093
:100748007F4506E04FF000005DF8044B5DF8045B60
:1007580070470CF0FF0205F0FF00012828BF904207
:1007680004BF4FEA1C2C2D0AF3D0A2EB00005DF861
:10077800044B5DF8045B704780EA0102844612F07E
:10078800030F4FD111F0030F32D14DF8044D11F082
:10079800040F51F8043B0BD0A3F101329A4312F035
:1007A800803F04BF4CF8043B51F8043B16D100BF0E
:1007B80051F8044BA3F101329A4312F0803FA4F19F
:1007C80001320BD14CF8043BA24312F0803F04BF26
:1007D80051F8043B4CF8044BEAD023460CF8013B93
:1007E80013F0FF0F4FEA3323F8D15DF8044B70473D
:1007F80011F0010F06D011F8012B0CF8012B002A7B
:1008080008BF704711F0020FBFD031F8022B12F069
:10081800FF0F16BF2CF8022B8CF8002012F47F4F24
:10082800B3D1704711F8012B0CF8012B002AF9D12C
:10083800704700BF20F0030110F00300C0F1000072
:1008480051F8043B00F1040C4FEACC0C6FF00002A5
:100858001CBF22FA0CF213434FF0010C4CEA0C2C8B
:100868004CEA0C4CA3EB0C0222EA030212EACC126B
:1008780004BF51F8043B0430F4D013F0FF0F1FBF3E
:10088800013013F47F4F013013F47F0F18BF01308C
:10089800704700BFF0B4002A46D041EA000313F0C5
:1008A80003032CD1032A07460E4643D904680D6872
:1008B800AC423FD1043A37D0A4F1013525EA04040B
:1008C80014F0803F18BF18462CD1041D0D1D0EE0F2
:1008D80054F8043B55F8041BA3F101308B4220EA7D
:1008E800030027D1043A1FD010F0803F1ED1032AFD
:1008F80027462E46ECD820462946002A1DD00478E3
:10090800013A0D78AC420CD172B18CB1002302E0EF
:1009180093420BD064B1013310F8014FCD5CAC4267
:10092800F6D0601BF0BC70471046FBE70020F9E7E3
:100938002046F7E738463146E1E724782D78F0E796
:1009480041EA000313F0030F0B4670B414BF0024F0
:100958000124032A94BF002404F001040546D4B9F5
:10096800BAB10E782B46013A03F8016B56B1AC1CAC
:100978007AB111F8015F2346013A04F8015C0134A9
:10098800002DF5D12AB19A18002103F8011B9342D2
:10099800FBD170BC7047194653F8044BA4F10136DB
:1009A80026EA040616F0803FDAD1043A45F8044BEB
:1009B800032A1946EFD8D3E701232DE9F0071D468E
:1009C80000264FF0FF37AC1900EB070C8C420DD214
:1009D8001CF805C010F80480E0452ED201252646F3
:1009E800E31BAC198C4200EB070CF1D34FF0010963
:1009F80000264D464FF0FF3C1360AC1900EB0C0885
:100A0800A1420ED918F8058010F804A0C2451AD9D9
:100A180001252646CCEB0409AC19A14200EB0C08D1
:100A2800F0D80CF101000137B8423CBF994638466E
:100A3800C2F80090BDE8F00770470BD00123374695
:100A48001D46F618BFE709D04FF00109B4464D46D8
:100A58004E44D2E79D4205D00135B4E74D4505D057
:100A68000135CAE72B4626460125ACE7A9462646A6
:100A78000125C2E72DE9F04FADF5826D81B014462E
:100A8800074610460DF580628B460C3219461D4606
:100A9800FFF792FF03AE04A901F57E72331F0090A1
:100AA80043F8045F9342FBD14DB1681E0023E25C1A
:100AB800C11A013303AEAB4246F82210F7D1DDF874
:100AC8000C142046009A6118FFF78AFB002877D19A
:100AD8000099814605F1FF380646C1F101020192ED
:100AE8005A46AB4609EB0B0501F1FF3AB81800214D
:100AF800AA1A00F0E5F900284FD1002D00F0C080B7
:100B08007B1903A913F8013C51F82330002B4CD171
:100B1800009B9E4228BF334698450FD903EB090135
:100B2800E05C7A18795C884205D038E012F8011F39
:100B3800E05C884233D101339845F7D8009A964251
:100B480080F0A48007EB090214F80A10534612F843
:100B58000A20914204BF0AEB0901791807D095E0F1
:100B680014F802C011F8010D844503D113465A1E2A
:100B7800B342F5D101369E4200F28D80DDF80C6457
:100B88002A46B144C6EB0B0609EB0B05B818002141
:100B9800AA1A00F095F90028AFD0002071E0019A58
:100BA8000026914499442A46EEE7002EFAD0DDF853
:100BB8000C2493423CBFC2EB0B0306469944F2E770
:100BC800009E4FF000080099AB1BB34238BF334674
:100BD800C1F101026E1E019201F1FF3A5A4689469F
:100BE800AB460133CDF80C3408EB0B05B8180021DF
:100BF800AA1A00F065F90028CFD1002D40D07B1942
:100C080003A913F8013C51F82330002B30D1B1452A
:100C180013D208EB090314F80910FA18FB5C99427F
:100C280018BF4B4627D14B4604E012F8011FE05C81
:100C3800884220D10133B342F7D3BAF1FF3F53467C
:100C48002CD007EB080C14F80A101CF80A20914263
:100C58000CD10AEB0802BA1804E0E05C12F8011D96
:100C6800884203D1013BF8D260460AE0DDF80C3433
:100C780098442A46B8E701992A4688449844B3E735
:100C8800284605B00DF5806DBDE8F08F009B013654
:100C98009E427FF673AF07EB0900F2E707EB080CFB
:100CA8006046EEE72DE9F04F8346037885B00C46A1
:100CB800002B00F0F9800A78A2B106460131012024
:100CC80002E011F8012B8AB1934214BF002000F012
:100CD800010016F8013F0D46002BF2D12B782BB1FD
:100CE8004FF0000B584605B0BDE8F08F0028F9D149
:100CF8000BF101002178FFF7CBFB2D1BA5F10102B9
:100D0800534243EB0203002808BF43F001030746A0
:100D180083B90BEB0508404594BFC0EB08084FF0BA
:100D280001081F2D08D9414622462B46FFF7A2FE8F
:100D38008346D7E78346D5E7294603AA2046FFF727
:100D48003BFE03996118814620464A46FFF748FA58
:100D580000284FD109F1FF33C9F10102064601927B
:100D680082464246C84699460AEB050BB818002148
:100D7800C2EB0B0200F0A4F80028B1D1BBF1000FC0
:100D8800B0D046452CBF334643469D420FD903EBAE
:100D98000A01E05C7A18795C884205D075E012F89F
:100DA800011FE05C884270D101339D42F7D1B04504
:100DB8007DD907EB0A0214F809104B4612F80920EE
:100DC800914202BF09EB0A01AC46791806D06EE0E1
:100DD800A55C11F8010D854203D113465A1EB34292
:100DE800F6D1654601369E4267D8039E5A46B244FC
:100DF800AE1BB9E7C9F10101C9EB0503424600265C
:100E080009F1FF3A88464B4538BF4B4601330393F7
:100E180006EB050BB8180021C2EB0B0200F050F8E6
:100E280000287FF45DAFBBF1000F3FF45BAF4D4589
:100E380012D906EB090314F80910FA18FB5C994259
:100E480008BF4B4605D026E012F8011FE05C884237
:100E580022D101339D42F7D1BAF1FF3F534628D042
:100E680007EB060C14F80A101CF80A20914217D157
:100E78000AEB0602BA1804E0E05C12F8011D884289
:100E88000ED1013BF8D2E3462CE7019A00269244A2
:100E98005A469A4468E74B4646445A46F618B7E716
:100EA800039B5A46F618B3E70D46012016E743465A
:100EB80098E707EB060CE34614E707EB0A0B11E784
:100EC80010F0030F034670B4C9B211D0002A22D023
:100ED80003788B421DD0013A013005E0DAB110F8F1
:100EE800014B013A8C4218D010F0030F0346F5D19C
:100EF800032A14D87AB1187888420ED0541E5D1C83
:100F080003E015F8016B8E4203D0013C2846F8D265
:100F1800002070BC70471046FBE71846F9E741EA25
:100F2800012646EA0646184653F8044B86EA0404A6
:100F3800A4F1013525EA040414F0803F03D1043AF2
:100F48001846032AEFD80346D4E700BF0000000084
:100F5800C1F30A5C0246ACF57E7C2DE9F84FACF192
:100F68000704132C0B4606460F468946804627DCA5
:100F7800002C52DB4FF6FF7CC0F20F0C4CFA04FA3F
:100F88000AEA0105054317D037A3D3E9002300F087
:100F980075F80022002300F0B3FC002856D0002F7B
:100FA80005DD4FF4801353FA04F407EB040929EA2A
:100FB8000A0900264B46324610461946BDE8F88F06
:100FC800332C07DDB4F5806FF6D100F057F80246F0
:100FD8000B46F1E74FF0FF3BACF11B0C2BFA0CFB77
:100FE8001BEA000FE8D020A3D3E9002300F046F85D
:100FF8000022002300F084FC40B3002F0ADD142CEB
:1010080006D00126C4F13404A64016EB080601D325
:1010180007F1010926EA0B0619E013A3D3E9002317
:1010280000F02CF80022002300F06AFC78B1002FB1
:1010380013DB46EA07054FF000094D45C3F6F07982
:101048000CBF2E46002608BFA94600E0B9464B460D
:10105800324610461946BDE8F88F00264FF0004981
:10106800F5E700BFAFF300809C7500883CE4377E4D
:1010780081F0004102E000BF83F0004330B54FEA41
:1010880041044FEA430594EA050F08BF90EA020FAE
:101098001FBF54EA000C55EA020C7FEA645C7FEA41
:1010A800655C00F0E2804FEA5454D4EB5555B8BF64
:1010B8006D420CDD2C4480EA020281EA030382EAD5
:1010C800000083EA010180EA020281EA0303362D67
:1010D80088BF30BD11F0004F4FEA01314FF4801C3A
:1010E8004CEA113102D0404261EB410113F0004F4C
:1010F8004FEA03334CEA133302D0524263EB430303
:1011080094EA050F00F0A780A4F10104D5F1200EA0
:101118000DDB02FA0EFC22FA05F2801841F10001FB
:1011280003FA0EF2801843FA05F359410EE0A5F1CF
:1011380020050EF1200E012A03FA0EFC28BF4CF000
:10114800020C43FA05F3C01851EBE37101F00045B6
:1011580007D54FF0000EDCF1000C7EEB00006EEBC3
:101168000101B1F5801F1BD3B1F5001F0CD349084D
:101178005FEA30004FEA3C0C04F101044FEA4452A4
:1011880012F5800F80F09A80BCF1004F08BF5FEA2B
:10119800500C50F1000041EB045141EA050130BD0B
:1011A8005FEA4C0C404141EB010111F4801FA4F1AE
:1011B8000104E9D191F0000F04BF01460020B1FA03
:1011C80081F308BF2033A3F10B03B3F120020CDA3B
:1011D8000C3208DD02F1140CC2F10C0201FA0CF019
:1011E80021FA02F10CE002F11402D8BFC2F1200C7E
:1011F80001FA02F120FA0CFCDCBF41EA0C01904034
:10120800E41AA2BF01EB0451294330BD6FEA04047C
:101218001F3C1CDA0C340EDC04F11404C4F1200267
:1012280020FA04F001FA02F340EA030021FA04F379
:1012380045EA030130BDC4F10C04C4F1200220FAD0
:1012480002F001FA04F340EA0300294630BD21FA0E
:1012580004F0294630BD94F0000F83F4801306BFD4
:1012680081F480110134013D4EE77FEA645C18BFC8
:101278007FEA655C29D094EA050F08BF90EA020F5F
:1012880005D054EA000C04BF1946104630BD91EA57
:10129800030F1EBF0021002030BD5FEA545C05D15A
:1012A8004000494128BF41F0004130BD14F5800499
:1012B8003CBF01F5801130BD01F0004545F0FE410D
:1012C80041F470014FF0000030BD7FEA645C1ABF42
:1012D800194610467FEA655C1CBF0B46024650EA79
:1012E800013406BF52EA033591EA030F41F40021A5
:1012F80030BD00BF90F0000F04BF0021704730B52B
:101308004FF4806404F132044FF000054FF00001FF
:1013180050E700BF90F0000F04BF0021704730B5C0
:101328004FF4806404F1320410F0004548BF404295
:101338004FF000013EE700BF42004FEAE2014FEAEA
:1013480031014FEA02701FBF12F07F4393F07F4FC5
:1013580081F06051704792F0000F14BF93F07F4FF7
:10136800704730B54FF4607401F0004521F000413A
:1013780020E700BF50EA010208BF704730B54FF0C0
:1013880000050AE050EA010208BF704730B511F0C5
:10139800004502D5404261EB41014FF4806404F1FD
:1013A80032045FEA915C3FF4DCAE4FF003025FEA7F
:1013B800DC0C18BF03325FEADC0C18BF033202EB07
:1013C800DC02C2F1200300FA03FC20FA02F001FA61
:1013D80003FE40EA0E0021FA02F11444C1E600BF00
:1013E80070B54FF0FF0C4CF4E06C1CEA11541DBFB3
:1013F8001CEA135594EA0C0F95EA0C0F00F0DEF87E
:101408002C4481EA030621EA4C5123EA4C5350EA62
:10141800013518BF52EA033541F4801143F48013B3
:1014280038D0A0FB02CE4FF00005E1FB02E506F044
:101438000042E0FB03E54FF00006E1FB03569CF099
:10144800000F18BF4EF0010EA4F1FF04B6F5007F9F
:1014580064F5407404D25FEA4E0E6D4146EB060611
:1014680042EAC62141EA55514FEAC52040EA5E509A
:101478004FEACE2EB4F1FD0C88BFBCF5E06F1ED844
:10148800BEF1004F08BF5FEA500E50F1000041EB7B
:10149800045170BD06F0004646EA010140EA020028
:1014A80081EA0301B4EB5C04C2BFD4EB0C0541EA4A
:1014B800045170BD41F480114FF0000E013C00F35F
:1014C800AB8014F1360FDEBF002001F0004170BD83
:1014D800C4F10004203C35DA0C341BDC04F114049C
:1014E800C4F1200500FA05F320FA04F001FA05F228
:1014F80040EA020001F0004221F0004110EBD370F5
:1015080021FA04F642EB06015EEA430E08BF20EA20
:10151800D37070BDC4F10C04C4F1200500FA04F3C3
:1015280020FA05F001FA04F240EA020001F0004155
:1015380010EBD37041F100015EEA430E08BF20EAC8
:10154800D37070BDC4F1200500FA05F24EEA020E10
:1015580020FA04F301FA05F243EA020321FA04F03F
:1015680001F0004121FA04F220EA020000EBD370F6
:101578005EEA430E08BF20EAD37070BD94F0000FF6
:101588000FD101F00046400041EB010111F4801F2A
:1015980008BF013CF7D041EA060195F0000F18BFDB
:1015A800704703F00046520043EB030313F4801F17
:1015B80008BF013DF7D043EA0603704794EA0C0FD1
:1015C8000CEA135518BF95EA0C0F0CD050EA4106E7
:1015D80018BF52EA4306D1D181EA030101F0004164
:1015E8004FF0000070BD50EA410606BF104619468C
:1015F80052EA430619D094EA0C0F02D150EA013698
:1016080013D195EA0C0F05D152EA03361CBF1046D8
:1016180019460AD181EA030101F0004141F0FE4177
:1016280041F470014FF0000070BD41F0FE4141F4FB
:10163800780170BD70B54FF0FF0C4CF4E06C1CEAFB
:1016480011541DBF1CEA135594EA0C0F95EA0C0FB0
:1016580000F0A7F8A4EB050481EA030E52EA03356B
:101668004FEA013100F088804FEA03334FF080558C
:1016780045EA131343EA12634FEA022245EA1115B9
:1016880045EA10654FEA00260EF000419D4208BF6A
:10169800964244F1FD0404F5407402D25B084FEA17
:1016A8003202B61A65EB03055B084FEA32024FF4C3
:1016B80080104FF4002CB6EB020E75EB030E22BF20
:1016C800B61A754640EA0C005B084FEA3202B6EBE0
:1016D800020E75EB030E22BFB61A754640EA5C008F
:1016E8005B084FEA3202B6EB020E75EB030E22BF1F
:1016F800B61A754640EA9C005B084FEA3202B6EB20
:10170800020E75EB030E22BFB61A754640EADC00DE
:1017180055EA060E18D04FEA051545EA16754FEA40
:1017280006164FEAC30343EA52734FEAC2025FEA5E
:101738001C1CC0D111F4801F0BD141EA00014FF0ED
:1017480000004FF0004CB6E711F4801F04BF0143BE
:101758000020B4F1FD0C88BFBCF5E06F3FF6AFAEDA
:10176800B5EB030C04BFB6EB020C5FEA500C50F16A
:10177800000041EB045170BD0EF0004E4EEA1131ED
:1017880014EB5C04C2BFD4EB0C0541EA045170BDF4
:1017980041F480114FF0000E013C90E645EA060E38
:1017A8008DE60CEA135594EA0C0F08BF95EA0C0F66
:1017B8003FF43BAF94EA0C0F0AD150EA01347FF4AE
:1017C80034AF95EA0C0F7FF425AF104619462CE785
:1017D80095EA0C0F06D152EA03353FF4FDAE1046E8
:1017E800194622E750EA410618BF52EA43067FF439
:1017F800C5AE50EA41047FF40DAF52EA43057FF4C9
:10180800EBAE12E74FF0FF3C06E000BF4FF0010CD3
:1018180002E000BF4FF0010C4DF804CD4FEA410C37
:101828007FEA6C5C4FEA430C18BF7FEA6C5C1BD004
:1018380001B050EA410C0CBF52EA430C91EA030F85
:1018480002BF90EA020F0020704710F1000F91EAE2
:10185800030F58BF994208BF90422CBFD8176FEAB0
:10186800E37040F0010070474FEA410C7FEA6C5C7E
:1018780002D150EA013C07D14FEA430C7FEA6C5C85
:10188800D6D152EA033CD3D05DF8040B704700BFB1
:101898008446104662468C461946634600E000BFFF
:1018A80001B5FFF7B7FF002848BF10F1000F01BDD1
:1018B8004DF808EDFFF7F4FF0CBF012000205DF89C
:1018C80008FB00BF4DF808EDFFF7EAFF34BF012021
:1018D80000205DF808FB00BF4DF808EDFFF7E0FFBA
:1018E80094BF012000205DF808FB00BF4DF808ED0B
:1018F800FFF7CEFF94BF012000205DF808FB00BF72
:101908004DF808EDFFF7C4FF34BF012000205DF853
:1019180008FB00BF4FEA4102B2F1E04324BFB3F530
:10192800001CDCF1FE5C0DD901F0004C4FEAC0024E
:101938004CEA5070B2F1004F40EB830008BF20F032
:101948000100704711F0804F21D113F13872BCBFEC
:1019580001F00040704741F480114FEA5252C2F141
:101968001802C2F1200C10FA0CF320FA02F018BF8A
:1019780040F001004FEAC1234FEAD32303FA0CFCDD
:1019880040EA0C0023FA02F34FEA4303CCE77FEA6C
:10199800625307D150EA01331EBF4FF0FE4040F4B6
:1019A8004000704701F0004040F0FE4040F4000065
:1019B800704700BF80F0004002E000BF81F00041A6
:1019C80042001FBF5FEA410392EA030F7FEA226CDD
:1019D8007FEA236C6AD04FEA1262D2EB1363C1BF6D
:1019E800D218414048404140B8BF5B42192B88BFDC
:1019F800704710F0004F40F4000020F07F4018BFFF
:101A0800404211F0004F41F4000121F07F4118BF1E
:101A1800494292EA030F3FD0A2F1010241FA03FCC6
:101A280010EB0C00C3F1200301FA03F100F00043AE
:101A380002D5494260EB4000B0F5000F13D3B0F176
:101A4800807F06D340084FEA310102F10102FE2AE5
:101A580051D2B1F1004F40EBC25008BF20F0010055
:101A680040EA03007047490040EB000010F4000F03
:101A7800A2F10102EDD1B0FA80FCACF1080CB2EB96
:101A88000C0200FA0CF0AABF00EBC25052421843F5
:101A9800BCBFD0401843704792F0000F81F400019A
:101AA80006BF80F400000132013BB5E74FEA41036D
:101AB8007FEA226C18BF7FEA236C21D092EA030FD9
:101AC80004D092F0000F08BF0846704790EA010F53
:101AD8001CBF0020704712F07F4F04D1400028BF80
:101AE80040F00040704712F100723CBF00F5000062
:101AF800704700F0004343F0FE4040F40000704798
:101B08007FEA226216BF08467FEA23630146420243
:101B180006BF5FEA412390EA010F40F48000704756
:101B28004FF0000304E000BF10F0004348BF4042FC
:101B38005FEA000C08BF704743F0964301464FF038
:101B480000001CE050EA010208BF70474FF0000394
:101B58000AE000BF50EA010208BF704711F00043D5
:101B680002D5404261EB41015FEA010C02BF8446A5
:101B78000146002043F0B64308BFA3F18053A3F504
:101B88000003BCFA8CF2083AA3EBC25310DB01FA4B
:101B980002FC634400FA02FCC2F12002BCF1004FCF
:101BA80020FA02F243EB020008BF20F00100704760
:101BB80002F1200201FA02FCC2F1200250EA4C00B4
:101BC80021FA02F243EB020008BF20EADC707047FA
:101BD8004FF0FF0C1CEAD0521EBF1CEAD15392EA08
:101BE8000C0F93EA0C0F6FD01A4480EA010C4002E4
:101BF80018BF5FEA41211ED04FF0006343EA50103E
:101C080043EA5111A0FB01310CF00040B1F5000F7F
:101C18003EBF490041EAD3715B0040EA010062F12E
:101C28007F02FD2A1DD8B3F1004F40EBC25008BF18
:101C380020F00100704790F0000F0CF0004C08BF36
:101C480049024CEA502040EA51207F3AC2BFD2F103
:101C5800FF0340EAC250704740F400004FF0000311
:101C6800013A5DDC12F1190FDCBF00F0004070474B
:101C7800C2F10002410021FA02F1C2F1200200FA89
:101C880002FC5FEA310040F1000053EA4C0308BF50
:101C980020EADC70704792F0000F00F0004C02BFA1
:101CA800400010F4000F013AF9D040EA0C0093F01C
:101CB800000F01F0004C02BF490011F4000F013B76
:101CC800F9D041EA0C018FE70CEAD15392EA0C0FE4
:101CD80018BF93EA0C0F0AD030F0004C18BF31F04F
:101CE800004CD8D180EA010000F00040704790F025
:101CF800000F17BF90F0004F084691F0000F91F0C9
:101D0800004F14D092EA0C0F01D142020FD193EA8E
:101D18000C0F03D14B0218BF084608D180EA010016
:101D280000F0004040F0FE4040F40000704740F0F2
:101D3800FE4040F4400070474FF0FF0C1CEAD052C0
:101D48001EBF1CEAD15392EA0C0F93EA0C0F69D01C
:101D5800A2EB030280EA010C49024FEA402037D087
:101D68004FF0805343EA111143EA10130CF000407E
:101D78008B4238BF5B0042F17D024FF4000C8B426E
:101D880024BF5B1A40EA0C00B3EB510F24BFA3EB4E
:101D9800510340EA5C00B3EB910F24BFA3EB91031E
:101DA80040EA9C00B3EBD10F24BFA3EBD10340EA78
:101DB800DC001B0118BF5FEA1C1CE0D1FD2A3FF6BE
:101DC80050AF8B4240EBC25008BF20F00100704773
:101DD8000CF0004C4CEA50207F32C2BFD2F1FF0316
:101DE80040EAC250704740F400004FF00003013A47
:101DF80037E792F0000F00F0004C02BF400010F4EB
:101E0800000F013AF9D040EA0C0093F0000F01F0FE
:101E1800004C02BF490011F4000F013BF9D041EA20
:101E28000C0195E70CEAD15392EA0C0F08D1420253
:101E38007FF47DAF93EA0C0F7FF470AF084676E726
:101E480093EA0C0F04D14B023FF44CAF08466EE7FF
:101E580030F0004C18BF31F0004CCAD130F00042CD
:101E68007FF45CAF31F000437FF43CAF5FE700BF25
:101E78004FF0FF3C06E000BF4FF0010C02E000BF4E
:101E88004FF0010C4DF804CD4FEA40024FEA4103F0
:101E98007FEA226C18BF7FEA236C11D001B052EAA6
:101EA800530C18BF90EA010F58BFB2EB030088BF6C
:101EB800C81738BF6FEAE17018BF40F001007047DB
:101EC8007FEA226C02D15FEA402C05D17FEA236CBD
:101ED800E4D15FEA412CE1D05DF8040B704700BF04
:101EE800844608466146FFE70FB5FFF7C9FF00289B
:101EF80048BF10F1000F0FBD4DF808EDFFF7F4FFD4
:101F08000CBF012000205DF808FB00BF4DF808ED6C
:101F1800FFF7EAFF34BF012000205DF808FB00BF8F
:101F28004DF808EDFFF7E0FF94BF012000205DF8B1
:101F380008FB00BF4DF808EDFFF7D2FF94BF012062
:101F480000205DF808FB00BF4DF808EDFFF7C8FF5B
:101F580034BF012000205DF808FB00BF42000ED20C
:101F6800B2F1FE4F0BD34FF09E03B3EB126209D4CC
:101F78004FEA002343F0004323FA02F070474FF082
:101F88000000704712F1610F01D1420202D14FF0F7
:101F9800FF3070474FF00000704700BF00F026F890
:101FA8000C4880F30888002103E00B4B5B58435032
:101FB80004310A480A4B42189A42F6D3094A02E009
:101FC800002342F8043B084B9A42F9D313F080FEF1
:101FD8007047000000C00020A8AF020800000020E1
:101FE800180E0020180E0020482F00207047FEE72A
:101FF80010B586B0002301244FF46022114801A9CE
:1020080001938DF80930039204938DF808408DF8F8
:1020180014401CF0CDF80B4821461CF0EFF8094895
:102028001CF0F6F807481CF0F8F80028FAD1054823
:102038001CF0F7F803481CF0F9F80028FAD106B0AC
:1020480010BD00BF00240140014610B50D48012213
:1020580003231CF0F9F80B4801211CF0EBF87F2052
:102068001CF028FF074802211CF038F90028F6D098
:10207800044802211CF038F90248BDE810401CF061
:102088002AB900BF002401400C4A0C2303FB01239A
:1020980010B59C880CB9588010BD5B8803F11304F7
:1020A800844204DA142B07D9133B834204DC0C2343
:1020B80003FB012102238B8010BD00BF581A0020AA
:1020C8000A4B10B500241C7021464FF48072084852
:1020D800FEF760F9074B43F6DE301C70064B1C70A8
:1020E8000DF0ECF8054B187010BD00BF081000206B
:1020F80010110020271200201312002015120020B2
:10210800074B1978013101F01F011970054B1A7836
:102118008A4203D1013202F01F021A70704700BFD1
:10212800131200202712002010B50A4B0A4A03EBAD
:10213800C0000A4B1978036802EBC10442F8313039
:102148004368002163600822FEF724F9BDE81040C7
:10215800FFF7D6BF0C10002010110020131200202A
:102168002DE9F3479846474B1746DA78054602F0BB
:102178002002D2B20E46BDF82890002A7AD1B8F1D2
:10218800000F0AD19B7803F04003DBB2C3B900F01B
:102198007F0000F56E50633009E0B8F1010F09D1F6
:1021A8009B7803F04003DBB2BBB949F2D8400DF08D
:1021B80085F8C4B2002C5FD0B8F1000F09D100E057
:1021C800012405F07F0149000DF1060001F5715168
:1021D8000CE0B8F1010F0CD100E04446E90101F52B
:1021E8000A41D8310DF1060001EB460102220DF03B
:1021F80076F8BDF9063013B9B8F1000F3ED0B9F141
:10220800000F06D1204B93F800A0FFF779FF1F4B72
:1022180008E01F4B93F800A00AF1010202F01F0228
:102228001A701C4BB8F1000F12D1BDF8061040F619
:10223800B8326DB212EA250538BF4FF47A756D18B9
:1022480003EBCA0223F83A509470D670177109E06C
:10225800B8F1010F06D1BDF8061003EBCA0223F846
:102268003A10947003EBCA0383F80580A3F806902C
:10227800012004E0002002E0204600E04046BDE8DE
:10228800FC8700BFA8210020131200201011002095
:10229800071000200C10002001228240094B0A4937
:1022A8001B78D2B2097808E0084800EBC3008078B0
:1022B800024205D1013303F01F038B42F4D1FF23FF
:1022C8001846704727120020131200201011002012
:1022D800F0B500EB800101F56E51314F042285B055
:1022E800304836310CF0FBFF2F4C3B7804EBC3022F
:1022F80056791EBB2B4D31222A7107326A7134F987
:10230800331001A8343A05F08FFD3B7802A804EB9E
:10231800C3031979022205F087FD3B780DF10A0005
:1023280004EBC304E178032205F07EFDA81D01A992
:102338000922FEF705FB2E740F250CE0012E0AD1A9
:10234800184A322111710531517134F8333008259A
:10235800190AD1719371002314481A4612E010F833
:10236800011FA1F13004E4B2092C04D8E318302984
:10237800DBB203D004E037395B1800E00A33DBB284
:102388000132D2B2AA42EAD10F21B3FBF1F108011E
:10239800411A5B1A0348C3F10F03835405B0F0BD1B
:1023A8000D11002016120020101100201512002017
:1023B8002DE9F3415E4B04461B7843B15D4B1B7816
:1023C80003F02403042B02D1002900F0AD805A4BFE
:1023D8005A4F1B78002B00F09280594821461BF079
:1023E80097F88046002840F08A803B191B7E2D2BE9
:1023F80001D0532B2DD1534E3578F5B10DF066FA37
:10240800611C034630B1337893201E3300930122B8
:10241800002302E0009001229320FFF7A1FE0DF0B7
:1024280055FA014628B1337813201E330093002152
:1024380001E0009013200A465EE0611C012293200F
:102448002B460095FFF78CFE0095132029462A4657
:1024580052E0542B05D10090611C94200122434680
:102468004BE0462B374D11D12E7866B10DF02EFA80
:10247800611C034620B12B789A201E33009314E088
:1024880000909A2018E000969A202CE02E7826B327
:102498000DF01CFA0346611C04F11C0043B12B78B3
:1024A80060F07F001E330093C0B20122434604E06F
:1024B80060F07F000093C0B20122FFF751FE0DF0DB
:1024C80005FA21B2024628B12B7803201E33009367
:1024D800002211E0009003200EE004F11C0060F0DF
:1024E8007F000096C0B2611C01223346FFF738FE18
:1024F80000960320214632460123FFF731FE10489B
:1025080021463F191AF0EEFF3B7E542B0CD8532B73
:1025180003D22D2B01D0462B06D10B48214602B001
:10252800BDE8F0411AF0E9BF02B0BDE8F08100BF94
:102538000A1000203C13002014120020EC1900207F
:1025480042130020541300204013002037B5114BCC
:1025580004461B780D4693B10F4821461AF0D8FF60
:10256800034660B9012D04F1010103D100902A4608
:10257800812002E0009001229820FFF7F1FD21461A
:1025880005481AF0AFFF0548214603B0BDE83040C2
:102598001AF0B3BF14120020421300202D1200209D
:1025A800024B1A7842F001021A707047F1130020AA
:1025B80008B50C4B1A780C4B03EBC203597921B1BF
:1025C80001290CBF0921002100E0102140221346F7
:1025D800064805F04DFA064B1A7842F002021A70C6
:1025E80008BD00BF0D110020101100201612002098
:1025F800F1130020034B1A7802F0F8026FF3C302BC
:102608001A707047F1130020024B1A7842F0040246
:102618001A707047F1130020024B1A7842F0080232
:102628001A707047F113002038B5114B1C7814F05C
:10263800010502D1FFF7B4FF05E004F00405EDB28F
:102648001DB9FFF7E1FF284638BD04F00805EDB2D3
:1026580015B9FFF7E1FFF6E704F00204E4B21CB98C
:10266800FFF7A6FF204638BDFFF7C4FF012038BD9D
:10267800F1130020014B1878704700BF08100020A4
:1026880030B50F4B85B01B780546BBB90D4C227889
:10269800024112F0010F11D0FF2201930121431CC6
:1026A800009202933C200B46FC3A0CF07BFE01237F
:1026B80013FA05F5237823EA0505257005B030BD22
:1026C80015120020111200202DE9F843134A0023A7
:1026D8001370134A1678134A11789046B14219D0EC
:1026E800114D2A78072A88BF2B7095F800902C780E
:1026F8000D4F2046FFF7D0FDFF280CD10134E4B27E
:10270800072C3C7001D900233B702B784B45EED148
:1027180088F80060FF242046BDE8F88308100020F0
:1027280027120020131200200E11002001218140E1
:1027380010B5C943C9B20023094A9A1894780833D6
:1027480001EA0404B3F5807F9470F5D1FFF798FF90
:1027580043F6DE300CF0B2FD024B187010BD00BF1E
:1027680010110020151200202DE9F0418B4E05466E
:1027780033788B4C13B12378834204D043F6DE3090
:102788000CF09CFD30702570864C2378072B00F2E6
:10279800E680DFE813F008002000330051005A00FB
:1027A80070008B00B500804B1E221A702846FFF778
:1027B80073FD7E4BFF28187000F0D5801AF000FAE0
:1027C8007B4B002093F8702042F0010283F87020C0
:1027D800784B187065E0744B1B78002B00F0C380B1
:1027E8001AF03AFB012840F00D81237814220133B6
:1027F8002370714B01381A70BDE8F0816A4B1B7861
:10280800002B00F0B0806C4E307808B901234AE004
:102818001AF022FB022804D01AF01EFB032840F00D
:10282800F1801AF0CDF923780422013323701D2397
:102838003370624B1A70E5E05B4B1E221A70284613
:10284800FFF746FD237801332370574B1B78002B85
:1028580000F08980584B1D78002D40F0D38010205F
:10286800FFF7E2FE002800F0D180237828460133E4
:102878002370BDE8F0814C4B1B78002B73D005F01A
:1028880061F9002800F0C2804B4B7D221A70494B39
:1028980000201870464B93F8702042F0010283F82C
:1028A8007020237801332370BDE8F0813E4B1B78FC
:1028B800002B58D01AF0D0FA01283F4F03D01AF055
:1028C800CBFA03280DD1012212FA05F53C4B1A78F0
:1028D80022EA05051D7064233B70237801332370B9
:1028E80090E03878002840F08D80344A0323237024
:1028F8001378013BDBB21370002B34D0BDE8F081B4
:102908002B4B2D4F93F86A3013B13B78002B79D1BC
:1029180000233B700133AB40244A2A481178904683
:1029280000EBC10090F802E02EEA030383703BB984
:10293800254B1A788A4203D1013202F01F021A701D
:102948002846FFF7A9FC1D4B0422FF2888F8000041
:102958001A703FD0032323701A333B7052E00020D3
:102968002070BDE8F081FFF745FE002323701AF0C0
:1029780027F93378013BDBB2337033B1134B9B78C3
:1029880003F04003DBB2002B3FD02846FFF7CEFE12
:102998000F4B1A7801321A7031E000BF151200206F
:1029A8000B10002008100020121200200D1100202A
:1029B800A623002009100020061000201012002075
:1029C800111200201011002027120020A821002039
:1029D8000E1100200E4B9A7802F04002D2B21AB1C2
:1029E8001A6842F400021A60FFF704FE1AF0E8F8C9
:1029F8000023237043F6DE300CF060FC3070FF20BB
:102A0800BDE8F0810020BDE8F081FF20BDE8F0813D
:102A1800A8210020044B1A780AB1013A1A701B78D1
:102A28000BB9FFF783BE704715120020044A054B07
:102A380010781B7803EA501000F00100704700BFBF
:102A4800A82100202D130020044B054A1B7810787C
:102A5800C3F3400303EA1010704700BF2D13002092
:102A6800A8210020034B044A1B78D078C3F38003C5
:102A7800184070472D130020A8210020044B054A58
:102A88001B78D078C3F3C00303EA5000704700BF37
:102A98002D130020A8210020044B054A1B78D0786C
:102AA800C3F3001303EA9000704700BF2D13002002
:102AB800A8210020044B1878044BDB785B005BB23C
:102AC800DB1103EAD01070472D130020A821002045
:102AD8002DE9F041154E0024B04620E02046294655
:102AE80017F0C0F990B1F35DFF2B0FD04FF4A0732E
:102AF80063430A2202FB053318F80330DB0905D0CB
:102B08000B4B1878C0F30010BDE8F08101350A3787
:102B1800202DE3D10134022C06F5A07602D000273F
:102B28003D46DBE70020BDE8F08100BFF22400202D
:102B38002D13002008B516F0DBFD034B1B7800EAC7
:102B4800931000F0010008BD2D130020044B054A26
:102B58001B78D078C3F3401303EAD000704700BF56
:102B68002D130020A82100202DE9F84FFFF75EFF64
:102B78008146FFF769FF8246FFF774FF8346FFF738
:102B88007DFF8046FFF788FF0446FFF7A1FF054653
:102B9800FFF7DCFF0746FFF7CDFF0646FFF78AFF82
:102BA8004FEA8B0343EA4A0343EA090343EAC803AB
:102BB80043EA471343EA861345EA040443EAC01389
:102BC800E0B243EA0010BDE8F88F0000044B9878A3
:102BD80000F00F00A0F10203584240EB03007047D9
:102BE8004C120020044B987800F00F00A0F101026D
:102BF800504240EB020070474C120020044B98787A
:102C080000F00F00A0F10301484240EB01007047BB
:102C18004C120020054B987800F00F00A0F1060C2C
:102C2800DCF1000040EB0C00704700BF4C120020A4
:102C3800514AF0B513781446012B29D003D3022B3F
:102C480040F098805EE04D484D4B047819786FF35A
:102C5800C304047001F0F80158786FF3C3011970C8
:102C680000F08001C9B2002900F0848001211170B0
:102C78009C78062204F00F04544302464148005D44
:102C880060F306025A701A7861F302021A70F0BDF6
:102C98003B494D780B4625F07F00002838D00A784C
:102CA80002F00802D2B222B9344A117841F0080180
:102CB80011709A7802F00F02012A04D12F4A117874
:102CC80041F00101117015F07F0F53D119789E78EA
:102CD80001F00700062206F00F0602FB0606294F40
:102CE8005D78BE5D013066F3060500F007005D7093
:102CF80090FBF2F502FB150262F302011970022340
:102D08002370F0BD1E494D780B4625F07F0028B989
:102D18008B7860F303038B701070F0BD174A11783D
:102D28006FF3C3011170997801F00F01012903D1E4
:102D380011786FF30001117015F07F0F1AD119780F
:102D48009E7801F00700062206F00F0602FB060631
:102D58000C4F5D78BE5D013066F3060500F0070094
:102D68005D7090FBF2F502FB150262F30201197027
:102D780001232370F0BD00BF611200202C12002037
:102D88004C1200201CEF010808B543F6ED200CF0AA
:102D980095FA014B187008BD2B120020014B1870D2
:102DA800704700BF30130020024B1A5C6FF3030218
:102DB8001A5470477512002070B50C46C10001F511
:102DC800CC411248683102220CF089FA00250F48DC
:102DD8002946EEB21AF09CFB98B10D4B2278EB5CB9
:102DE8001A420ED13046FFF7DFFF294609481AF08C
:102DF80084FBF608074B06F5CA40A830995D0CF02D
:102E080053FA01350C2DE2D170BD00BF32130020FA
:102E1800661200204F12002038B546F2F0554024C3
:102E28002046FFF7C1FFA5F5CA43094AB03BD15C6C
:102E380011F0100F06D06FF30411D1542846002169
:102E48000CF032FA0134E4B20135B82CE8D138BDBF
:102E5800751200207FB58D4B05461B78002B00F0BE
:102E68000C818B4E325C541C04F00F0464F3030293
:102E78000B2832542AD8002C00F0048101339C42DC
:102E880040F0FD80D3B26FF303033354814BC40881
:102E98001B1993F84C2000F0070352FA03F313F0C0
:102EA800010F40F0EE8029467B481AF01BFB7A4B55
:102EB80004F5CA40195DA83001240CF0F5F92D1964
:102EC80002230093019402951820D0E03F2840F295
:102ED800D680002C00F0D68001339C4240F0CF8091
:102EE800335C01216FF30303335400F5CA40B0305B
:102EF8000CF0DAF9735D43F010037355A5F1400344
:102F0800DBB2032B07D8042200920133023201926C
:102F18000293192031E0A5F14803DBB2032B0CD84A
:102F28000422009201330332019202931A200121F4
:102F3800043A0B460CF036FAA3E0502D07D10423CF
:102F4800009301240333019302941B208FE0572D33
:102F580007D1042300930124033301930294212011
:102F680085E0A5F15B03DBB2012B09D804220092AE
:102F7800013302320192029322200121033AD8E759
:102F88005D2D04D1042300930193043B06E05E2DDC
:102F980007D10423009301330193053B029328468C
:102FA8004FE0A5F15F03DBB21F2B09D80422009282
:102FB800013392180192029333200121053AB8E7B0
:102FC80005F16103DBB2032B07D804220092013319
:102FD8000332019202935F20A9E705F15903DBB29E
:102FE800012B07D804220092013303320192029385
:102FF80060209CE7AA2D07D1042300930124043BF9
:1030080001940293612032E0A92D07D10423009393
:10301800023B0193023B0293622012E0AC2D08D1DF
:10302800042300930322043B0192029363200121AD
:103038007FE7AB2D08D104230093043B019302934F
:1030480064200121032274E7AD2D07D104230093E6
:103058000124023301930294682008E0B12D10D1B5
:103068000423009301240233019302946A20214629
:10307800032223460CF096F904E01C4602E00024E3
:1030880000E00124204604B070BD00BF000000200D
:1030980075120020EC1900204F120020024B185C1A
:1030A800C0F30010704700BF75120020F8B5002467
:1030B80006460F460470447046F268653B78234123
:1030C80013F0010F08D02946064802220CF007F930
:1030D800304604491AF0CBF901340835042CEDD1F7
:1030E800F8BD00BF36130020024846F2A85102225C
:1030F8000CF0F5B84F12002070B5044600F56A5080
:1031080044300CF0DBF80B4D06462B7813F0010F1A
:1031180002D1CC201AF0E4FF2B8843F001032B8066
:10312800054B1E55054B13F8242042F0010203F805
:10313800242070BD3C1300204212002031120020D0
:10314800024B185C084100F001007047661200202D
:1031580070B505460024094BE0B2E618E35C4BB1B4
:103168002946FFF7EDFF28B10023337004482146B4
:103178001AF0C3F901340C2CEDD170BD46130020B0
:103188004812002038B5054600242846E1B2FFF76A
:10319800D7FF10B1044BE35C23B90134042CF4D1FC
:1031A800002038BD012038BD4212002038B5054640
:1031B8000CF08CFBA0B100242846E1B2FFF7C0FF59
:1031C80040B1084B13F8243013F0010F02D0064B1E
:1031D800E35C23B10134042CEED1002038BD01207A
:1031E80038BD00BF3112002042120020F8B5114846
:1031F80000210C22FDF7CEF846F26865002401276D
:103208000D4829460222A7400CF069F8FFB20026B3
:10321800094831461AF07CF920B1064BF25C47EABE
:103228000202F25401360C2EF2D101340835042C76
:10323800E5D1F8BD66120020361300202DE9FF41C4
:1032480000263446B0461A4B1B78234113F001027E
:10325800184B23D0184F1D5D17F82430A84538BFE8
:10326800A84613F0010F1AD0CDB965F3000307F88B
:10327800243023B20122F71902935B2029462B46FA
:10328800009201950CF08EF87B78B878F97818439D
:10329800621C2B460095FEF763FF00E01A550134C7
:1032A8000436042CCFD1054B83F80080BDE8FF819C
:1032B8002B12002042120020311200202A12002076
:1032C80010B50C4B1B78A3B10B4B1B788BB10024AA
:1032D8000A4821461AF01CF940B1094821461AF05B
:1032E80017F918B920460121FFF762F801340C2CB0
:1032F800EED110BD141200200A1000204013002047
:103308004A1700202DE9F043364D374A2B8800260E
:103318006FF386136FF3C4032B80344B344F85B09F
:1033280016701E709146984617F8013B5BB32A78D1
:10333800D20052B243EAA2122B880C2E62F3C403C5
:1033480043F040032B801ED000243046E1B2FFF743
:10335800F7FEA8B117F8013C13F0010F06D00122BF
:10336800A24099F800100A4389F8002013F0020FD0
:1033780006D00123A34098F80020134388F80030B2
:103388000134042CE1D10136F6B20D2ECCD12B78C4
:1033980003F04004E4B20CBB03F02403042B12D165
:1033A800FFF78EFFFF23009340202146012223468A
:1033B800019402940BF0F6FF802021460122234657
:1033C8000094FEF7CDFE2B8800226FF345136FF3B0
:1033D80082036FF3C4032B80064B1A7005B0BDE857
:1033E800F08300BF3C130020A0220020BD22002053
:1033F800541200203113002010B50024054821463E
:103408001AF086F808B9044BE05401340C2CF5D1B5
:1034180010BD00BF2E1300205412002070B51646B0
:103428000D46317804469DF81020002925D0002B40
:1034380023D012B111491AF00FF80121204609F0E2
:103448008FFD20462946324609F062FDACB10222C2
:1034580046F2A8510A480BF042FF214608481AF0E4
:1034680006F80749022246F2A8500BF032FF054839
:103478000349BDE870401AF01BB870BD3A1A002025
:10348800281200204F12002030B5064B04781D7812
:1034980024EA05040C7001781B7823EA01031370F1
:1034A80030BD00BF2B12002038B50A4D002415F896
:1034B800013F2D2B09D0532B07D0542B05D0462B79
:1034C80003D0054821461AF018F801340C2CEED127
:1034D80038BD00BF031A00204013002010B50D4866
:1034E80019F0B2FF00240C4821461AF011F860B117
:1034F8000A4BE3181B7E462B03D0542B01D02D2BEF
:1035080003D10448214619F0EDFF01340C2CEAD10F
:1035180010BD00BF6212002040130020EC190020EB
:10352800094A0A4B117831B1997801F00F018142AB
:1035380001D0002111709A7860F303029A705A78CA
:1035480042F080025A707047611200204C1200202D
:103558007FB5604B154604461A780E4600235E492F
:1035680011F8231011F0010F05D001219940C1F184
:103578000F0101EA02020133042BF0D1574B1A70F4
:10358800002C6FD014F0010F0AD0FF230121009303
:10359800FF3B0193029352200A460B460BF002FFB1
:1035A80014F0020F0AD0FF2301210093FF3B01937F
:1035B800029353200A460B460BF0F4FE14F0040F56
:1035C8000AD0FF2301210093FF3B0193029354206B
:1035D8000A460B460BF0E6FE14F0080F0AD0FF234C
:1035E80001210093FF3B0193029355200A460B46A5
:1035F8000BF0D8FE14F0100F0AD0FF23012100931E
:10360800FF3B0193029356200A460B460BF0CAFE75
:1036180014F0200F0AD0FF2301210093FF3B0193F0
:10362800029357200A460B460BF0BCFE14F0400FDD
:103638000AD0FF2301210093FF3B019302935820F6
:103648000A460B460BF0AEFE14F0800F0AD0FF239B
:1036580001210093FF3B0193029359200A460B4630
:103668000BF0A0FECEB100242846214619F050FFE9
:1036780060B1FF230093FF3B0193631C1BB2012140
:1036880002935A200A460B460BF08CFE2146284628
:10369800013419F032FF0C2CE6D110481049114AB8
:1036A800FFF7F2FE104B00221A7001320092063228
:1036B8000192083202920A490A4A084809F0DAFBDC
:1036C8000A4B3C2251201A7004B0BDE870400CF03F
:1036D800E3B900BF2B120020311200205C14002037
:1036E800C2140020B614002021140020411200202A
:1036F80010B5FFF739FA0446074819F0DCFED0F197
:10370800010138BF002104B929B1034A2046BDE8A8
:103718001040FFF71DBF10BD73120020054B03EBCF
:10372800D00393F84C3000F0070053FA00F000F093
:1037380001007047EC19002010B50C4B04461B78AB
:1037480013F001030FD0FFF71DFD68B10CF0BEF8B0
:1037580018B92046FFF7E2FF30B10548214619F0B5
:10376800C1FE012010BD184610BD00BF3C1300204B
:1037780073120020024B1878003818BF01207047D8
:103788004112002010B5034C04EB83035870997064
:10379800DA7010BD3112002010B50024094800214C
:1037A800001908220834FCF7F5FDB4F5807FF5D13F
:1037B800054A00231370054A002199520233AA2BA7
:1037C800F9D110BD0C10002007100020361500207C
:1037D8007FB5444B04461B780E46AA2B74D042484A
:1037E800214619F095FE054600286DD12046FFF7C1
:1037F800A3FF002869D13D48214619F089FE50B938
:103808003B48214619F084FE054620B92046FFF7BB
:1038180021FB002859D1374B1B7823B9364B1B782D
:1038280013F0010F08D1354BDB7803F02003DBB22E
:1038380013B9334B03221A73012E05D82B4821469E
:1038480019F066FE40B13FE0022E07D12848214614
:1038580019F05EFE10B137E0244800E02448214604
:1038680019F040FE2748214619F047FE022E12D1D2
:10387800012564194A20294603222B460096019502
:1038880002940BF08FFD0023182021462A4600934E
:10389800FEF766FC19E0012E09D102230093631C90
:1038A80002930196122031460322334609E07EB97D
:1038B800012102230093631802930191112003222E
:1038C8000B460BF06FFD03E00025284604B070BDE1
:1038D800012000232118024600930125FEF740FC31
:1038E800F3E700BF301300204F1200202D120020F4
:1038F800521300202B12002032150020A82100208E
:1039080054120020421300202DE9FF4704460D46BB
:103918006148214619F0FCFD8046002840F0B88037
:1039280021465D4819F0DEFD5C48214619F0E5FDA9
:103938005B4E0DBB012708F10208E31902934246CA
:10394800032039463B46CDF8008001970BF02AFD4D
:10395800327862B10BF0BAFF024630B13378404694
:103968001E33009321462A4604E0009000E00092AE
:10397800404621463B461CE0012D1FD1631C022214
:1039880002930E2029462B46009201950BF00AFD62
:1039980032788AB10BF09AFF024630B133780D20A5
:1039A8001E3300932146424602E000900D20214636
:1039B8002B46FEF7D5FB50E00092F7E7022D0AD11F
:1039C80001216318029314202A4643460095019169
:1039D8000BF0E8FC41E0032D3FD101272A464FF0C8
:1039E800020904EB070A4D2039463B46CDF8009002
:1039F8000197CDF808A00BF0D5FC3578EDB10BF0A8
:103A080065FF024630B1337848461E33009321469D
:103A1800424602E00090214648463B46FEF7A0FB9E
:103A28000BF054FF611C034620B133781A201E3373
:103A380000931FE000901A2020E021462A463B46CA
:103A480048460095FEF78CFB1A2051463A462B460D
:103A58000095FEF785FB38461BE033789BB10BF0E9
:103A680035FF0346611C04F11C0033B10C4B1B7875
:103A78001E3300930122002301E000930122FEF788
:103A88006FFB012005E0009304F11C00611CF5E7C1
:103A9800002004B0BDE8F087401300204213002046
:103AA80054130020064B1B1893F83C00492804D0F7
:103AB800452814BF0320022070470120704700BF2B
:103AC800EC1900202DE9F041244F00243C702448D3
:103AD800214619F01DFDE5B2224B002837D01E5DA6
:103AE8003B789E4200D303B93E70002E30D1314658
:103AF8001C480C22FCF74EFC1B4B1C4803EBD5035F
:103B080093F84A8004F0070348FA03F8214608F0BE
:103B1800010819F0FDFC68B9B8F1000F02D0284679
:103B2800022101E028463146FFF7EEFE28460BF059
:103B3800B3FF0DE0B8F1000F0AD12846FFF7B2FF36
:103B48000B4BDB7803F02003DBB20BB9094B18559C
:103B580001340C2CBBD1BDE8F08100BF5413002008
:103B68004812002046130020EC19002040130020C2
:103B7800A8210020541200202DE9F04F8F4B89B066
:103B88001B7813F0010F06D08D4B1A786FF386124D
:103B98001A7001F0E0B98B498B4A0B7810788B4D7D
:103BA800984218BF8A49137018BF0B706B7803F0DE
:103BB8000803DBB24BB143F6CF200BF07FFB844BFD
:103BC80018702B886FF3CB232B80824B1B78AA2B82
:103BD80008D18149AA3B0B702B8843F080032B80C6
:103BE80000F036BE6A78794B02F01002D2B27B4CF4
:103BF8009AB11A886FF30C321A80794B1B7823B963
:103C0800784B1B7813F0010F07D1E37803F02003FA
:103C1800DBB213B9744B03221A732368734F6FF323
:103C2800186323603A7802F00202D2B232B96A49C4
:103C38004A781AB1694A43F080731360E67816F03F
:103C4800010647D05D20FFF729FA002859D16B7883
:103C5800DFF8788103F00203DBB22BBB5D30FFF79E
:103C6800F9F8064600BBB8F80030012143F40073A8
:103C7800A8F80030042303220093019302900B4616
:103C88000D200BF08FFB45200BF006FF314601227B
:103C980033460D200096FEF763FA09203146324676
:103CA80001230096FEF75CFA6B7803F00203DBB29F
:103CB8003BB34B4B1B7823B94A4B1B7813F0010FCE
:103CC8001FD1E37803F02003DBB2D3B9464B0322BC
:103CD8001A7316E06B7803F00203DBB26BB131465E
:103CE800324601230A200096FEF73AFA8D20314623
:103CF800012233460096FEF733FA2B886FF34923E7
:103D08002B802368344A6FF35963236093787BB11F
:103D1800D37823B93B7813F00C0F05D108E03B7832
:103D280003F00C03042B03D0236843F000732360D3
:103D3800E17801F00201C9B2002959D05E20FFF7ED
:103D4800ADF9002863D16B78204F03F00403DBB290
:103D5800EBB95E30FFF77EF80646C0B93B88012113
:103D680043F480633B8004230093013303220193CF
:103D780002900B4617200BF015FB45200BF08CFE2C
:103D88000D203146012233460096FEF7E9F96B789B
:103D980003F00403DBB2002B39D0114B1B7823B995
:103DA800104B1B7813F0010F31D1E37803F0200397
:103DB800DBB263BB0C4B03221A7328E05D140020AE
:103DC8000423002034130020351300203C13002066
:103DD8005513002030130020180E0020A8210020C1
:103DE8002B1200203215002054120020E819002060
:103DF8006B7803F00403DBB22BB18D2001220B4654
:103E08000091FEF7ADF92B886FF38A232B80236886
:103E1800DFF8CCB26FF3DF7323605F2307930026CC
:103E2800D94695E03046394616F01CF8002870D07F
:103E38001BF80A30FF2B6CD04FF4A0727243A8F124
:103E48005E03DBB206930A2303FB072219F802E09C
:103E580009EB02035FEADE1E4FD02268404642F0BB
:103E6800004222600593FFF719F9059B00285BD1F2
:103E78001A7912F0040F24D14046FEF7EBFF059B98
:103E88008446F0B91A79322042F004021A71069970
:103E9800042300930291DB180121032201930B46AE
:103EA800CDF814C00BF07EFA4A200BF0F5FDDDF8D2
:103EB80014C00C20069901226346CDF800C0FEF715
:103EC8004FF94FF4A07373430A2202FB07334B44A4
:103ED8001B7913F0040F27D07C4B1B7823B97C4B3C
:103EE8001B7813F0010F1FD1E37803F02003DBB236
:103EF800D3B9784B03221A7316E01B7913F0040F19
:103F080007D08C20069901227346CDF800E0FEF711
:103F180027F94FF4A07373430A2202FB07334B447B
:103F28001A796FF382021A71013708F10108202FFC
:103F38005FFA88F80AF10A0A7FF474AF079A013623
:103F480002F12003DBB2022E0BF5A07B079305D00C
:103F58004FF0000ADDF81C80574663E723685E4986
:103F680023F080636FF39E7323600B79002B00F0BE
:103F7800DC83DFF870A1DFF870B14FF09F080026EE
:103F88001AF8011F3746013600294FD02368A8F1D7
:103F98005F0943F080635FFA89F923604846FFF7B9
:103FA8007DF8002858D14D4A122303FB072399783E
:103FB80011F0200F21D148460593FEF74BFF059BD2
:103FC8008146D0B99A78012142F020029A700423E0
:103FD80000930233019333B2032202930F200B465E
:103FE8000BF0E0F945200BF057FD0D204946012262
:103FF8004B46CDF80090FEF7B3F8384A122303FB7E
:1040080007239B7813F0200F26D0304B1B7823B959
:104018002F4B1B7813F0010F1ED1E37803F0200318
:10402800DBB2CBB92B4B03221A7315E02B4B1222B0
:1040380002FB07329278994612F0200F05D08D20A6
:1040480001220B460091FEF78BF8122303FB07931E
:104058009A786FF345129A701BF8011F002945D012
:104068002368404643F080432360FFF717F8002891
:1040780052D11A4B4FF0120909FB073999F802304F
:1040880013F0400F48D14046FEF7E4FE07460028EB
:1040980042D199F80230012143F0400389F80230F7
:1040A800042300930333019333B2032202934B207A
:1040B8000B460BF077F950200BF0EEFC192039462F
:1040C80001223B460097FEF74BF825E02B12002013
:1040D8003215002054120020180E0020552200200E
:1040E800F22400204D22002028220020A04B12227A
:1040F80002FB07329278994612F0400F05D09920BA
:1041080001220B460091FEF72BF8122303FB0797B9
:10411800BB786FF38613BB7008F10108042E5FFAB1
:1041280088F87FF42DAF934B1978002944D0236881
:10413800B12043F080632360FEF7B0FF00284AD126
:104148008D4B1A78984612F0400F1FD1B130FEF708
:1041580081FE0746D0B998F80030032243F04003A7
:1041680088F8003000960623033E31460193692003
:10417800334602960BF016F945200BF08DFC0D2006
:10418800394632463B460097FDF7EAFF98F800307B
:1041980013F0400F1FD0794B1B7823B9784B1B784D
:1041A80013F0010F17D1E37803F02003DBB293B9C2
:1041B800744B03221A730EE06F4E337813F0400FDE
:1041C80005D08D2001220B460091FDF7C9FF3378F9
:1041D8006FF3861333706C4B197800292DD0236840
:1041E800502043F080432360FEF758FF002833D166
:1041F800614E337813F0200F2ED15030FEF72AFE8F
:10420800074648BB3378032243F020033370042366
:10421800012600930333314601931020334602965A
:104228000BF0C0F850200BF037FC19203946324605
:104238003B460097FDF794FF0EE04F4E337813F09E
:10424800200F05D0992001220B460091FDF788FF29
:1042580033786FF3451333704C4B1978002945D0E8
:104268002368AD2043F080632360FEF717FF002822
:104278004BD1474B1A78984612F0400F20D1AD30F9
:10428800FEF7E8FD0746D8B998F80030012643F054
:10429800400388F800300423009302333146032298
:1042A80001936720334602960BF07CF845200BF00B
:1042B800F3FB0D20394632463B460097FDF750FF89
:1042C80098F8003013F0400F1FD02C4B1B7823B9FF
:1042D8002B4B1B7813F0010F17D1E37803F0200361
:1042E800DBB293B9274B03221A730EE0284E3378BA
:1042F80013F0400F05D08D2001220B460091FDF7E9
:104308002FFF33786FF386133370224B1978002907
:1043180042D02368572043F080432360FEF7BEFE57
:10432800002848D11A4E337813F0200F43D1573064
:10433800FEF790FD074600283DD13378032243F06D
:10434800200333700423012600930333314601937D
:104358001F20334602960BF025F850200BF09CFBEB
:104368001920394632463B460097FDF7F9FE22E010
:10437800552200201A2200200B2200202B12002098
:104388003215002054120020AC210020DE2100202C
:10439800F0210020E32100209D4E337813F0200FF8
:1043A80005D0992001220B460091FDF7D9FE3378FC
:1043B8006FF3451333704FF000094FF0A70AC84652
:1043C8004E46944B08F10108F15C00294DD0236852
:1043D800AAF14C0B43F080635FFA8BFB23605846CD
:1043E800FEF75CFE002853D1162373438A4FFA5C0C
:1043F80012F0200F22D158460593FEF72BFD059B9E
:104408008346D8B9FA5C012142F02002FA54042309
:104418000093023301930FFA88F3032202932020BA
:104428000B460AF0BFFF45200BF036FB0D2059461E
:1044380001225B46CDF800B0FDF792FE16237343C8
:10444800FB5C13F0200F23D0744B1B7823B9744BFB
:104458001B7813F0010F1BD1E37803F02003DBB2C4
:10446800B3B9704B03221A7312E0162373436A4FD1
:10447800FB5C13F0200F05D08D2001220B46009124
:10448800FDF76EFE16237343FA5C6FF34512FA5478
:10449800654BF15C002936D02368504643F08043D1
:1044A8002360FEF7FBFD002842D15B4B4FF0160B53
:1044B8000BFB063B9BF8013013F0200F38D1504618
:1044C800FEF7C8FC0746002832D19BF801300121CD
:1044D80043F020038BF80130042300930333019346
:1044E8000FFA88F3032202934C200B460AF05AFF76
:1044F80050200BF0D1FA1920394601223B4600978B
:10450800FDF72EFE14E0444F162303FB06735B7879
:1045180013F0200F05D0992001220B460091FDF7DA
:104528001FFE162303FB06777B786FF345137B701A
:104538003E4B1B78002B00F08F803D4B364FF35CD1
:104548001622002B76D002FB06F3FA5C07EB090172
:10455800C2F3801BBBF1000F1BD142F04002FA549A
:1045680078234B8004230093DB18012101930FFA71
:1045780088F3032202932E200B460AF013FF4620ED
:104588000BF08AFACDF800B00920414601225B46BB
:1045980060E0B1F9021029BB5FEAD21B22D143F6D1
:1045A800DE2005930AF08AFE059BD8B1FA5C01214A
:1045B80042F08002FA5404230093DB1801930FFAA7
:1045C80088F3032202932F200B460AF0EBFE4720C4
:1045D8000BF062FA0920414601225B46CDF800B093
:1045E800FDF7BEFD16237343FB5CDB0934D00B4B90
:1045F8001B7823B90A4B1B7813F0010F2CD1E378F1
:1046080003F02003DBB23BBB064B03221A7323E003
:10461800F021002026220020B22100202B120020A9
:1046280032150020541200201C220020EA2100200C
:10463800E52100207243B95C11F0400F0CD063F300
:10464800861163F3C711B9544F447B8089200093C6
:1046580041460122FDF784FD01360AF1010A022EC6
:1046680009F116095FFA8AFA7FF4ABAEDFF8C4A342
:104678004827023E1AF8011FB0460136002937D0F4
:104688002368384643F080432360FEF707FD00287F
:1046980047D14FF01C0909FB08F9DFF884B31BF870
:1046A800093013F0200F3CD13846FEF7D3FB804683
:1046B800002836D11BF80930012143F020030BF8FC
:1046C8000930042300930333019333B20322029386
:1046D80013200B460AF066FE50200BF0DDF9192076
:1046E800414601224346CDF80080FDF739FD18E028
:1046F8001C2303FB08F3DFF8289319F8033013F0A1
:10470800200F05D0992001220B460091FDF728FDC6
:104718001C2303FB08F819F808306FF3451309F850
:1047280008300137042EFFB2A4D1A37803F00803A0
:10473800DBB2002B40F08C8048F68E24A4F50A47A3
:104748008E3FA248394618F0E3FE28B9A0483946FA
:1047580018F0DEFE002875D09E48394618F0D8FEBD
:1047680000286FD139469B4818F0BCFE20460AF055
:10477800A5FD994EC0B23070002863D00138C0B290
:10478800307009F013FF00285CD13078934E00F5A3
:104798006A506E300AF092FD914BC0B2E31813F8DC
:1047A8006A8C307000EA08083946884818F0B0FE6C
:1047B800DFF87CA2DFF82C9238B18548394618F02A
:1047C800A7FE10B99AF8003014E08148394618F06D
:1047D8009FFE38B17D48394618F09AFE10B99AF80C
:1047E800003004E09AF8003018EA030F02D023EAF8
:1047F800080801E048EA03087A487B4989F80080FC
:104808007A4AFEF741FE784879490FF057FB68B1BC
:104818000BF05CF850B9764808F0E4FB30B9012396
:1048280073487449704A0093FEF7F8FD002300931B
:104838000133019333786B4802936B496B4A6D4B94
:1048480008F018FB013448F69A239C427FF476AFAF
:10485800694E73786FF3C71373702B7803F0800277
:10486800D2B2002A00F0F08064490C78002C40F0A5
:10487800EB8003F02403042B12D1FEF721FDFF2364
:1048880000934020214601222346019402940AF015
:1048980089FD80202146012223460094FDF760FC13
:1048A8002B8800246FF3C7136FF3820364F3451357
:1048B80064F3410364F30003514A64F3492364F346
:1048C8008A2314702B804F4B1A7842F0C0021A705A
:1048D8005A7864F3C3025A70FEF7E6FD4A4818F0A6
:1048E800B3FD4A4818F0B0FD494818F0ADFD0D2257
:1048F80048482146FBF74EFD474B9A7802F0BF0225
:1049080064F345129A701A7D02F0BF0264F34512EF
:104918001A7593F8262002F0BF0264F3451283F853
:10492800262093F8382002F0BF0264F3451283F87A
:1049380038203A4B1A7802F0DF0264F386121A70B4
:10494800374B1A7864F345121A701A7F64F34512CC
:104958001A7793F8382064F3451283F8382093F8CF
:10496800542064F3451283F854202E4B1A7802F031
:10497800DF0264F386121A702B4B5A7864F34512DF
:104988005A701A7802F07F0264F345121A70DA7DC1
:1049980064F34512DA759A7D02F07F0264F34512DA
:1049A8009A7511E04FF4A07262430A2101FB0322B9
:1049B8001E4901338A181179202B6FF38201117176
:1049C800F0D10134022C37D00023EBE7E0190020A6
:1049D800E2190020E419002072120020801400203F
:1049E800EC8FFF1F5C140020C2140020B6140020B6
:1049F8002F120020211400204C120020180E002035
:104A08003113002004230020521300202D1200200F
:104A18004812002054120020552200200B220020AA
:104A28001C230020F0210020B2210020F2240020C5
:104A38002B1200200622002004226E480021FBF7DA
:104A4800A9FC6D4B00221A706C4F3878002843D1AE
:104A58002A786B4B02F00202D2B2B2B1694A51789D
:104A680060F3C30151701A88CA3042F080021A807C
:104A780019F036FBC62019F033FB19F07BFB0BF05D
:104A880097F8FEF7C9F9FEF787FE5F4A2B88117879
:104A98006FF341036FF300016FF3000311705B487C
:104AA80000210C222B80FBF775FC594818F0CCFC30
:104AB800584818F0C9FC584818F0C6FC574818F070
:104AC800C7FC04224B480021FBF764FC4A4A002338
:104AD8001370534A137067E02C7804F00203DBB2BA
:104AE80093B914F001040FD1494818F0ADFC3B7894
:104AF800E0B2234113F0010F03D0FEF7FDFA0AF0EC
:104B0800DBFE0134042CF2D12B783D4C13F0010F5D
:104B180022D0FEF7EDFD238843F002032380FEF741
:104B28008DFB354B1F78A7B9CA2019F0D9FACD20CB
:104B380019F0D6FA23883B4867F300032380324BE9
:104B48001A7842F001021A7018F07EFCFEF764F938
:104B580002E00120FEF7E4FC2B7803F00202D2B257
:104B680012B32F4A12782AB113F0010F02D1022092
:104B7800FEF7D6FCFEF7A6FF2B49264818F082FC64
:104B88002449254818F068FCFEF7A8FC2149274865
:104B980018F062FC2649254818F069FCFEF72CFC41
:104BA8001E481C4918F084FC22481F4918F054FC80
:104BB800214A13780BB9FEF7A5FB737803F080033D
:104BC800DBB2002B40D12B7803F02403042B06D151
:104BD80043F6EC200AF072FB08B1062032E0FEF73B
:104BE800C9FD08B105202DE00BF0B6F830B303205D
:104BF80028E000BF421200202A1200202B120020B9
:104C08003C130020042300202C120020461300200F
:104C1800511B00202E1300204812002044130020AE
:104C280054130020731200204F120020401300205C
:104C38006212002046120020180E002001F016F81B
:104C480010B10420FEF76CFC684B1B781BB173781D
:104C58006FF3C713737066490B7813B1654B1B78F4
:104C68000BB32B78644E03F04403402B1BD1002474
:104C780021460122234620460094FDF771FAFF23BE
:104C880000933F20214602222346019402940AF011
:104C980089FB338843F6CE2043F0040333800AF0BF
:104CA8000DFB564B1870524A554E13789BB1514B19
:104CB800197881B92A78504B02F04002D2B252B129
:104CC8001A8861F382021A80337823B943F6CE201A
:104CD8000AF0F4FA30702A78474902F00400C0B2AA
:104CE800484B002873D002F02000C0B2434C68B192
:104CF8001A7842F0C0021A702378002B6BD10A8808
:104D080063F3820263F345120A8064E0D20052B270
:104D180019789211D2B241F0C00112F0010F197046
:104D280003D0C9B260F3C711197012F0020F03D093
:104D38001A786FF386121A701B78324A03F0400310
:104D4800DBB21BB9537843F00803537043F6CD2008
:104D58000AF0B4FAC0B20128307002D1284B0222FE
:104D68001A702478002C36D1FEF7AAFA21460122BF
:104D7800234680200094FDF7F3F9FF2301220093D6
:104D8800402021462346019402940AF00BFB2B880D
:104D980043F6CD2043F020032B800AF08FFA174BFF
:104DA8001870194B1C70134B1A780AB1013A1A7013
:104DB800197881B90E4A13786BB1FF23009341200B
:104DC80002220B46019102910AF0ECFA03E01A78EC
:104DD80042F0C0021A700AF06FFF0C4818F06BFB23
:104DE8000B4BB8B91A7860F3820216E00A2A002041
:104DF80034130020551300203C13002031130020E9
:104E08005312002004230020180E002064120020F2
:104E18002C1200201A7842F004021A706A784F485F
:104E280012F001011A780CBF61F3410242F002024C
:104E38001A704B4918F03CFB4A49484818F017FBD0
:104E48004648494918F013FB3378012B40F083801A
:104E58002B8800246FF349236FF38A232B80434B5D
:104E68000D221C7021464248FBF794FA414818F07D
:104E7800EBFAFEF719FB3B4818F0E6FA3A4818F047
:104E8800E3FA3D4B9A7802F0BF0264F345129A7038
:104E98001A7D02F0BF0264F345121A7593F82620B2
:104EA80002F0BF0264F3451283F8262093F83820F5
:104EB80002F0BF0264F3451283F838202F4B1A78AA
:104EC80002F0DF0264F386121A702D4B1A7864F32D
:104ED80045121A701A7F64F345121A7793F838202E
:104EE80064F3451283F8382093F8542064F345128C
:104EF80083F85420234B1A7802F0DF0264F38612F9
:104F08001A70214B5A7864F345125A701A7802F0D5
:104F18007F0264F345121A70DA7D64F34512DA757C
:104F28009A7D02F07F0264F345129A7511E04FF4FE
:104F3800A07262430A2101FB0322144901338A1833
:104F48001179202B6FF382011171F0D10134022CF9
:104F580001D00023EBE709B0BDE8F08FAA1E0020BE
:104F6800401300202D12002052130020531200205D
:104F78005412002048120020552200200B22002045
:104F88001C230020F0210020B2210020F224002060
:104F98002DE9FF4104460D460AF0B8FE9C4B1A194C
:104FA800177E9C4A98461278AA2A0AD1A7F14F037D
:104FB800DAB20B2A00F2AD81974A5BB29A4040F10F
:104FC800A881964B0C2202FB04335A7A0833AA4272
:104FD800C0F09F81FF2A00F09C81FF229A7008EBA5
:104FE800D40393F84A5004F007031D41502F05F0ED
:104FF800010500F0278114D8462F00F0F08009D869
:10500800412F00F08F80452F00F01C812D2F40F09C
:105018007E8130E0482F00F0BD804F2F40F077812F
:105028000DE0542F5BD005D8522F7BD0532F40F082
:105038006E8118E0A7F15903012B00F268817848C6
:10504800214618F065FA0646002840F062815A2F7A
:1050580001D1744809E1592F03D07248214618F04C
:1050680041FA714801E17148214618F051FA0646A3
:10507800002800F055816E48214618F049FA0028AA
:1050880040F0478121466A4818F02CFA69482146C1
:1050980018F033FA012602224DB1A4191420314622
:1050A80000230092019602940AF07CF938E1013459
:1050B8000A20294633460092019602940AF072F9B2
:1050C800214632462B4613200095FDF749F8122059
:1050D80029462A4633460095FDF742F820E1544810
:1050E800214618F015FA0546002840F012810126DD
:1050F8000222A7193E2031463346009201960297B4
:105108000AF050F9394632462B4614200095FDF72F
:1051180027F82146464818F0E5F92146454818F091
:10512800ECF9FDE04148214618F0F2F9064600285E
:1051380000F0F6804048214618F0EAF9002840F0CF
:10514800E8803B48214618F0E3F9064628B920468E
:10515800FDF780FE002840F0E380002D40F09E809F
:105168002046FEF7E9FA002840F0D5802046FEF7F1
:1051780099FC324BDB7803F02003DBB20BB9304BE0
:105188001855412F00F09880522F40F0C0802046DB
:10519800012193E02848214618F0BAF9002840F088
:1051A800B8802348214618F0B3F928B92046FDF7FE
:1051B80051FE002840F0AD80002D6FD12046FEF74B
:1051C800BBFA002840F0A7801C4BDB7803F02003D3
:1051D800DBB2002B70D11A4B03221A736CE016480D
:1051E800214618F095F9002840F093801048214690
:1051F80018F08EF9064628B92046FDF72BFE002840
:1052080040F08E80002D49D12046032156E000BF92
:10521800EC1900203013002000003080581A0020BC
:10522800E4190020E0190020E21900202E130020C4
:1052380040130020421300204F120020A821002014
:10524800541200203848214618F062F90646002812
:1052580066D03648214618F05BF90646002858D132
:105268002046FDF7A3FF20B13148214618F03AF94E
:1052780056E0502F28D12F4B1B782BBB2046FDF72B
:1052880081FF08BB2C48214618F042F9064620B990
:105298002046FDF7DFFD002842D115B12046022146
:1052A8000CE02046FEF7FEFB244BDB7803F02003DE
:1052B800DBB20BB9224B185520460021FEF724FB20
:1052C800061E18BF01262BE02046FDF75BFF0546AA
:1052D800F8B91C48214618F01BF90646D8B92046EB
:1052E800FDF7B8FD0746D8B91648214618F0FAF870
:1052F800154A135D8BB911494E7806F02006F6B2AF
:105308006EB908EB040393F83030135508E0012612
:1053180006E0002604E02E4602E03E4600E01E4677
:10532800304604B0BDE8F0812E1300204F12002053
:10533800731200205413002040130020A8210020DD
:10534800541200204812002046130020032210B5F2
:1053580005490648FBF7F4FA054806490222BDE864
:105368001040FBF7EDBA00BF02180020020200202F
:10537800070200200018002070B5804C237813F035
:10538800010F0AD00AF0AAFA38B100207C4902F0CD
:1053980025FD7C4B7C48197849E07C4D2B78002B07
:1053A8004AD00AF0A1FA002846D0794B1B7873B985
:1053B800784B5B7813F0010F09D00AF087FA30B9FF
:1053C800237803F02403042B01D10330B6E0724C98
:1053D800207870B10020714902F000FD2178012287
:1053E8006F4802F021FD00201021621C07F0C4F96B
:1053F80002E06C4902F0F2FC6B4C644807F00CFACE
:105408002378002B00F00A810AF068FA002800F0DF
:105418000581664966481022FBF792FA64485B21C9
:10542800FBF736F8002800F0F98021780130832254
:10543800BDE8704002F0F8BC5E4C237803F0050329
:10544800012B5DD100205C4902F0C8FC202110220C
:105458005A48FAF79FFF601D59490322FBF71AFAC9
:1054680040BBE01C57490222FBF714FA30B95648F2
:10547800FBF7E0F95449024650480BE0E01C534959
:105488000222FBF707FA40B95148FBF7D3F9504914
:1054980002464A48FBF754FA0EE0E01C4D49022246
:1054A800FBF7F8F930B94C48FBF7C4F94A4902460A
:1054B8004248EFE7FFF74AFF6278303AD3B2092B48
:1054C80000F2AC803B4B9B78303BDBB2092B00F2FF
:1054D800A5800A2101FB0231C9B2002900F09E8093
:1054E800334BFF220C291A7740F2988010295A77FB
:1054F80040F2948013299A7740F29080DA7770BD51
:10550800234E3378F3B9234B5B7813F0010F19D08E
:105518000AF0DCF9B0B9314817F0CDFF68B1304C6A
:10552800304B226802EA03033BB914F0E1F820B9D2
:10553800E37803F04003DBB223B10020BDE87040FC
:1055480008F02EBC337863B90AF0C0F948B1264B8D
:105558001B7803F00603042B03D02B780BB901202A
:10556800ECE7FEF707F910B10020204952E0204B84
:105578001C78002C40D01F494CE000BF3C13002091
:10558800996502082A120020FE0100202B12002033
:105598007E140020321500204114002070430208B8
:1055A800030200202E430208541300204F43020830
:1055B800F2010020FD1700207748020802020020AF
:1055C8009CAD0208A0AD0208DA480208A3AD0208A3
:1055D800B9480208A6AD02089848020864120020DB
:1055E800A82100203000000F2C1200209D55020831
:1055F8001D0E00209143020802F094FB02F086FB86
:1056080017F05CFA064BDB7803F02003DBB22BB112
:1056180004492046BDE8704002F0E0BB70BD00BF01
:10562800A821002089420208054B1B78D8019B015C
:105638005BB2DB1140B243EAE070C0B2704700BF12
:105648003C13002070B50E4686B041000122054685
:1056580001F5E97105A809F042FE0021012E8DF837
:1056680015104FF0FF0205F1010305D100920191D9
:1056780002930920FB3A04E00092019102931E2054
:1056880004220B4609F08EFE05A83F49FAF786FF6B
:1056980050B105A83D49FAF781FF28B105A83C4952
:1056A800FAF77CFF00286BD105A83949FAF776FF8D
:1056B800384B0446C0B95A78214642F010025A7055
:1056C800FF23022200930190FE3B02903D2009F047
:1056D80069FE4D200AF0E0F91220691C01222346D8
:1056E8000094FCF73DFD03E05A786FF304125A70FA
:1056F8000024294BE35C552B07D12846214611F09D
:105708005AFF10B1204611F045FF0134082CF0D1A2
:10571800002E32D121482249224AFDF7B5FE204801
:1057280021490EF0CBFBC0B10AF0D0F8A8B91E4849
:1057380007F058FC88B905A81349FAF72FFF012389
:1057480020B9009318481949154A04E01648174922
:10575800134A00933346FDF761FE154B10491D703F
:105768000023009305330193124B0E4A1B780B4814
:1057780002930E4B07F07EFB02E00F4B00221A70DB
:1057880005A806B070BD00BFD7AD0208A9AD0208D4
:1057980094AF020804230020A12200205C140020FA
:1057A800C2140020B61400202F120020211400205B
:1057B8008C230020801400204112002007B54100EE
:1057C800012201A801F5E97109F089FD002301A86A
:1057D80004498DF80530FAF7E1FED0F1010038BF31
:1057E80000200EBDD7AD020807B54100012201A86F
:1057F80001F5E97109F073FD002301A804498DF84A
:105808000530FAF7CBFED0F1010038BF00200EBDFD
:1058180066AF020870B5124B04461B181D7E89B18D
:105828001048214617F05EFEA5F15903DBB2012BA3
:105838000CD94F2D0AD0542D08D021460A4817F00C
:1058480051FE07E00748214617F057FE0648214653
:1058580017F053FE03480549BDE8704017F0FCBD3A
:10586800EC190020641200204A1200204413002082
:10587800024B1878C0F38000704700BF2C1200203C
:10588800024B1A8860F308221A8070473C130020E4
:10589800034B5878C00140B2C011C0B2704700BF76
:1058A8003C130020014B1878704700BF2B120020D2
:1058B80030B5457800230021C218917055FA03F1DC
:1058C80011F0010F08D0064959188C7C017804EAB8
:1058D8000101A14208BF91700133042BEBD130BD07
:1058E8004114002046F65221042209F0F8BC0000B9
:1058F80070B5104C0546102220460021FAF74AFDE3
:10590800002004F8010C2A78103414F8011FC3B2DF
:1059180091420BD152B10849013301F8013B1122E0
:1059280046F6A243BDE8704002F096B9013004285B
:10593800EBD170BD42140020411400202DE9F34141
:105948002D4C0722E37848F6242702FB0030C0B22A
:1059580000F50A40453009F0B1FC257964795FFA11
:1059680080F8002648FA06F313F0010F3AD03946BA
:10597800042201A809F0B3FC9DF804009DF8053045
:105988009DF806109DF8072000282BD0002929D063
:10599800002B27D0002A25D0934204D19C4221D144
:1059A80085421FD30FE09A4210D99C421AD39442E1
:1059B80018D89C4201D994421AD39C4201D18542FD
:1059C80016D294420ED18D420CD811E09C4201D1DE
:1059D80085420DD2944201D18D4209D99C4207D803
:1059E800944205D301360437082EBBD1002000E0CD
:1059F8000120BDE8FC8100BF7827002010B50446CF
:105A0800C00800F50A407D3009F058FC04F007048E
:105A1800C0B2204100F0010010BD70B5C50805F501
:105A28000A457D35044628460E4609F047FC04F031
:105A38000704C0B2012126B9A14040EA0101C9B258
:105A480002E0A14020EA01012846BDE8704009F0C3
:105A58002BBC0000F0B57C4B8DB0DE78042200EB47
:105A6800C606F6B2F10001F5EC4104A8AC3109F024
:105A780036FC764B764C1A78002304A9C95C312988
:105A880005D13039994041EA0202D2B205E0302905
:105A980003D12F39994022EA01020133042BECD1BA
:105AA80022706B486B496C4AFDF7EEFC694B1B781A
:105AB80013B9694B1B78F3B1664868490EF0FEF9D3
:105AC80068B109F003FF50B9644807F08BFA30B9A0
:105AD8000123624862495F4A0093FDF79FFC002357
:105AE800009302330193FD330293594859495A4AA6
:105AF8005B4B07F0BFF906EB0611002501F5F041F5
:105B0800257004A86C31082209F0E9FB2C462F46C1
:105B1800544B0135E35C542B36D104AB1B5D312B60
:105B280003D1204611F03EFC38B104AB1B5D302B8D
:105B38002AD1204611F036FC30B34FB9FF23009329
:105B48003420394604223B460197029709F02AFC83
:105B580004AF385D2146303811F032FC3B5D012737
:105B6800312B4FF0030305D100932BB20197029319
:105B7800352004E000932BB20197029336200021D0
:105B880004220B4609F00EFC0134082CC0D1B101E7
:105B980001F5F84104A82431202209F0A0FB083CB3
:105BA80004AD274615F8013BE6B20134302B03D18A
:105BB8003046FFF723FF38B115F8013C312B2CD1C3
:105BC8003046FFF71BFF40B34FB9FF230093342043
:105BD800394604223B460197029709F0E3FB15F882
:105BE800011C30463039C9B2FFF717FF15F8013CE0
:105BF8000021302B4FF0FF0305D1009323B2019110
:105C08000293372004E0009323B2019102933820D5
:105C180004220B4609F0C6FB0127202CC2D1124DE5
:105C28006B7803F00403DBB263B1203C2046FFF736
:105C3800E5FE38B90134E4B2202CF7D16B7860F373
:105C480082036B700DB0F0BD782700202B12002066
:105C58005C140020C2140020B61400202F1200206B
:105C680021140020A122002004230020014B1878D1
:105C7800704700BF1D0E00202DE9F04F4A4B00224F
:105C88001A704A4A85B01678002E40F08A80484B30
:105C98004FF4B468DA78997808FB02F24FF03C08C0
:105CA80008FB01285A78434F90441FFA88F8BA46EF
:105CB80065E03AF815303C24DAB2544304EB132477
:105CC8004C44A4B2042CEEB207D842F25A73984559
:105CD80003D904F51C546034A4B2444511D948F6DC
:105CE800442009F0EBFAC8EB0403834209DC324B89
:105CF8001A787B1993F83830934302D02A49012344
:105D08000B702B4AD378B3422BD142F26073B4FBA9
:105D1800F3F203FB12439BB243451CD1274B9B78FC
:105D280013F0090F3DD1264B5B7803F02003DBB25B
:105D3800002B36D1234B1A781BEA020F11D1019997
:105D4800009841EA02021A70FFF7F8FD48B9009876
:105D5800FFF780FE05E01B4B02991A7801EA020260
:105D68001A70013509F5B469072D1FFA89F9A0D110
:105D7800039E07370136042E0AF10E0A11D04FF0A0
:105D8800010B0BFA06FB5FFA8BF301936FEA0B0327
:105D9800F2B2DBB24FF00009009202934D4603962F
:105DA80087E705B0BDE8F08F1D0E002057130020CF
:105DB80078270020581300202B120020A82100204B
:105DC800122300205613002073B50C4601EBC001C6
:105DD800C9B2C90001F5EC410546042201A8AC315D
:105DE80009F07DFA104B002003EBC402121B521974
:105DF80082F8380001AA125C312A0AD101218140B7
:105E080003EBC402121B521992F83860314382F82E
:105E1800381001300428EDD101A93122302317F0C0
:105E28007FFBC0B27CBD00BF5813002000B501EB5A
:105E3800C001C9B2890189B001F5F8412431202295
:105E4800684609F04CFA202069463122302317F0C1
:105E580067FBC0B209B000BD07B501EBC001C9B20C
:105E680001EB011101F5F0416C310822684609F097
:105E780036FA082069463122302317F051FBC0B2A8
:105E88000EBD00002DE9F843002634462BE02146DC
:105E98002846FFF799FF214681462846FFF7C6FFA7
:105EA800214640EA09092846FFF7D6FF5FFA89F933
:105EB80049EA000010F0FF0F05D04046394602229B
:105EC80009F00DFA03E04FF0FF33A8F80030013570
:105ED800EDB20237072D08F10208D8D10134E4B237
:105EE8000E3E042C07D0054BC6F5EC47C6EB03085D
:105EF8003C370025CBE7BDE8F88300BF58130020E6
:105F080010B518F06BFB4FF4803018F087FB18F0D1
:105F18009FFC0128044628D1102018F081FA02209D
:105F280018F072FA002018F0B9FB002018F0CAFB2C
:105F38004FF4806018F0BCFB4FF4404018F0CCFBE5
:105F48004FF480304FF4E01118F084FB204618F02D
:105F58008DFB392018F068FC0028FAD0022018F0D0
:105F68008BFB18F093FB0828FBD17C20012118F04B
:105F780025FC46F60120012118F020FC0C480121DF
:105F880018F028FC0B48012118F024FC04200121FA
:105F980018F020FC7E2018F047FC38B118F06EFC91
:105FA800054B04211A7861F344021A7010BD00BF32
:105FB8000340060000080818ED29002010B50C461B
:105FC800014620B110220C48FAF7BAFC04E00A484E
:105FD80020211022FAF7DEF934B1084821461022B0
:105FE800BDE81040FAF7ACBC044820211022BDE8F7
:105FF8001040FAF7CFB900BFF201002002020020DA
:1060080010B5FF2B1446029A03D0421802F8013C3F
:1060180008E06FF07F439A4204D0131443701312C0
:106028008370C27015F02AFD02E07F2018F042FF4D
:1060380015F010FD0028F8D1ACB10B4890F82010ED
:10604800163001F00F0115F019FD02E07F2018F05D
:1060580031FF15F0FFFC0028F8D1044B93F86930A4
:1060680013F0010FE9D110BD4C0C002008290020C5
:1060780010B50A4B002203EB8003013B1046084988
:1060880051184C7813F8011F8C4205D10130C0B269
:106098000C320428F3D1FB3010BD00BF46EF0108D5
:1060A800581A002070B50D4C05460E464FF4807204
:1060B80000212046FAF76EF92A46314604F5807029
:1060C800FAF7C0F8642004F8025C16F055FF0023C4
:1060D80084F8F131024B64221A6070BD702A0020E6
:1060E8000818002010B5054C002120464FF4807296
:1060F800FAF750F9002384F8F13110BD702A002016
:10610800164B2DE9F0415D8907462846FBF708FD47
:106118001349FBF711FE134B134E1860D723B5FB39
:10612800F3F5EDB2822229460446F01901F07CFE0F
:106138002846FBF7F9FC01462046FBF73FFC0B49D4
:10614800FBF746FDFBF70AFF0337BE19C1B28122F0
:106158003046BDE8F04101F067BE00BF241B0020B7
:1061680000005743AC130020F2010020000020413A
:1061780070B54B4D2868FBF7DFF845A3D3E900233A
:10618800FAF77AFFFBF7C6FBFBF7D6F842A3D3E989
:106198000023FBF725F93EA3D3E90023FBF74AFACE
:1061A800FBF7B8FBFBF7C8F8FAF7D2FEFBF7B2FB30
:1061B8003C4906462860FBF7B3FE20B13046FBF7A2
:1061C800CDFEC4B25EE030463649FBF7BDFE50B1A5
:1061D80030463549FBF7A4FE28B13046FBF7BEFE32
:1061E800C0B2441C4EE030462F49FBF7ADFE50B11B
:1061F80030462E49FBF794FE28B13046FBF7AEFE39
:10620800C0B2841C3EE030462849FBF79DFE50B1E1
:1062180030462749FBF784FE28B13046FBF79EFE3F
:10622800C0B2C41C2EE030462149FBF78DFE50B1A8
:1062380030462049FBF774FE28B13046FBF78EFE46
:10624800C0B2041D1EE030461A49FBF77DFE50B16E
:1062580030461949FBF764FE28B13046FBF77EFE4D
:10626800C0B2441D0EE030461349FBF76DFE48B13D
:1062780030461249FBF754FE20B13046FBF76EFE5C
:10628800C0B2841D0A202146BDE8704009F00CB850
:10629800736891ED7CFF7F400000000080842E41F0
:1062A800B0130020000010410000F04100004842F7
:1062B80000008E420000B8420000E0420000F242B6
:1062C8002DE9F04F9DB015F06FFB092016F080FF07
:1062D80016F0D6FD4FF4614016F0B6FF092017F00E
:1062E80033F80022A1484FF4804118F0FEF8A04886
:1062F800002118F0C7FC9F4904224B78DFF898E288
:106308006FF300034B709C4B9C4C1A705A709A7038
:10631800DA709B4B033A1A709A4B00201F328EF8A2
:10632800000020705A7005900546069006467F20AA
:1063380018F0C0FD23780E2B01F2B281DFE813F0CC
:106348000F004F009500E0007902DE033004850459
:10635800E806DA07ED075608AF08CE087E098A4E28
:106368008A48317801F00F01013149014118FFF7DE
:1063780025FE337813F00F0308D1854A92F891204F
:10638800012A41F08D81834A138024E0012B03D137
:106398007F4B93F8A9300BE0022B04D17C4B93F888
:1063A8009D30032B05E0032B06D1794B93F89D30E4
:1063B800012B41F075810EE0774901220A70774878
:1063C8004FF4007118F091F8754BC8221A603378B1
:1063D8006FF30303BFE333785A1C01F05DB8704BC9
:1063E8001A6822B96D484FF4007118F07EF8DFF88A
:1063F80098816C4898F8001001F00F0101314901AB
:106408004118FFF7DBFD36B198F800305A1C62F3EB
:10641800030388F800305F4B00221A8098F80010B8
:1064280001F00F02022A03D11A7842F010020AE0A2
:10643800042A03D11A7842F0040204E0052A05D19F
:106448001A7842F040021A7001F02AB9062A04D1DB
:106458004D4B6FF3030119707EE301F00F01012228
:1064680012FA01F1198001F01BB9474E4E483178F4
:1064780001F00F01013149014118FFF79FFD96F81E
:10648800008008F00F08B8F1070F27DC18F0010F9B
:10649800464B02D00020588002E04FF0FF3159806F
:1064A8004FEA6809062209F1010902FB09394FF090
:1064B800FF32A9F802204046FFF7DAFDFF2806D090
:1064C8003B4B03EB40005823437401F0E9B8002329
:1064D800A9F8023008F1010801F088B8002110225B
:1064E80013A8F9F757FF0FA800211022F9F752FF58
:1064F80023780133237033786FF3030301F079B8FD
:10650800DFF884A09AF8008018F00F0840F03F8167
:10651800284E337803F04003DBB2F3B926486FF016
:106528007F43817A0122009301F00F01FF23FFF7D7
:1065380067FD224B93F8692012F0400F08D093F8BA
:106548006C3013F0040F03D0337843F040033370FA
:106558007378142262F3C7037370737813F0F80F1B
:1065680030D0174800F12001A5E300BF0018014012
:10657800002C01403E1B0020EC190020B61300201F
:106588001B0E002055220020B513002066EF0108DD
:10659800581A00200423002038180020000C01405D
:1065A8000818002006F00108E6F00108BE220020C5
:1065B800F2010020952100204C0C00200829002021
:1065C80006F20108BC4B1B7803F04003DBB2002B3A
:1065D80000F0D980DFF80483DFF8049398F80030DE
:1065E80013F00C0B30D1B54E6FF07F4396F82B109B
:1065F80006F12100009301F00F0101220523FFF7A6
:10660800FFFC96F84C104FF4860A06F1420001F0A0
:106618000F010122FF23CDF800A0FFF7F1FC96F847
:106628004110FF2306F1370001F00F015A46CDF85B
:1066380000A0FFF7E5FC042389F8003098F8003043
:1066480043F0080301F02AB803F00803DBB2002B7B
:1066580039D099F800A0BAF1000F03D0984800F19A
:10666800400138E0954E6FF07F4B717D06F10B00CD
:1066780001F00F010122FF23CDF800B0FFF7C0FCA5
:1066880096F82B1006F1210001F00F0101220723D3
:10669800CDF800B0FFF7B4FC96F836104FF4860337
:1066A800009306F12C00FF2301F00F015246FFF77B
:1066B800A7FC98F800306AF3C303DBB243F0040385
:1066C80088F800305AE099F800C0BCF1000F08D0F3
:1066D8007B4800F16001FFF771FC99F80020303227
:1066E80008E2764E6FF07F40717DFF23009001F045
:1066F8000F0106F10B000122CDF80CC0FFF780FC5A
:106708009AF80030DFF8C4B103F0100A5FFA8AFA89
:10671800DDF80CC0BAF1000F0CD098F800206CF32B
:10672800820288F800205A1C62F303038BF80030B9
:1067380000F0B6BF96F82B106FF07F42009206F17A
:10674800210001F00F0101220C23FFF759FC96F8F4
:1067580036104FF4860300935246FF2306F12C00AF
:1067680001F00F01FFF74CFC9BF8003083F010029A
:10677800C2F3001262F304138BF80030042389F883
:10678800003000F08DBF4E4800F1800193E2B8F16F
:10679800010F3CD14A4800F1A001FFF70FFC002E81
:1067A80000F07E879AF80030444E5A1C62F30303C7
:1067B8008AF8003096F82B106FF07F4906F1210017
:1067C80042460F2301F00F01CDF80090FFF718FCA7
:1067D80096F82B1006F1210042460E2301F00F0116
:1067E800CDF80090FFF70CFC96F82B1006F121006D
:1067F800424601F00F010F23CDF80090FFF700FC8F
:1068080030488021424617F070FE00F049BF2C48FE
:1068180000F1C001FFF7D2FB002E00F041872A4BA0
:1068280096221A609AF800306FF303038AF8003052
:1068380092E1264E317811F00F0A16D1244800F162
:106848002001FFF7BBFB204B1B68002B40F028877B
:1068580013A8F9F7EFFF40221346014613A801F0E9
:1068680007F93378012200F017BEBAF1010F39D1C8
:1068780012486FF07F4390F82010002200931630E2
:1068880001F00F01FF23FFF7BBFB01F05BF90028C4
:1068980000F006873378022262F3030333700D4B4E
:1068A8001A7842F080021A700B4B5A7842F00202B2
:1068B8005A7000F0F5BE00BF952100204C0C002056
:1068C80006F201080010014008180020B513002046
:1068D800E6F201089A21002018240020F82E002052
:1068E800472F002001F00F0101F10E0303F00F0301
:1068F800012B44D89B4849014118FFF75FFB9A4890
:106908006FF07F4390F8201000221630009301F0BA
:106918000F01FF23FFF774FB16F06AF9337803F0D1
:106928000F03022B13D112F0B7FE002800F0B8862F
:106938008E4B1A7842F040026FF304121A705A789C
:106948006FF345125A703378032200F0A5BD12F098
:106958008DFE78B112F038FF12F004FE844B00204F
:106968001A7858816FF3C7121A703378042262F3C9
:10697800030333707F4B1A786FF3000263E5BAF1B3
:10698800040F4DD1DFF8DC914901DFF8108249444A
:106998004846FFF713FB98F80010774B01F0040204
:1069A800D2B27AB941F004016F4883F800A088F8A0
:1069B800001090F836104FF4860300932C3001F045
:1069C8000F01ECE293F800A0BAF1000F40F06886DE
:1069D80065486FF07F45417D01220B3001F00F01C2
:1069E800FF230095FFF70CFB64480122817AFF23FF
:1069F80001F00F010095FFF703FB98F8003005221E
:106A08006AF3820388F800303378484662F3030358
:106A1800337009F1A001FFF7D1FA554600F040BEE6
:106A2800DFF84481FF2398F8201000226FF07F4997
:106A380008F1160001F00F01CDF80090FFF7E0FA19
:106A48002BB2072B18D1337808F121006FF3030319
:106A58003370237801220133237098F82B100E230A
:106A680001F00F01CDF80090FFF7CAFA44488021E1
:106A7800002217F03AFD0025424E96F86B3013F0CD
:106A8800040F00F00D8698F857106FF07F4300222E
:106A980000933D48FF2301F00F01FFF7B1FA96F884
:106AA8006B303A4A03F00F03012B137003D1002D0A
:106AB80008BF01250CE0022B04D12BB2012B08BF23
:106AC800032505E0032B03D12BB2032B08BF0725B1
:106AD800ABB213F0010F02D02D4A3121517713F0D8
:106AE800020F02D02A4A3221917713F0040F00F0E6
:106AF800D7853322264BDA7700F0D2BD1948254EC8
:106B080000F1C001FFF75AFA96F80090DFF85C80B0
:106B180019F00F090CD112F03FFC98F8003069F316
:106B2800000388F8003033785A1C62F3030333708B
:106B380012F0C4FC98F8003013F0010F00F0B08593
:106B480000221548802117F0D0FC0A4B00225A7009
:106B5800337862F30303337023780133237000F032
:106B68009FBD00BFE6F201084C0C0020182400204D
:106B78009A21002094230020472F002001000020A4
:106B88000010014008290020990C002094210020C1
:106B9800F2010020B513002000180140F82E002053
:106BA8008548864E00F1E001FFF708FA0FA8F9F7CB
:106BB80041FE0FA902468248F9F7C2FE002181482A
:106BC800B18090F8C5106FF07F4300220093BB306E
:106BD800FF2301F00F01FFF713FA7B4A92F86B10BD
:106BE80092F86C30327843EA012312F0010FB38037
:106BF80010D0A3F1EB0292B20A2A04D9A3F5E673E6
:106C08009BB2282B02D8F3880133F38033786FF3D3
:106C1800000333707378002B40F04285674AD288AE
:106C28007AB16A4A1BA8117863F3030111702278BC
:106C38008DF86F300132227028228DF86C2017F001
:106C480073FC0022F28000F02BBD614EDFF8A8A192
:106C5800337803F00408B8F1000F15D109A84146AC
:106C68001522F9F797FB5B4BCAF800801B6845466D
:106C7800CDF827303368474643F004033360564B5A
:106C880083F8F98100F00CBD03F08003DBB2002B20
:106C980067D1DAF80010002940F002854F48FFF765
:106CA8008DF94F484FF4805117F015FC012806D094
:106CB8004A4800F1A001FFF781F900F0F1BC46490C
:106CC80091F8F921002A43D008314648013AF9F7EA
:106CD80037FE444B03F1100113F8012B0D2A01D0A4
:106CE8000A2A02D1202203F8012C8B42F4D13E4B10
:106CF8004FF03C0808FB073808F11E084046F9F732
:106D080099FD414602463948F9F7C4FDD8B9022F22
:106D180003D1336843F0100304E0032F03D1336831
:106D280043F040033360327853005BB203EAC26336
:106D3800DB173268DBB263F3C71232601BB1FFF7AF
:106D4800D1F900F0ADBC0137FFB2042F08BF02270C
:106D5800254B3C2606FB07363046F9F76BFD3146D6
:106D680026E0DAF80080B8F1000F40F099847378D3
:106D780003F02002D2B2002A40D11D4B09A81A887C
:106D88009B781C498DF82630ADF82420F9F75CFB78
:106D9800114B1B7A302B07D1FFF7A4F9336843F462
:106DA8000053336000F07CBC09A8F9F743FD09A93A
:106DB800FFF778F900F074BCE6F20108942300208C
:106DC800060200204C0C002008290020B5130020E2
:106DD8000C180020ABAD0208682A0020E6F3010871
:106DE80000080140020200200C000020702A002048
:106DF800B0AD0208B4AD02080818002003F0400343
:106E0800DBB2002B40F08980B14800F16001FFF748
:106E1800D5F8B048F9F70EFD8046AE49AE4842466F
:106E2800F9F738FD002873D1AC4B43441B7A302B5B
:106E38006ED1FFF757F93368DFF8D09243F48043F7
:106E4800336099F82B106FF07F43009309F121000C
:106E5800082301F00F010122FFF7D2F86423CAF8D2
:106E680000307F2018F026F8DAF80030002BF8D12F
:106E7800984699F88E10D633994E89F886304B3B50
:106E88006FF07F4A89F88730964801F00F01424633
:106E98007433CDF800A0FFF7B3F896F8B91106F5EA
:106EA800D670033001F00F014246FF23CDF800A051
:106EB800FFF7A6F896F8C41106F5DD7001F00F018A
:106EC8004246FF23CDF800A0FFF79AF896F8CF11B5
:106ED80006F5E270013001F00F014246FF23CDF8BC
:106EE80000A0FFF78DF896F8DA1106F5E87001F0C2
:106EF8000F014246FF23CDF800A0FFF781F899F86B
:106F080099107948CDF800A001F00F01424646E0FB
:106F18007648F9F78FFC75494AE796F802B0DFF82A
:106F2800EC910BF0020B5FFA8BFBBBF1000F3AD12F
:106F380099F82010FF236FF07F4809F1160001F03F
:106F48000F015A46CDF80080FFF75AF8684B93F8BE
:106F58006B3003F00803DBB2002B00F0A18399F833
:106F68002B10012209F1210001F00F010323CDF8B4
:106F78000080FFF745F83368554843F4003300F1C3
:106F880080013360FFF71AF855485A4690F8E51122
:106F980000F5EC70CDF80080033001F00F01FF23FD
:106FA800FFF72EF87CE3CAF8008099F820106FF0FC
:106FB8007F4300934246FF2309F1160001F00F01B9
:106FC800FFF71EF82AB241F211139A421DD1434B22
:106FD8001B7A302B13D1FFF785F83368454668F3E1
:106FE800514368F38E3368F34D333360414B1A785D
:106FF80068F303021A7023780133237050E33E4884
:10700800F9F718FC3C49FFF74DF8394E96F86B3004
:1070180013F0040F00F0448325B9384820211022CA
:10702800F9F7B8F97F2017F045FF99F857106FF076
:107038007F43002200933248FF2301F00F01FEF73F
:10704800DFFF96F86B202F4B02F00F020D2A1A7003
:1070580005D125B92C4A412191754FF480551A78EC
:10706800062A08D12AB2B2F5805F04D1264A362111
:10707800D1754FF488551A78082A08D12AB2B2F582
:10708800885F04D1204A3821117641F210151B7807
:107098000B2B09D12AB241F210139A4204D11A4B90
:1070A8002A225A7641F211150D486FF07F4390F865
:1070B800F0110022009300F5F370FF2301F00F0197
:1070C800FEF79EFF96F86B3013F0010FAAD0E7E2A7
:1070D800E6F301081A010020702A0020682A00201F
:1070E80001000020D00C0020DB0C0020FC00002058
:1070F80008290020B51300203801002002020020D2
:10710800990C002094210020F20100204C0C002052
:10711800A34B1A7842B300221A700F20FAF794FF93
:1071280006460A20FAF790FF9E4B9F4958814A78F5
:1071380012F0010F18D06436301A58829B4B1A7817
:10714800642A01D19B321A701B78984EFF2B0BD002
:107158000A21B3FBF1F1964B23311980954817F0BA
:1071680091FD337801333370DFF8648298F800308A
:1071780013F00F0612D18E4B23228B481A804378C6
:10718800232143F0010343708A4817F07BFD8A48A6
:1071980000F12001FEF712FF04967AE2012E68D171
:1071A800804B5A8AA2F1690189B2112908D8049939
:1071B80011F0010F04D141F00101C9B20491059207
:1071C800049A12F0020F0DD15B897C4A1380A3F553
:1071D800AE630B3B9BB2D72B04D8049840F0020354
:1071E800DBB204931B20FEF78BFF0599744B0AB2A0
:1071F800632A05DD642192FBF1F230321A7401E052
:10720800092A0CDD059A11B2642291FBF2F002FB07
:1072180010120A2012B292FBF0F230325A7405981A
:1072280002B2642092FBF0F100FB11210A2209B29C
:1072380091FBF2F002FB101230329A745B4B1B7810
:10724800FF2B08D158495B484B786FF300034B700C
:10725800002117F017FD049A032A40F021825248B2
:10726800002143786FF300034370524817F00AFD7A
:107278000FE2022E03D1534BC8221A6009E2032EF3
:1072880016D1504B1B68002B40F00A824A4800F187
:107298004001FEF793FE1B20FEF732FF414B5B894E
:1072A800A3F51E630F3B9BB2542B00F2F981F0E16A
:1072B800042E0CD13B4B98890CF006FA002840F0BC
:1072C800EF813D4800F16001FEF778FEE1E1052E0F
:1072D80007D1344B98890CF0F7F9032840F0E08186
:1072E800D7E1062E40F0D58122786FF303030132EF
:1072F8002270D3E1344800F12001FEF75FFE334BE2
:107308001B78002B00F0CC81237801332370304B9D
:107318001A786FF30302FFF796B82D4EDFF8A480B2
:10732800337813F00F021AD12A4800F12001FEF732
:1073380045FE2948F9F77EFA274902462748F8F713
:1073480081FF2548F9F776FA254BA3F8160233781A
:107358005A1C62F30303337016F020F891E0012AF7
:1073680016D1D8F80030002B40F09A8116F042F878
:10737800012840F095811B48F9F75CFA1949024643
:107388001948F9F787FA002840F08A8111486FE018
:10739800D8F80020002A40F083810B217BE000BF51
:1073A8001E0E0020241B00203E1B0020C4130020BA
:1073B800480C0020002C0140A6F40108B813002056
:1073C800F20100200818002026F50108B413002057
:1073D800B513002066F5010874010020831F002002
:1073E800CC2C002092010020CD2C0020864E337832
:1073F80013F00F080CD185484146FEF7DFFD3378BE
:107408005A1C62F303033370814BA3F8028047E1EF
:10741800B8F1010F18D17F48042117F05CF8002853
:1074280000F03E81794800F12001FEF7C7FD33786E
:107438004FF0FF315A1C62F303033370764B64221A
:107448001A60734B59802BE1B8F1020FDFF8C8813D
:107458001BD1D8F80030002B40F022816D48042160
:1074680017F039F8002840F01B81694B58806748AD
:1074780000F14001FEF7A2FD33785A1C62F30303C2
:1074880033706423C8F800300AE1D8F80020002AD5
:1074980040F006810C21217062F30303A9E05F49E3
:1074A80010234FF40052CB700D3B8B700A805C4860
:1074B80016F0C2FF0A2200215A48F8F76BFF802015
:1074C80016F01EFF2378013323704F4B1A786FF3A1
:1074D80003021A70504BC8221A60E1E05248DFF8E4
:1074E80044A100F12001FEF769FD9AF80030002B55
:1074F80000F0D6804D48DAF80020434E0260BAF812
:10750800042082809AF806208271317811F00F01E8
:1075180059D1DFF80481D8F80010002940F0C08064
:107528009AF80410A2F5A6524FF0640B103A0BFB20
:1075380001229AF805004FF00A0909FB002003937D
:10754800FAF7EEFA3A49FAF7F7FB02469AF8020018
:10755800039BA0F5A65010380BFB030B9AF801000B
:10756800344B09FB00B018600392FAF7D9FA039A72
:1075780001461046FAF724FA2F4B1860F9F7DCFE9B
:107588001DA3D3E9002382468B46FAF7AFF90028FA
:1075980000F086805046594619A3D3E90023FAF72C
:1075A8009BF900287CD0FEF7E3FD337848465A1C47
:1075B80062F303033370C823C8F8003007F07EFE77
:1075C800C0B207906CE001296AD10D300799832277
:1075D80000F02AFC104BD3F80080B8F1000F5FD1FF
:1075E800404616F08DFE237801332370337868F314
:1075F8000303337054E000BF736891ED7CFF7F4054
:107608000AD7A3703D008040B5130020C6F50108D5
:10761800BE220020000C0140081800203A1B002060
:1076280000100140CC13002026F6010802020020B9
:1076380000007A44C8130020B01300208448854E07
:1076480000F12001FEF7BAFCF37913F0010F27D0FF
:10765800DFF8488298F8009019F00F0920D17E4B86
:107668000A2259781878103902FB0011B17019797B
:10767800D878103902FB00117170D9799B791039CB
:1076880002FB0312327013F0F9FAF37969F300037D
:10769800F37198F800305A1C62F3030388F800303D
:1076A800DFF8FC9199F8006016F001063EF43FAE51
:1076B8006A4B01221A7014F04DFF2378092B01D070
:1076C8000D2B28D1012066490EF05CFC654B664AFB
:1076D8005B7803F01F03D35C644A522B137002D10A
:1076E800634B01221A70634B634A03F1200153F87C
:1076F800040B8B4242F8040BF9D1002117A80EF0B5
:107708005DFC17A80D2115F0E5FD5C4B1A780132D8
:1077180002F003021A7099F8006006F00206F6B249
:10772800002E00F08B800CF025FA0FF0D3FD0698A0
:107738000322431C93FBF2F202EB42029B1ADBB2D8
:107748000693002B79D1DFF8488198F84960C24642
:10775800002E4DD0022E03D198F80130312B49D09C
:1077680023780E2B13D1464846490522F9F792F89B
:107778008246002840D1B21F37484349F9F7E0F85C
:10778800344B5646DA7942F00102DA7135E00D2BB6
:1077980003D13E483A49072227E0032B22D13C4B2C
:1077A800002713F8012F2C2A03D00137FFB2B74264
:1077B800F7D113A832493A46F9F7C2F87B1C07E01B
:1077C8000AEB03025278303AD2B2092A03D80133BD
:1077D800DBB2B342F4D30AEB0701FA430FA8023134
:1077E800D21802E0264909A8721EF9F7A9F803E0A1
:1077F800069E02E0012600E000261E4B204A03F107
:10780800100153F8040B8B4242F8040BF9D1214BB9
:10781800214A03F1100153F8040B8B4242F8040B80
:10782800F9D1402388F811301C3B88F82230023BFC
:1078380088F84B3015F046FB00E0002699F8003038
:1078480003F0F5036FF3000389F80030FEF76FBD0E
:1078580066F6010878270020BA1300201E0E0020C3
:10786800692C0020682C0020E42402080122002052
:10787800B4130020F20100202E220020AD210020A8
:10788800172A0020B7AD02081C2A0020CC130020BC
:10789800162A002002020020282A0020B513002002
:1078A800F0290020AFF30080084B187800F004009E
:1078B800C0B250B11A6822F004026FF341021A6094
:1078C800034B00221A70034B18787047A821002038
:1078D800F0130020D8130020084B1B7813F0010F79
:1078E8000AD1074B1B783BB1064B1B6823B9064AE4
:1078F800136843F002031360704700BFF1130020C0
:10790800F0130020EC130020A8210020064B0021D2
:107918001970064B06481A6822F0020261F38202C7
:107928001A601222F8F736BDF0130020A8210020B3
:10793800D813002038B5094C094922780546F8F7CC
:1079480081FC23780021E954064B1A6822F00402CE
:1079580061F341021A60207838BD00BFF01300209F
:10796800D8130020A82100200D4B1B7813F0010F1D
:1079780014D10C490C4A0818137810F8010C0B495B
:10798800112BC85401D801331370094B4FF4967268
:107998001A60084A136843F004031360704700BF75
:1079A800F1130020A6F60108F0130020D8130020D8
:1079B800EC130020A821002070B5294C002384F87E
:1079C800293084F8283014F8103094F82A2003F06D
:1079D8000F0363F3030284F82A202A2604EB4000ED
:1079E800417873431F4D61F3071284F82A20628C93
:1079F800E95A1D48E28417F043F994F82A301A48E6
:107A080003F00F0306FB03535988013989B217F0B5
:107A18003BF901210A46144817F002F901211248DE
:107A280017F0EFF894F82A3010481B097343E95A05
:107A380017F026F994F82A300C481B0906FB035561
:107A48006988013989B217F01DF901210A460748EA
:107A580017F0E6F805480121BDE8704017F0D1B8E5
:107A6800F2130020B2F6010800080040003401407B
:107A780030B5164C94F82B50A38445F0010500232B
:107A880084F82B50628484F8211084F8203019E09F
:107A9800C55CA5F13002D2B2092A08D9A5F1410284
:107AA800D2B2052A9ABFA5F13702D2B22A46084DAA
:107AB800013305EB420292F8515192F8502125709A
:107AC80062700234DAB28A42E2D330BDF213002087
:107AD800B2F60108124B10B59A8C0024DA8483F8A8
:107AE800294083F82840224601210E4817F098F8CB
:107AF80064210C4817F0C4F832210A4817F0C4F87A
:107B080001212246084817F08BF86421064817F02F
:107B1800B7F805483221BDE8104017F0B3B800BFE8
:107B2800F2130020000800400034014010B5002185
:107B38002C220348F8F72EFCBDE81040FFF7CABF17
:107B4800F213002070B5204C2378042B37D8DFE8D7
:107B580003F0030D152A30001C4B012093F82B303D
:107B680013F0010F2ED02070013870BD174B93F819
:107B78002000FFF721FF0223237020E0134DEE8C35
:107B8800EEB9FFF7A7FF95F8203095F821200133CB
:107B9800DBB29A4285F8203001D8042300E00323A1
:107BA8002370304670BD094BD88C50B9012323701F
:107BB80070BDFFF7BBFF00232370012070BD0020BC
:107BC80070BD002070BD00BF1E140020F2130020FD
:107BD800202102480A46F8F7DDBB00BFF201002069
:107BE80038B5044608460D46F8F724FE98B103193F
:107BF800202B094BC8BFC4F120001C19002308E042
:107C080014F8012BE02A14BFEA5C202204F8012CA6
:107C180001338342F4DB38BDF20100200D4B46F6F8
:107C280012221B689B6893420FD043F6EE229342C0
:107C38000BD0122B09D0B3F5E97F08D046F6B62051
:107C48001B1A584240EB030070470120704701207F
:107C5800704700BF58140020F0B51F4687B006468D
:107C68000C46084600211546F8F794FB244B07B14B
:107C78009F80B3F9041005A801EB8601042207F0E0
:107C88002EFB002605AB9B5D013BDBB2B92B34D83C
:107C98001D2B4FEA031208D8D31803F51441684680
:107CA800EE31112207F01BFB0BE01649D3185B18C5
:107CB8006A4603F11007186859680833BB4203C2C3
:107CC800F9D12046F8F7B6FDC7B26846F8F7B2FD15
:107CD8003818A84203D8E0196946F8F74DFD6846F8
:107CE800F8F7A8FD7B1C1B18AB4203D8E01906491E
:107CF800F8F7AAFB0136042EC4D107B0F0BD00BFC7
:107D0800C4140020BF990208CBAD020810B5044C7A
:107D1800002120466C22F8F73DFB0123A37010BD1B
:107D2800C4140020044B00225A701A709A7842F04A
:107D380001029A70704700BFC41400202DE9F8436F
:107D4800244C8046A3780D4613F0010F3FD06FF303
:107D58000003A37015F08EF86378002B37D12378D1
:107D68000BB90A336370A3781B4F6FF30003A3703A
:107D780015F080F8217807EB0806611807313046BE
:107D88002A46F8F7DDFD3046F8F754FDC6B2AE4294
:107D9800DFF840900FD80CD2002306EB080089F8D2
:107DA800003038180A332021AA1B89F80130F8F767
:107DB800F1FAAE420BD12178064B6418227A1AB137
:107DC80001311970BDE8F8831A700A225A70BDE8AB
:107DD800F88300BFC4140020F2010020054B1A7874
:107DE8000AB100221A701B7845F6551202FB0311DE
:107DF800FFF7F6BE3E140020F8B505460C460818F5
:107E0800002107F051FA013CE4B26719384607F03F
:107E180055FAC6B2202E03D83846002107F044FA96
:107E28000CB1202EEFD9F8BD02F00F03032B22F07E
:107E38007F0230B5D2B20CD94FF47A7491FBF4F4C6
:107E48002025E4B2057002B114B130340470002268
:107E58000130B1F57A7F05DB4FF47A7491FBF4F5C4
:107E680004FB1511022B0BD9642491FBF4F4202593
:107E7800E4B2057002B114B130340470002201304C
:107E8800632904DD642491FBF4F504FB1511012B2F
:107E98000AD90A2391FBF3F32024DBB2047002B160
:107EA8000BB1303303700130092904DD0A2391FB3B
:107EB800F3F203FB12113031017030BD13B5104BD2
:107EC80001461B689A899C7B12F0100214BF02209D
:107ED800012034B10B4C9B7C2478634303FB0011D5
:107EE80009B23AB10DF10600022207F0F8F9BDF81F
:107EF800060002E0084607F0E1F900B21CBD00BF29
:107F0800581400207314002010B50F4B1B689A8971
:107F18009C7B12F0100214BF0221012134B10B4CDA
:107F28009B7C2478634303FB010000B22AB1084913
:107F38000222BDE8104007F0CCB9054B1968BDE82E
:107F4800104007F0B1B900BF581400207314002086
:107F58008C1400203038C0B2092894BFFF200020BC
:107F680070470000044B1A786FF300021A70034B35
:107F780000221A70704700BFB51400203B1400207F
:107F880070B58B4CFFF7EEFF2578264605F0F00517
:107F9800202D6BD107F09AFC002867D1854B1B7800
:107FA8003BB92378C3F30312013262F3071323703A
:107FB80070BD814B1B7803F08003DBB2002B51D0DE
:107FC8007E48F8F737FCC4B2C4B17D4E7D493046CF
:107FD8002A46F8F7B5FC0A2C0BD8224630467749D2
:107FE800F8F7AEFC30192946C4F10A02F8F7D2F9BD
:107FF80004E0304671490A22F8F7A2FC704C0422CA
:1080080004F10C00A521F8F7C5F96F4B1A7852B1A5
:10801800FF23012A237306D9022A637303D0032A94
:10802800A37318BFE373694C94F8A33013B9684875
:10803800684902E0664804F1A3010622F8F780FCCB
:10804800654B1B78452B40F06281237813F00C0FA9
:1080580040F05D81022243F0100362F301035B4AA2
:10806800137070BD56485D492A4645E1347804F0DE
:10807800F004102C3FD107F029FC00283BD1202226
:1080880057494F48F8F75CFC4D4855492246F8F7E0
:1080980057FC544B1B7813F0010F06D05248F8F7E1
:1080A800C9FB51490246514805E05148F8F7C2FB5F
:1080B8004F4902464D48F8F743FC3E4B1B781BB925
:1080C8004C484D49102217E14A484C491022F8F70C
:1080D80037FC394B1B7803F08003DBB22BB14248E5
:1080E800F8F7A8FB024646484FE04148F8F7A2FBDC
:1080F8000246434842E0337803F0F003302B46D180
:1081080007F0E4FB002842D12D4C20223D492046AF
:10811800F8F716FCA521052204F10B00F8F73AF947
:10812800394B1B78042B02D9FF23E37300E002D1FB
:10813800FF23A37301E0032B02D1FF23637301E044
:10814800022B02D1FF23237300E00BB1FF23E3725C
:108158002E4B5B7813F0600F05D03F23E372237337
:108168006373A373E3732A4B1B7803F02003DBB21A
:1081780033B11F48F8F75EFB024626481C49BBE0AE
:108188001948F8F757FB024622481749B4E03378F4
:1081980013F0F00344D120221F490948F8F7D0FB17
:1081A8001E4B074819888322BDE87040FFF73CBE84
:1081B800B5140020381800200C18002010180020D2
:1081C800F2010020906802080519002040180020DC
:1081D8000C020020FB480208201400204E68020808
:1081E800F0950208182400205B970208FF01002080
:1081F8007C970208020200209C9B02081196020844
:108208000F020020A0490208E9190020441B0020A1
:10821800A82100200D0200203D4902083814002042
:10822800502B1ED107F052FBD8B9394920223948C2
:10823800F8F786FB3848F8F7FDFA37490246374819
:10824800F8F77EFB3648F8F7F5FA3549024635481F
:10825800F8F776FB3448F8F7EDFA33490246334825
:108268004AE0337803F0F003102B06D107F02EFB19
:1082780018B128482E4920223EE0337803F0F00256
:10828800402A3DD123482B49203AF8F759FB2A4B7D
:108298001B781BB3294B1C7834B92948F8F7CAFA5C
:1082A8002749024627481FE0022C06D12648F8F73E
:1082B800C1FA25490246234816E02448F8F7BAFAD5
:1082C800224902461F48F8F73BFB012C0ED12048F3
:1082D800F8F7B0FA1E4902461E480DE01E48F8F7A6
:1082E800A9FA1D4902461748F8F72AFB1B48F8F770
:1082F800A1FA1A4902461748BDE87040F8F720BBB2
:10830800174A6FF307131370164B00221A6070BDDB
:108318001C490208F20100201C420208F601002054
:108328002642020806020020214202080D0200200F
:108338007F4902083296020893210020A71E0020D8
:108348007C970208FB010020959602085B970208BB
:10835800539602080B0200209D97020874960208A3
:10836800B514002058140020204B70B5F022204D81
:108378001A702B7813F0010F0BD01E4C207810F0D8
:10838800010006D11C49FFF729FD237843F00103BA
:1083980023701A4E3378532B0ED1164C237813F0D2
:1083A800010F07D000201649FFF718FD23786FF357
:1083B80000032370FFF7D6FD3378232B14D10D4B20
:1083C8001B7813F0010F0FD1FFF7CCFD2B780D4A66
:1083D80043F006032B701378013BDBB213700A4A93
:1083E80052F82320094B1A6070BD00BFC114002049
:1083F800B51400205D140020C98C02082014002048
:10840800A88C0208A3140020A414002058140020EB
:108418002DE9F0415B4BF0225B4D1A702A7802F08F
:108428001003DBB2002B2DD1584963F347120B60C0
:108438001C462A70564A9A5C2D2A01D00134E4B2AF
:108448000133082BF6D1534E3A213046F8F720F87D
:1084580038B1801BC0B20130301821460222FFF724
:10846800E3FC4D4B1B78452B40F0898000242046C7
:1084780001340EF087FF082CF9D12B7843F0100354
:108488002B7036E0454C237813F0010F16D13F4E80
:10849800FFF73CFC3F4F3168384601310222FFF7B5
:1084A800C3FC2D23BB70307846F63E433C49652219
:1084B800FFF7D2FB237843F00103237003200D213B
:1084C800FFF73CFC2D78304E15F0E00541D1102027
:1084D8003449FFF783FC304B1B78442B0DD12B4AD2
:1084E800136801332A4903F00703C95C2D29F8D022
:1084F8001360BDE8F041FFF735BD532B0DD132783D
:108508004E3B63F347123270204A2749126806200F
:1085180000FB02125380BDE8F081232B2FD11B4BA7
:108528001D60337803F0EF0365F347133370FFF7EB
:1085380019FD23781D4A43F0060323701378013B85
:10854800DBB213701A4A52F823201A4B1A60BDE89E
:10855800F081104C10201849FFF740FC04F110007E
:108568002821F7F795FF50B1001B3178C0B20130D0
:10857800201849098022BDE8F041FFF755BCBDE845
:10858800F08100BFC11400205D1400208C1400206D
:10859800A1220020F201002020140020B5140020A0
:1085A800CB140020458C0208BE220020A314002012
:1085B800A414002058140020668C0208434B2DE9AF
:1085C800F041F022424E1A703378424D43F00103D5
:1085D80033702B68404C9B7C33B9404B1B7803F0BD
:1085E8004003DBB22BB10DE0012B0BD111F098F851
:1085F80040B907F0DDFA236800206FF35553236074
:10860800374943E0A778DFF8D08007F02003DFB2CE
:10861800B7B907F0CDFA2968324B897C1A78384601
:1086280061F301021A70D8F800302D4943F40013A1
:10863800C8F80030FFF7D2FB2B4B802283F8432089
:108648000AF0F2FB804678B12B689B7C012B08D19D
:10865800264B5B7803F01003DBB213B100202449EA
:1086680014E00020234911E00AF00EFC074610B17F
:10867800404621490AE00AF04FFC10B138461F492C
:1086880004E0194B93F8433013B91D49FFF7A6FBD3
:108698001C4B1B78232B16D1FFF764FC337843F06F
:1086A8000603337007F084FA23686FF35553236089
:1086B80009F02CFC144A1378013BDBB21370134AFF
:1086C80052F823302B60BDE8F08100BFC1140020B0
:1086D800B514002058140020A82100200C180020F0
:1086E800EA8C02081E240020B1160020182400205D
:1086F8002C8D02080B8D02086E8D02084D8D020824
:108708008F8D020820140020A3140020A414002038
:10871800614B2DE9F341F022604E1A703378604DB9
:1087280043F0010333702B685E4C9B7C8BB95E4B26
:108738001B7803F04003DBB283B15C4B1B7803F07A
:108748000403DBB2ABB1A37803F04003DBB22BB177
:108758000FE0012B0DD110F0E3FF50B9F9F7B0FC91
:108768002368002023F480036FF3D7532360504914
:1087780064E0A778DFF82C8107F04003DFB22FBB55
:10878800F9F79EFC29684B4B897C1A78384661F3C7
:1087980001021A70D8F80030454943F4800367F3A2
:1087A800D753C8F80030FFF719FB2B68198A21B98D
:1087B8000091082001220B4606E00BB2012B05D1DF
:1087C80000970E2039463A46F9F7CAFC0AF02CFB06
:1087D800074678B12B689B7C012B08D1364B5B7818
:1087E80003F01003DBB213B10020344926E0002067
:1087F800334923E0F9F750FDFF2809D1A07800F0AC
:108808008000C0B210B138462E4917E02E4915E055
:108818000AF03AFB804660B1F9F72CFFC0B2022893
:1088280002D83846294909E0062809D8384628498F
:1088380004E00AF071FB18B126494046FFF7CEFA6A
:10884800254B1B78232B23D1FFF78CFB337843F080
:1088580006033370F9F734FC2368204A23F48003B5
:108868006FF3D75323601378013BDBB213701C4AB4
:1088780052F823302B600F4B1B7813F0030F02D1F3
:108888000AF0A8FA20B102B0BDE8F04109F03EBBF9
:1088980002B0BDE8F08100BFC1140020B51400206B
:1088A80058140020A82100200C180020401800208F
:1088B800EA8C02081E240020182400202C8D0208AF
:1088C8000B8D0208F28D0208138E0208B08D020883
:1088D800D18D02084D8D020820140020A314002019
:1088E800A414002010B5FFF73DFB124B2522DA77C0
:1088F800114B124C1B6816219A7C01FB02425178DD
:1089080001F00F000F2814D00A2803DD0A2060F3B5
:10891800030151709B7C162202FB034463780A21F1
:1089280003F00F03594306486D32BDE81040FFF7C6
:108938007BBA10BDF201002058140020B22100209B
:108948000E0200202DE9F74F984BDFF8B0A2F02275
:108958001A70DAF80030D0469C6847F27803E11ABA
:108968004C4244EB0104DA3A6243914B9D5C9F18F8
:10897800C5F30005EEB29946002E29D130468D493F
:10898800FFF72CFA8C4B1B78232B40F035857B782E
:1089980066F304137B70FFF7E5FA884B1A7842F008
:1089A80006021A70864A1378013BDBB21370854AB7
:1089B80052F82330CAF80030834B1D70834B1D706A
:1089C800834B1D70834B1E60834B1D7000F014BDDC
:1089D800824E814D337893B1814A4FF4A071137858
:1089E80003F01F005B0959430A2303FB00137D4969
:1089F800CB18DB78002B40F06682137084E06E4B56
:108A08001B78532B40F0FC8095F80080B8F1000FDC
:108A18002ED14046214611F060FC5FFA80FABAF187
:108A2800000F25D07B7868F304137B706E4F3A787B
:108A38001AB9204611F068FB13E0531E6B49002B4E
:108A4800184603EA0101B8BF02F11E0040110029CF
:108A580003DA013961F01F01013111F0A1FB002394
:108A68003B7011F0CDFC85F800A00022594BE2E0E4
:108A78002B78002B00F0278256490A680F460B2AEC
:108A880001D10C2316E00C2A11D1013B6101544A93
:108A980059181170554903EA0101002903DA01390F
:108AA80061F01F010131204611F07AFB1CE0092A10
:108AB80002D10A230B60D0E10A2A27D14B49013B96
:108AC80003EA0101002903DA013961F01F010131CC
:108AD800204611F0A7FB2B786201D318DBB2404A7D
:108AE800591E1170404A13704FF00008C7F80080F3
:108AF800FFF738FA162303FB04935A7842F0100262
:108B08005A7085F8008014233370DCE1043A042A93
:108B18003FD83749D2B20878364F60B30020087082
:108B2800397841B13448401810F8010C032802D0B4
:108B3800002840F0C881013B0A2058434FF4A07E2A
:108B48000EFB0400DFF89CE070448018417160015E
:108B58001B18D8B200EB800000F5E840FC30801804
:108B680006F0A2FB387818B1013811F0B1FCAAE17F
:108B78000BF0AAF8A7E101200870013B0A214B433A
:108B88004FF4A07101FB04331649CB189A18537996
:108B98000AE00F4F3B7823B901223A700A4A137052
:108BA80091E1FFF7DFF900233B708CE1C11400204D
:108BB800B22100200857020820140020B514002014
:108BC800A3140020A41400204014002060140020E6
:108BD800731400208C1400207D140020361400200B
:108BE80074140020F2240020311500201F0000809A
:108BF8008914002030150020EC190020581400209A
:108C0800432B1AD1964A1278002A40F043812B78D8
:108C1800002B00F05881934B1A78002A40F05381BA
:108C2800914B19680C2903D00A2903D02A7014E142
:108C38000B2200E009221A600FE1232B7ED1884A1B
:108C48001278002A40F026812978DFF818A2002936
:108C580035D09AF8003053B184490F2B0A708449F3
:108C68000A7000F2308101338AF800302BE17E4A25
:108C78001368082B1ED84FF4A077674301394FF0CB
:108C88000A0E0EFB01717B4F181F7918C978062749
:108C9800013907FB0101784800EB810151F8040F05
:108CA8000133002840F0D880032B40F2D580082BF0
:108CB800F4D9D1E0092B40F006810233CCE07B786F
:108CC8006E4E61F304137B7032781AB9204611F0A6
:108CD8001BFA13E0531E6A49002B184603EA0101E8
:108CE800B8BF02F11E004011002903DA013961F012
:108CF8001F01013111F054FA0023337011F080FB89
:108D08000AF0E2FFFFF72EF95E4B1A7842F00602EE
:108D18001A705D4A1378013BDBB213705B4A52F854
:108D28002330524AC8F8003000231370504A8AF89A
:108D3800003013704C4A2B7013605DE32A2B3CD132
:108D4800474A1278002A40F0A58046490B784BB173
:108D58004648012B02704648027040F2B480013B3D
:108D68000B70B0E02878002800F0AD803E4A136808
:108D7800002B00F0A880092B1AD84FF4A07161438A
:108D880001384FF00A0E0EFB00103A491F1F081851
:108D9800C1780620013900FB0171374800EB8101D9
:108DA80051F8040D013B002856D1032BF8D853E0A5
:108DB8000B2B40F08880023B4EE0442B1AD1284A06
:108DC8001278002A66D1274B1B78002B7BD1287894
:108DD800431EDBB21E2B76D8214611F07EFAC0B2B4
:108DE800002870D0204A13680C2B6CD00A2B6AD04C
:108DF80028701BE0552B4DD1194A1278002A49D109
:108E0800184B1B78002B5ED1287801285BD90238D3
:108E1800214611F073FAC0B2002854D0124A1368E0
:108E28000C2B50D00A2B4ED019490870043B042B48
:108E380013D84FF4A071614301380A2707FB0010CB
:108E48000C490818C1780620013900FB01330A498A
:108E580051F823300BB904331360FFF783F832E07D
:108E680089140020731400208C1400204014002062
:108E780060140020F2240020400D0020311500204D
:108E88001F000080B5140020A3140020A4140020A3
:108E98007D140020303BDBB2092B14D89B4A1268A2
:108EA800043A042A0FD89A4A117861B9994A127873
:108EB8004AB1994A0A27107807FB0033DBB20C2B1A
:108EC800137088BF11702F78DFF8B082002F5FD140
:108ED80098F8000010F0010012D114B920468F490B
:108EE80000E08F49FEF77AFF98F8003043F6DF205C
:108EF80043F0010388F8003006F0E0F9894B187058
:108F0800337813B98848894901E0874888490A2293
:108F1800F7F716FD204611F0CFF9864D01460222DB
:108F280005F11900FEF780FF834B1B7803F08003DF
:108F3800DBB22BB3814B1B88EB81337803BB804BAF
:108F480018781A4618B9204611F0AAF818E07D4B8F
:108F5800411E01EA0303002B03DA013B63F01F0300
:108F680001334FF4A07161430A2505FB03137649C9
:108F7800CB18DB7813B911F071F901E000231370F5
:108F8800162303FB0494637843F01003637033E201
:108F98004FF4A0736343013F0A2202FB07336A4E72
:108FA800F31893F803B06301FF1898F80030FFB284
:108FB80013F0010F45D1FEF7A9FE07EB071101F5E4
:108FC800E0417C311022614806F089F9604B59482C
:108FD80011229A7144230370173BC370791C013026
:108FE8000F3AFEF721FF494B1B6813B91020594966
:108FF8001FE0012B02D1102057491AE0022B02D1A1
:109008001020564915E0092B02D11020544910E0D0
:109018000A2B02D1102053490BE00B2B02D1102050
:10902800514906E00C2B02D11020504901E050496B
:109038001620FEF7D3FE98F8003043F0010388F8B5
:109048000030334B1A789846002A00F0EA8007EB84
:10905800071707F5E0477C3710223648394606F0EF
:109068003EF900229146334B995C9A4641B109F189
:1090780001095FFA89F90132B9F1100FF3D106E05D
:1090880003EB09002021C2F11002F7F783F998F8E1
:10909800000048450BD90138C01906F00FF930B95E
:1090A8001B4B202118780138C01906F0FDF8DFF8AD
:1090B800D09099F8003018460193FEF74BFF4A46C6
:1090C800019BDFF8C09018B9432B40F0848001E081
:1090D800432B04D1002389F80030202172E0DFF807
:1090E800A8E024499EF800C023489C454ED10B783F
:1090F800ACF1300C0133DBB24FF00A0E0B700EFBF3
:109108000C33C35C002B53D10B7051E08C1400203E
:109118007314002089140020301500206B570208B2
:10912800EF5702081B220020F801002031580208DE
:1091380052580208F2010020A8210020CAAD0208F6
:10914800311500201F000080F2240020CB140020DD
:10915800C41400205A590208395902087B590208D8
:10916800205A0208415A0208625A0208835A020821
:10917800A45A02086014002024F80108B51400203D
:1091880020140020401400203D1400208EF80030E8
:1091980099F800304FF0000C81F800C043B198F8FE
:1091A80000300F2B04D803F1010E954B83F800E033
:1091B800402389F8003013780978303B0A2202FBF3
:1091C8000313C15C98F8000001380AF80010381839
:1091D80006F06AF80EE08B4B1B7803F08003DBB2D5
:1091E80043B199F800302BB998F80030FF22534466
:1091F80003F8012C99F8003013B1834A013B13702E
:1092080099F80030012B10D198F800300F2B02D8B4
:109218007B4A013313707D4A002389F800301370AC
:1092280003E004200C21FEF789FD794B1F681FBB62
:109238004FF4A07254432B780A22013B02FB0344EB
:10924800361975782D090F2D00F0D680714CA5219F
:1092580004F11C00063AF7F79DF8FF232377002D49
:1092680000F0CA80012D637700F0C680022DA37735
:1092780000F0C280E377BFE0012F18D14FF4A0724D
:1092880054432B780A21013B01FB034436197378B8
:1092980003F00F030F2B00F0AF80092B04DC013320
:1092A8005D485943BD3AA2E05B4859436AE0022F42
:1092B80038D10BF1FF3B5FFA8BFBBBF1070F98BF6F
:1092C800564BDFF850819CBF5B4493F8647008F1FB
:1092D8001B0088BF002720210522F7F75BF82878B4
:1092E800C7EB08080138002318E04FF4A072624366
:1092F8000A2101FB0022B25C08EB07011A4112F0B7
:10930800010FC7F1000202D08A18DB2101E08A1898
:10931800A52182F82010013308F10108DAB2BA4217
:10932800E3D369E0032F2FD14FF4A07254432B7875
:109338000A25013B05FB0343F218F35C13F0400FC9
:1093480002D01020364906E093785A1ED2B2FD2A80
:1093580006D93449102003B0BDE8F04FFEF73EBDF2
:10936800FE2B02D110203049F5E710202F49FEF7D7
:1093780035FD2F4B2F481B78013B05FB03442E4D31
:109388002C19A178832232E0043F042F34D8062216
:10939800FFB20BF1FF3B02FB0B7B284B284853F82D
:1093A8002B100A31F7F7CCFA264B1B7893B1154BE3
:1093B8001B7803F08003DBB23BB123482021022253
:1093C80003B0BDE8F04FF6F7E5BF204B1E4819780B
:1093D80082220CE02B780A22013B53434FF4A072FF
:1093E80002FB04343619F71917487979BE3A03B0E5
:1093F800BDE8F04FFEF718BD03B0BDE8F08F00BF21
:1094080073140020A82100204014002060140020BC
:109418008C140020F20100200D02002024F801081D
:10942800DE5902089C590208BD590208FF59020872
:109438007D1400200F020020F2240020400D00209F
:10944800020200208914002010020020301500209C
:109458002DE9F0474C4C4D4F2378F02243F001039F
:1094680023704B4BDFF85C911A703B68494A9E6841
:1094780047F27803F01A464246EB0006162171437C
:10948800555C5318C5F300055FFA85F89246B8F1A4
:10949800000F23D140464049FEF7A0FC99F8003060
:1094A800232B6FD1FEF75EFD23783C4A43F0060379
:1094B80023701378013BDBB21370394A52F823301A
:1094C8003B60384B1D70384B1D70384B1D70384B46
:1094D800C3F80080374B1D70BDE8F08799F800206D
:1094E800232A23D15A786FF304125A7010F088FF98
:1094F8000AF0EAFBFEF736FD2378284A43F0060314
:1095080023701378013BDBB21370254A52F82330DD
:10951800244A3B6000231370234A1370234A1370B4
:10952800234A1360234A1370BDE8F087532A0DD1EC
:109538005A78C2F300144CB942F010025A7021460E
:109548003046013410F02CFE202CF8D1304610F0B3
:10955800B3FE162303FB06A67378C1B213F0100FEF
:109568000AD0202902D10020134901E01349002024
:10957800BDE8F047FEF732BC11480222BDE8F047CB
:10958800FEF752BCBDE8F087B5140020581400203F
:10959800C1140020B221002008570208A31400209B
:1095A800A41400204014002060140020731400202C
:1095B8008C1400207D140020E18F0208029002081C
:1095C8000B020020201400202DE9F0412D4E2E4FD3
:1095D800307800F5E0405A3005F070FE3B78C4B2B0
:1095E80013F0010F26D0294D2B78552B0AD1EC2CDE
:1095F80001D0013CE4B23078214600F5E0405A3011
:1096080005F052FE2B78442B0DD1A4F11403DBB2E4
:10961800D72B01D90134E4B23078214600F5E04077
:109628005A3005F041FE2B78532B03D1FEF79AFCF4
:109638000AF04AFB164B1B7803F08003DBB253B1E8
:109648003B7813F0010F06D0124820210422BDE810
:10965800F041F6F79FBE14F0800F0F4805D12B2379
:109668000A2103746143113006E02D230374373B4C
:109678005C43113004F520610322BDE8F041FEF798
:10968800D3BB00BF73140020B514002020140020A1
:10969800A821002002020020F20100201FB5204B63
:1096A80020491A781AB1087840F001000870097842
:1096B8001C4C11F0010F31D01B490978532901D0F6
:1096C8000AB103E082B901221A700DE023290BD1F7
:1096D800002018701549FEF781FBFEF743FC23783C
:1096E80043F00603237019E01B78012B16D12021C3
:1096F8000A460F48F6F74EFE0E4B68461B681022C6
:10970800996805F0ECFD002409491DF8040001EBF7
:109718004401013413F017FF102CF5D11FBD00BF11
:1097280073140020B514002020140020D8920208D9
:10973800F201002058140020034B1B78532B01D151
:10974800FEF710BC704700BF20140020084BFF280C
:109758001A68936807D1917B41B10649927C0978D0
:1097680001FB023302E0927C02FB0033184670478B
:1097780058140020731400204328F8B504460D46F9
:10978800174608D1114B0A261A7891FBF6F66FF3A3
:10979800C3021A7000E00E462046FEF7DBFB90B1CC
:1097A8000A4B303C1A780A2602F00801C9B200298F
:1097B80018BF002506FB05466FF3C30236B21A70C0
:1097C800BE42A8BF3E4630B2F8BD00BFB514002067
:1097D800634B2DE9F3411A689846157C977C614CD8
:1097E8002DB1614821780222FEF71EFB00E02570AA
:1097F800FF01237807F50A47D83707EB43075B4E85
:109808000BB90DB10FE015B901A8394601E001A85F
:10981800B91E022205F063FD9DF80430F3759DF82A
:109828000530337605E006F117003F210222F6F7EE
:10983800B1FD5B23B375023373764D4B1B7813F080
:10984800010F61D04B4B1B78A3F13002D2B2092A29
:1098580035D822780AB9002D40D1474A11781446E4
:109868009942464A01D000211170DFF814E10DF148
:10987800080C9EF800E0A3F13000E644DFF80CC1C4
:10988800117800EB8000604400EB010C0131C9B293
:1098980040189CF86CC090F86C000EF804CC11705D
:1098A80008B1032901D90021117023700DB9384678
:1098B80000E0B81E01A9022205F00BFD17E0232BDA
:1098C80004D12F4B1A7892B9013205E02A2B05D121
:1098D8002B4B1A785AB1013A1A7008E0532B06D16B
:1098E800284A533B1370264A1370FFF725FF264B6F
:1098F8001B7803F08003DBB2002B2FD0204B1B78A2
:10990800F6182023F37529E045B31A4B1878A0F10F
:109918003003DBB2092B10D81A4A137803B9237025
:10992800013303F001031370D8F800302178B3F93C
:109938001020FFF721FF207005E0432803D1114BC9
:109948001B7803B92370104B1B7803F08003DBB23C
:1099580023B1054820210222F6F71CFDBDE8FC8151
:10996800581400206114002000020020F201002099
:10997800B5140020201400203D140020601400209D
:109988003A1400207D140020A821002024F80108A2
:10999800F7B5364E364D3378364C6FF34103337096
:1099A80013F0CEF8FFF7C8FE02238DF807302B78A6
:1099B8008BB1314AD17941F00101D1712F4A207818
:1099C80002EBC303D3F8A07093F8A5203978FFF70A
:1099D800D3FE38700DE0337813F0010F06D02378EA
:1099E800303BDBB2062B9CBF234AD37003238DF890
:1099F8000730337813F0010F12D0214B1B7803F096
:109A08008003DBB263B129781C4B1E4803EBC1030A
:109A180093F8A4309DF80720C0182021F6F7BAFC67
:109A28002378232B09D1184A2B781268927C013AA3
:109A3800934202DA0E4A0133137023782A2B04D199
:109A48002B7813B10A4A013B13702378532B0AD1A0
:109A580011F014F90021084B2970DA7961F300023A
:109A6800DA71FFF769FE00232370FEBDB5140020EC
:109A78007D140020201400207827002024F80108F5
:109A8800A8210020F2010020581400202DE9F14FF0
:109A9800914E924C3378924D232BDFF888820BD16C
:109AA8002368B3F90800FEF709FA286098F800302F
:109AB80043F0080388F800303378532B40F0E280F5
:109AC800236848F685229B68934202D12A68854B11
:109AD80005E04AF21422934203D12A68824B1A7095
:109AE8000EE043F6DD2293420AD1804B29681A78AA
:109AF80061F300021A7005F0E9FE08B105F004FFF1
:109B0800236843F6E0229B68934206D1774B296885
:109B18001A7861F3C7121A7019E043F6EA229342E1
:109B280006D1724B29685A7861F300025A700EE028
:109B380043F6E72293420AD129686D4B19B11A6896
:109B480042F0005202E01A6861F35D721A602368FD
:109B580043F6DA229B68934202D12A68654B05E0F6
:109B680043F6E822934203D12A68634B1A7008E04F
:109B780048F68E22934204D12B6813B9584B012220
:109B88001A602368986848F6CF23984202D12A6859
:109B98005A4B05E048F6D023984203D12A68584B1F
:109BA8001A7016E048F6CE23984203D12A68554B1E
:109BB8001A7015E048F6D123984203D12A68524B0F
:109BC8001A701BE048F6D223984202D12A684F4BFC
:109BD8001AE048F6D423984202D12A684C4B13E085
:109BE80048F6D523984202D12A684A4B0CE043F63E
:109BF800E233984202D12A68474B05E049F2DC4338
:109C0800984202D12A68454B1A7000B2FEF77CF9D7
:109C180023689A6843F698139A4231D12968DFF885
:109C28000CB1DFF8BCA00BEBC1031B793C4FC3F3AD
:109C38004113012BDFF8F8901EDD387800F56650E7
:109C48001C3005F031FB3B78DAF8001009EB030211
:109C580011710BEBC1021279C2F34112032A0BD125
:109C68001E4A126890680830C01805F01DFB3B7842
:109C7800DAF800204B441A723B782A6809F8032066
:109C8800FFF75AFD98F80030264F13F0010F00F047
:109C9800B1802368114F9A6843F698139A4267D1A6
:109CA8003378442B4ED12F7844E01F4B01371B7873
:109CB800FFB233B109EBC7031B79C3F34113012B7F
:109CC80040DC05F003FE28B109EBC7031B7913F04C
:109CD800100F2FD02F6035E02014002058140020DA
:109CE8008C14002038180020932100203215002001
:109CF800A8210020062A0020EA2100201A2400209A
:109D0800EA240020ED240020EB2400201C2400205D
:109D180093230020EC1500200A1000205713002080
:109D280073140020B51400203E0D00200804002004
:109D3800EC190020914B03EBC7021279994612F0F7
:109D4800080FB2D03378552B5ED12E780DE0013E46
:109D5800F6B205F0BBFD30B1884B03EBC6031B79A7
:109D680013F0100F01D02E604EE0002EEFD14BE023
:109D780005F0ACFD00282CD03B6843F6C4219A6856
:109D88008A4203D046F6AA718A4204D13078B5F9DE
:109D980000102D2219E0A2F56A516139052903D96D
:109DA80043F6E9218A4201D1012307E043F6E02185
:109DB8008A4202D00A318A4202D100232B6023E072
:109DC8003078B5F90010B3F91020FFF7D5FC2860FA
:109DD8001AE03B686A4A99688A18012AF0D83278EA
:109DE8002F2A11D9B3F9103030339A420CDC303AAB
:109DF8002A6009E02368B3F90800FEF75FF82860D5
:109E08003B7843F008033B70FFF796FC216843F664
:109E1800D2228B6893420BD12B6813B959485A49FF
:109E280001E0584859490222F6F78AFD0226D2E095
:109E3800534A9A18012A17D82B6813B95448554918
:109E480008E0012B02D15248534903E0022B05D107
:109E58004F4852491022F6F773FDBBE0032B40F040
:109E6800B9804B484E49F5E748F6D32293424D4F07
:109E78000DD129680A22B1FBF2F302FB131230322A
:109E8800FA7730332E22BA777B770326A3E043F69E
:109E9800981293425ED12E68384D102255F836102C
:109EA80007F1100005EBC605F6F74AFD2D7905F018
:109EB8000705012D02DC781D3B4910E0022D0AD16F
:109EC8003A490B22781DF6F73BFD394BB81D197836
:109ED8002A4601313BE0032D09D13649781D0B2272
:109EE800F6F72EFD324BB81D197801312EE0042DFE
:109EF80002D1781D304903E0052D10D12F49781D76
:109F08002B4D0B22F6F71CFD2978B81D01310222D2
:109F1800FDF78AFF297807F10A00053116E0062DBA
:109F280058D1234D26490B222648F6F709FD2978F2
:109F3800254801310222FDF777FF297823480531AA
:109F48000222FDF771FF2978214809310222FDF725
:109F58006BFF3FE0B1F91060092E04DD632ECCBF22
:109F68000326022600E00126C6F1200038182968D9
:109F780046F08002FDF758FF2DE000BF08040020DE
:109F88003175FFFF10020020F4F80108F6F8010807
:109F980002020020B6960208D7960208F896020830
:109FA80019970208F201002063980208BE97020878
:109FB800731400204298020800980208DF970208EC
:109FC80021980208F7010020F8010020FC01002078
:109FD80000020020102698F8003013F0010F0BD073
:109FE800264B1B7803F08003DBB22BB124482021D9
:109FF800801B3246F6F7CEF9224EB37803F00203FF
:10A00800DBB2002B36D0FDF709FE1F4D034628B9F9
:10A018002878F11D6522FDF71FFE08E0B27929783E
:10A02800B388F01D01FB023109B205F058F9236825
:10A0380046F6AA729B6893420FD006DC43F6C42208
:10A0480093420AD043F6784205E046F6EA72934214
:10A0580003D048F68E2293420CD105200B21FDF740
:10A068006DFE297809480131022201B0BDE8F04FA0
:10A07800FDF7DABE01B0BDE8F08F00BFA8210020CF
:10A0880012020020C414002073140020F3010020E1
:10A09800F0B5114B1F78114B303F1E680DE0D6F814
:10A0A80014C01CF803C00133644501D112E0002339
:10A0B800DAB28242F3D301350D70094B0622094901
:10A0C80002FB07330D785B1993F8D440002CEED1CE
:10A0D8000C70F9321046F0BD2014002058140020EE
:10A0E80024F80108601400202DE9F74F984C99498D
:10A0F80025680878AB682E8A9AB200FB06260746C0
:10A1080047F2AC608342B6B288460BD1924B1A78BC
:10A118005B7802F00702C3F3420303EBC20306EBCA
:10A12800C3062CE047F66C018B4212D18A4B8B4850
:10A138001A78597802F0070288235A43C1F342017A
:10A14800773B03FB012320210822F618F6F722F9B2
:10A1580015E047F624418B420BD17F4B1A785B7888
:10A1680002F00702C3F3420303EBC2039B01F61894
:10A1780005E0B3F5E97F04BF3B4602EB4306784FA1
:10A18800784D3B7813F0010F54D123689A6846F64E
:10A19800B2639A4204D046F6B2439A4240F04681EE
:10A1A800714B1B782A2B3CD1704B93F8009009F126
:10A1B800010909F0010983F80090B9F1000F1BD0DB
:10A1C80046F6B2439A4208D1694B46F63E329A8027
:10A1D8009A7842F002029A7028E1202110226548FC
:10A1E800F6F7D8F898F8003000205901C918624BE2
:10A1F800C918FDF7F3FD19E1FDF788FD2368484606
:10A208009A6846F6B2439A420CBF5C495C49FDF72E
:10A21800E5FD98F800105B4801310222FDF704FEC5
:10A2280004E1552B02D0442B40F000814F4B002213
:10A238001A70FBE023685869F6F7FCFA4A4B834624
:10A2480093F800A09946BAF1450F02D14E4B00226F
:10A258001A705046FDF77EFE00284ED04B4B5FFA31
:10A268008BFB1A7852450ED15846FFF711FFFF288D
:10A2780004D15846FFF70CFFFF283ED0444B1A780C
:10A2880001321A7015E0DFF808A100228AF80020D0
:10A2980058460193FFF7FCFEFF28019B04D09AF86B
:10A2A800002001328AF8002099F80020FF281A704F
:10A2B80023D02168374A4B6910601B5C886846F6D2
:10A2C800B26188421360924610D1562B01D0542BAC
:10A2D8000CD198F80030123BDBB2022B06D82B7851
:10A2E80030B2C01804F0EAFFCAF800002B7830B288
:10A2F800C018DAF8001004F0D7FF99F80030552B91
:10A3080017D12368997C0F2913D92A7808398A42EA
:10A31800144B01DA083200E000221A70144B9B78C3
:10A3280003F00203DBB20BB1FDF7FCFC184B002273
:10A338001A7099F80030442B3BD123689A7C0F2A75
:10A3480037D92978074B072926D90839197025E004
:10A3580058140020731400207814002002020020F2
:10A36800B51400207D14002020140020C014002003
:10A37800C4140020F2010020617F0208727D0208E7
:10A38800B47D0208F30100203A1400203D14002097
:10A39800601400208C140020083A1A70914B9B78A6
:10A3A80003F00203DBB20BB1FDF7BCFC8E4B0022BD
:10A3B8001A7099F80030432B0CD1236830B25B69CE
:10A3C80019788A4B19602B78C01804F06DFF864BFA
:10A3D80000221A7099F80030232B13D122682B78A9
:10A3E800927C013A93420DDA814A013313707E4B15
:10A3F80000221A707B4B9B7803F00203DBB20BB18F
:10A40800FDF790FC99F800302A2B0FD12B786BB10F
:10A41800774A013B1370744B00221A70714B9B787A
:10A4280003F00203DBB20BB1FDF77CFCFFF784F904
:10A43800704A2B7811789246994288BF1370127827
:10A448000F32934202DD6B4A0F3B137023684FF0C3
:10A45800000B93F81290B9F10F0F9ABFC9F12009B8
:10A468005FFA89F94FF010099AF8003030B2C01835
:10A47800584404F023FF604B03F8090009F101096F
:10A488005FFA89F9B9F11F0F05D822680BF1010BA2
:10A49800927C9345E8DB3A7812F0010F16D02268D7
:10A4A8005649927C09780F2A01F0800198BFC2F1C1
:10A4B8001002C9B294BFD2B2002239B129789AF8F1
:10A4C800000010319A18091A5F23535423689868BA
:10A4D80049F2DA43984209D1494B1B78532B05D1ED
:10A4E80004F0ECFE474B187004F0D8FF3D4EB378EB
:10A4F80003F00203DBB2002B55D0FDF78FFB0346B8
:10A5080088B9226847F6244192688A420BD046F6F9
:10A51800B2418A4214BF287898F80000F11D6522DC
:10A52800FDF79AFB10E02368B2799B683648B3F5CB
:10A53800E97F0CBF98F800102978B38801FB023135
:10A54800B27909B204F0CBFE23689A7C032A08D9B1
:10A558009A6847F2AC618A4203D046F6B2418A4211
:10A5680013D19B6847F2AC6293420BD13B7813F04E
:10A57800010F01D0102013E0202107222348F5F70E
:10A5880009FF10E0B3F5E97F02D105200B2108E0AF
:10A5980046F6B242934202D10020102101E0002089
:10A5A8000721FDF7CBFB23689A7C032A16D9B278DA
:10A5B80002F00202D2B28AB19B6847F2AC629342BF
:10A5C8000CD046F6B242934208D02978104801319F
:10A5D800022203B0BDE8F04FFDF726BC03B0BDE88A
:10A5E800F08F00BFC4140020601400208C140020D9
:10A5F8007D14002075140020F2010020A8210020FD
:10A60800201400203F140020CB1400200202002058
:10A61800F30100202DE9F74F874C884F2368884EB7
:10A628009968B3F910303A78B3F1010848BF03F1DB
:10A6380006084FEAE808337808F1010812F0010F1C
:10A6480003FB08187F4D00F0AD807F4B1A789946C0
:10A65800432A4DD128780FFA88FA0AEBD00004F083
:10A668002DFE2268794B916846F2A25291421860F9
:10A6780001D12A783AB12A78012102F0070211FAA9
:10A6880002F250401860287819780AEBD00004F0DC
:10A698000BFE236847F24A029B68934209D1694B33
:10A6A8001A786B4B03EBD203684A126883F8502080
:10A6B8001EE046F65222934205D13178002001313E
:10A6C8000AF07AFB14E046F2686A4FF0000B236840
:10A6D8009B68534504D101200BEB00010AF06CFB89
:10A6E8000AF1080A46F288639A450BF1010BEED18C
:10A6F80099F80030232B10D122682B78927C013AEC
:10A7080093420ADA4F4A01331370524B9B7803F095
:10A718000203DBB20BB1FDF705FB99F800302A2BD9
:10A728000CD12B7853B1474A013B1370494B9B78A6
:10A7380003F00203DBB20BB1FDF7F4FA99F800302D
:10A74800552B14D12368997C0F2910D92A780839F8
:10A758008A423C4B01DA083200E000221A703D4B75
:10A768009B7803F00203DBB20BB1FDF7DBFA99F833
:10A778000030442B7FD123689A7C0F2A7BD9297813
:10A78800304B072902D90839197001E0083A1A70C4
:10A79800304B9B7803F00203DBB2002B6BD0FDF744
:10A7A800C1FA68E048F6452399420DD1264B1B783B
:10A7B800A3F13101C9B2032906D842F006023A7062
:10A7C80007225343573B337023689A6843F6E333B1
:10A7D8009A4250D11C4B1B782A2B45D11E4B93F81B
:10A7E800009009F1010909F0010983F80090B9F115
:10A7F800000F13D033781B2B08D9164B46F63E3280
:10A808009A809A7842F002029A7034E05A01134909
:10A81800D3180020C918FDF7E1FA2CE0FDF776FA05
:10A8280048460F49FDF7DAFA31780E48013102221D
:10A83800FDF7FAFA1FE000BF58140020B5140020F5
:10A84800731400207D140020201400208C14002094
:10A85800EC190020C41400207F1400206083020833
:10A868001E830208F3010020552B01D0442B02D18E
:10A878007D4B00221A70FEF75FFF7C4A2B78117817
:10A888009346994288BF137012780F32934202DDC3
:10A89800764A0F3B137023684FF0000A93F8129022
:10A8A800B9F10F0F9ABFC9F120095FFA89F94FF082
:10A8B80010099BF800004FFA8AF318180FFA88F26B
:10A8C80002EBE000019304F0F9FC9BF80020019BE7
:10A8D8005FFA80FC9B1803F0070316E04CFA03F0BC
:10A8E8006349013300F0010000280CBFA520DB20DC
:10A8F800DBB201F809000AF1010A09F10109082B84
:10A908005FFA8AFA5FFA89F903D0B9F1200FE5D125
:10A9180009E0B9F1200F06D023684FFA8AF19B7C31
:10A9280089189942C5DB3B7813F0010F15D02368CD
:10A9380050499B7C09780F2B01F0800198BFC3F127
:10A948001003C9B294BFDBB2002331B129781031AA
:10A958008A1A4749CB185F219954474FBB7803F0AF
:10A968000203DBB2002B60D0FDF758F90346F8B9B3
:10A97800226846F6522192688A4206D024318A42D9
:10A9880003D043F6E5118A4204D130783B49652269
:10A99800002308E043F6E3318A4207D130781C38B7
:10A9A800C0B2F91D6522FDF757F918E02878F8E7D5
:10A9B800236846F612229B68934203D043F6EE22A0
:10A9C800934202D1BA79317801E0BA792978BB8803
:10A9D8002A4801FB0231BA7909B204F080FC2368E5
:10A9E8009A7C102A1DD89B6846F6122293420ED0F4
:10A9F80006DC43F6E512934209D043F6EE2204E062
:10AA080046F65222934202D02432934202D11020B9
:10AA1800072108E043F6E332934202D100201021D7
:10AA280001E005200B21FDF789F9236846F6B621D8
:10AA38009A688A4214D046F670118A4210D09B7CDC
:10AA48000B2B0DD9BB7803F00203DBB243B1297895
:10AA58000B480131022203B0BDE8F04FFDF7E4B91D
:10AA680003B0BDE8F08F00BF7F14002075140020EC
:10AA7800F2010020A8210020C4140020CB140020DB
:10AA8800F30100202DE9F04F714E89B033689C68BE
:10AA98009F7C122C01D00B2C0DD16E4A1778303FB9
:10AAA800122CFFB209D19B7B3BB96B4BD879FEF7CF
:10AAB8004DFE054615E0013FFFB2FF20FEF746FEBA
:10AAC8004AF248139C4205460BD14AF2152004F07D
:10AAD800F5FBC0B2069020B15F4B9B790BB1FDF737
:10AAE80041FA33689A68122A17D19B7BC3B1594B34
:10AAF80018783138401904F0E1FB574B5FFA80FAB7
:10AB08009B7973B1AAF13003DBB2092B09D8534BF7
:10AB18001B7833B9FDF726FA03E04FF0000A00E08E
:10AB28009A464F4CDFF84C812178DFF84C9111F0B0
:10AB3800010100F06B8198F80030DFF840B1002186
:10AB48008BF80010184605910493FDF703FADFF817
:10AB580030B10599049B002800F0B5804148DFF822
:10AB680024E101709EF800003F4A984213603B4977
:10AB780040F08A8033689B8903F00F03032B21D1AF
:10AB8800A0F1300C0A2000FB0CF0384BDFF8E0C0D5
:10AB980093F800E00390704407900EF1010E1CF842
:10ABA8000000DDF80CC05FFA8EFE106083F800E04C
:10ABB8000CEB0E00DFF8B8E01EF80000002870D19A
:10ABC80018706EE0082B2CD1A0F1300C27480CEB44
:10ABD8008C0E03780793264B9E44079B734493F887
:10ABE8006CE00793224BBEF1000F01D180F800E022
:10ABF80090F800E00CEB8C0C634403EB0E0C0EF1A8
:10AC0800010E5FFA8EFE73449CF86CC093F86C30AA
:10AC1800C2F800C080F800E0002B42D1134803704E
:10AC28003FE0072B0ED130280ED1DFF840E09EF828
:10AC3800003003B10538013303F0010310608EF8CA
:10AC480000302EE0062B2CD10B78013328E000BF12
:10AC5800581400203F140020801400207D14002088
:10AC6800B51400200B2A00208C140020601400204A
:10AC780024F8010820140020621400203B1400204E
:10AC8800401400203D14002099488EF800309BF8AD
:10AC980000304FF0010C80F800C013B10B7863440A
:10ACA8000B7040238BF800300B78BB4202D3914BDA
:10ACB800781E187008781168281804F0F5FA2378B7
:10ACC80043F00403237098F80030232B1ED1894BDE
:10ACD8007A1E1878904219DA0130C0B21870281814
:10ACE800049304F0EBFA049B20B918782021281863
:10ACF80004F0DAFA804B40221A7023787C4A43F039
:10AD08000403237000238BF80030137098F8003088
:10AD18002A2B10D1774B1A786AB1013A1A70764B00
:10AD280040221A702378724A43F0040323700023E8
:10AD38008BF80030137098F80030432B1ED16D4B00
:10AD48001878B84205D228182021049304F0ACFAE8
:10AD5800049B9BF8002032B91B787A1E934202DAD2
:10AD6800644A013313702378634A43F00403237061
:10AD7800002313705E4A8BF8003013709BF8003084
:10AD880013B15E4A013B13709BF80030012B0ED1C2
:10AD9800584B1A78BA4201D201321A70544A002329
:10ADA8001370227842F0040222708BF80030237866
:10ADB80003F00402D2B2002A3BD0514A6FF3820357
:10ADC8001370002111224F48F5F7E4FA4E4A494B17
:10ADD80011781B78994288BF137011780F318B4214
:10ADE80002DD49490F3B0B7048481378017810225F
:10ADF800C9184919434804F072FA4248F5F71AFD90
:10AE0800C2B20F2A15D809EB02000DE011224846FC
:10AE1800F5F7C0FA10222946484604F060FA484679
:10AE2800F5F708FD024648442021C2F11002F5F763
:10AE3800B1FA98F80030532B20D133689A684AF257
:10AE480048139A4208D1284604F038FA20B14AF249
:10AE58001520012104F028FA28463946FCF7CCFFD2
:10AE6800264A00231370294A01201370264A0146F6
:10AE7800137000930246034609F0CAFFFEF75CFC14
:10AE8800204B234A03F1100153F8040B8B4242F87C
:10AE9800040BF9D133689A68122A50D19B7B002B96
:10AEA8004DD0AAF1300A5FFA8AFABAF1090F46D8EA
:10AEB800237813F00107174B08D09A7932B10D4A5D
:10AEC8001178154A1278313A914238DA9B792BB9C0
:10AED800104BDA79114B1B789A4230D00E4B054A49
:10AEE80018781178054A30381278002325E000BF19
:10AEF800601400207D1400200B2A0020401400203C
:10AF0800B514002062140020751400203B140020A2
:10AF180002020020801400203F1400207314002037
:10AF280017B1994200D132B9DFF8F4C04FF02A08BE
:10AF38009C448CF810800133DBB28342F0DB32682A
:10AF480093680B2B01D0122B0AD1334B991D13F8A0
:10AF5800010B202802D10D3003F8010C8B42F6D1E9
:10AF680092684AF248139A4210D12C4B9B796BB1E4
:10AF7800069B5BB10027781904F0A0F918B1284B9B
:10AF88002A22DB191A740137102FF4D1237813F011
:10AF9800010F0ED0234B1B7803F08003DBB243B1C3
:10AFA800214B224A1B78127810339B1A1C4A5F21C6
:10AFB800D1541F4CA37803F00203DBB2002B28D036
:10AFC800FCF72CFE1B49034628B908786522E11DC9
:10AFD800FCF742FE12E03068B4F90430A2798468C4
:10AFE8000978122C01FB023105D1807B18B90B4975
:10AFF800C97902FB0131104804F071F933689B6884
:10B00800122B06D10820014609B0BDE8F04FFCF725
:10B0180095BE09B0BDE8F08F020200208014002020
:10B02800F2010020A82100207D14002075140020C2
:10B03800C414002073140020CB14002024282DE908
:10B04800F041144609D15C4B5C48197880180131ED
:10B058000222FCF7E9FE0234AAE0E72809D1564BA0
:10B0680056481978801801310322FCF7DDFE0334B5
:10B078009EE0A3282AD1504D2B780B2B15D81046CB
:10B088004F49FCF7ABFE4E48F5F7D4FB2A212418AC
:10B098004A48E4B2F5F7FCF9002800F08A802978DC
:10B0A80002220131FCF7C0FE83E05901C918454D61
:10B0B80001F56C516D3110466918FCF78FFE05F5E6
:10B0C80072505830F5F7B6FB241871E0F22821D1F8
:10B0D800394F3A4D3978072605EB0208B1FBF6F1EE
:10B0E800404601310222FCF79FFE39782D23B1FB3F
:10B0F800F6F688F80230F3009E1B8B1B324FDBB24A
:10B1080007EB83031988E21CA9529B78A81883705F
:10B1180006344DE025280BD12C4B46F63E329A805A
:10B1280045229A719A78053842F002029A703CE0FA
:10B138005E280BD1254B46F63E429A8045229A71ED
:10B148009A783E3842F002029A702EE07C280BD1A1
:10B158001E4B46F222029A8011229A719A785C3824
:10B1680042F002029A7020E0EC280BD1174B46F609
:10B1780082429A8045229A719A78CC3842F002022B
:10B188009A7012E0A7280BD1104B46F6A2429A807B
:10B1980045229A719A78873842F002029A7004E040
:10B1A800E02801D1541C03E018B1044B18550134B0
:10B1B800E4B22046BDE8F08173140020F2010020BB
:10B1C800407F0208684202081D660208C414002075
:10B1D80038B50A4B45F655151B78002405FB0305C1
:10B1E80007E0074B22461978FFF728FF041B2D19A3
:10B1F8000446287808B11F2CF3D938BD3E14002026
:10B208007314002070B5002543F6FA44204604F074
:10B2180055F8064604F1080004F050F816F0FF0F40
:10B2280006D020F07F0010F0FF0F01D00135ADB23D
:10B2380046F219039C4201D00934E7E7284670BD5D
:10B2480038B5B0F900500B4C05EBC50505F574553C
:10B258000235284604F032F8C1B211F0800F07D049
:10B2680023882846013B01F07F01238004F01CF865
:10B27800208838BD38140020454B2DE9F74F1B882E
:10B28800444A044689461788DFF80C8123B14FF0F9
:10B29800000A0AE09A4608E00529FBD198F8003030
:10B2A80043F0040388F8003070E098F8003013F099
:10B2B800030F0BD013F0010F02D0B4F1FF3F05D1FB
:10B2C80003F00203DBB21BB1012C01D03F19BFB25E
:10B2D8003BB2B3F1FF3F04D0B3F57A7F08BF002734
:10B2E80001E040F2E7370FFA87FB0BEBCB0303F5DE
:10B2F800725303F17A00019303F0E0FF10F0FF0F9F
:10B30800019B16D0B9F1050F09D103F1820003F0B2
:10B31800D5FF20F07F0010F0FF0FC6D022E0B9F172
:10B32800000F1FD003F1820003F0C8FF00F07F0672
:10B3380018E00AF1010AB4F1FF3F1FFA8AFA04D1B2
:10B3480098F8003043F0010305E0012C05D198F886
:10B35800003043F0020388F80030BAF57A7F0DD048
:10B368003D46A2E74E4505D0B9F1000F02D0B9F12C
:10B37800050F9AD1BAF1000F05D000E03D46054A05
:10B388002DB2156002E0034BC3F800B0BDE8FE8F94
:10B39800381400208C14002090140020F0B5037895
:10B3A8009BB05A1ED2B26B2A0F4600F2C8805E01CB
:10B3B800644AF3189B18644A45F65516127845787E
:10B3C80006FB0236E7213046F5F762F80446F0B985
:10B3D80030467C21F5F75CF80446C0B93046252193
:10B3E800F5F756F8044690B930462421F5F750F899
:10B3F800044660B930464021F5F74AF8044630B9AA
:10B408003046F921F5F744F80446002876D0A41B05
:10B418000FB14E4800E04E4831462246A619F5F7CE
:10B428008FFA3046E721F5F733F830B128466946F8
:10B43800652246F68243FCF70FFC30467C21F5F77F
:10B4480027F850B1691EC9B201EB011101F5C041DD
:10B4580068462231112203F042FF30462521F5F7D4
:10B4680017F838B1681EC0B26946652246F63E3301
:10B47800FCF7F2FB3046F921F5F70AF838B1681EF7
:10B48800C0B26946652246F63E43FCF7E5FB304606
:10B498004021F4F7FDFF50B1691EC9B201EB01115B
:10B4A80001F5E04168467C31112203F018FF30466F
:10B4B8002421F4F7EDFF50B10FB1244800E02448EF
:10B4C800001929460222FCF7AFFC02340BE00FB149
:10B4D8001E4800E01E4800196946F5F74DF9684610
:10B4E800F5F7A8F90419002F29D01A4B9A781C19D6
:10B4F80042F002029A700023E37116E03046F5F735
:10B5080099F905461FB9124831462A4615E0102810
:10B5180010DD2A460D483146F5F712FA0D4B9A7898
:10B528005D1942F002029A70EC7110200146FCF796
:10B5380005FC04E0084831461022F5F701FA1BB073
:10B54800F0BD00BFDA6902083E140020CB140020C9
:10B55800351C0020C4140020020200200C4B1B786C
:10B5680013F0010202D000200A4905E003F00200AE
:10B57800C0B218B108491046FCF730BC03F0040308
:10B58800DBB20BB10549F7E705480121FFF706BF14
:10B5980090140020244A0208034A0208454A020877
:10B5A800B714002070B5124D124C00201249FCF758
:10B5B80017FB2846A1780222FCF736FCE81CE17844
:10B5C8000222FCF731FC05F1080021790222FCF780
:10B5D8002BFC05F10B0061790222FCF725FCA1790F
:10B5E80005F10E000222BDE87040FCF71DBC00BF4B
:10B5F800F2010020B714002034F901082DE9F341C5
:10B608004F4F504C3B689D7C237813F0010F2FD18E
:10B61800022243F6F8410DF1060003F060FE4A4E9F
:10B62800BDF806304FF0FF3033602946FFF724FE9F
:10B63800237843F001032370444B1B7813F0030F66
:10B6480014D1B6F90010424801EBC10101F572515D
:10B658007A31092203F043FE3E4B1B881BB130466A
:10B66800FFF7EEFD10B90020FAF70AF9FFF79AFF85
:10B67800394E3378552B0CD1DFF8D080FCF746FBD8
:10B6880098F800304FF0FF306FF3410388F800302E
:10B698000CE0442B2AD1DFF8B480FCF737FB98F88C
:10B6A800003001206FF3000388F800302946FFF7C7
:10B6B800E3FD98F8003013F0030F15D1224D24480C
:10B6C800B5F90010092201EBC10101F572517A3177
:10B6D80003F005FE1F4B1B881BB12846FFF7B0FD82
:10B6E80010B90020FAF7CCF8FFF75CFFFFF736FF38
:10B6F8003378232B21D1154B1A7802F0FC026FF313
:10B7080082021A70FCF72EFC144B9A786FF34102F0
:10B718009A70134B1D782DB9FCF704FBFCF7F6FA69
:10B728003D600AE02278013DEDB242F00602227047
:10B738001D700C4B53F825303B60BDE8FC8100BF01
:10B7480058140020B51400208C14002090140020F8
:10B75800B71400203814002020140020C41400203E
:10B76800A3140020A41400202DE9F0411646104A25
:10B778000F4653780E21C3F342034B43117803F568
:10B78800EC433C330B4D01F00701044603EB410148
:10B79800022203F0A4FDE81921780222FCF744FBF9
:10B7A8006178A8190222BDE8F041FCF73DBB00BF53
:10B7B80078140020F2010020044B02225978044B2F
:10B7C800C1F3420118180131FCF72EBB7814002090
:10B7D800F201002010B5074B074C1B78074A03F00D
:10B7E800070304EB83031C88111814529B788B7091
:10B7F80010BD00BF781400201D660208F201002069
:10B80800084B1B789B0902D0012B06D102E01020BF
:10B81800054904E01020054901E005491020FCF71E
:10B82800DDBA00BF78140020635602088456020867
:10B83800A55602082DE9F041DFF868800F4698F810
:10B848000010174DC1F382010446164605F10800A1
:10B8580001310222FCF7E8FA98F80010042201F0FE
:10B868001C0101F50A412431204603F038FDE8198E
:10B8780021780222FCF7D8FAF81C281861780222ED
:10B88800FCF7D2FAA819A1780222FCF7CDFAF01C2D
:10B89800E17828180222BDE8F041FCF7C5BA00BFDC
:10B8A800F20100203C140020064B1B7803F08003B3
:10B8B800DBB233B1435C04482021C0180222F4F7FC
:10B8C80069BD7047A8210020F20100202DE9F74347
:10B8D800484D494C2B6821789B68022203EB4101B3
:10B8E8000DF1060003F0FBFCBDF806604FF4616340
:10B8F800B6FBF3F103FB11663C22B6B2B6FBF2F3DA
:10B9080002FB13665FFA81F8DFB23A3A3B484146D8
:10B91800FCF78AFAF6B2022239483946FCF784FA6B
:10B92800022238483146FCF77FFA374BA9461B7884
:10B9380013F0010F4BD0354B354D1878232804D11F
:10B948002B78012B3FD8013305E02A2805D12B7825
:10B95800002B38D0013B2B7035E0A0F13003DBB26F
:10B96800092B01D9432828D12B7833B94146112214
:10B97800FDF702FF5FFA80F80CE0012B05D139468C
:10B988003B22FDF7F9FEC7B204E031463B22FDF742
:10B99800F3FEC6B23946324640460BF04AFED9F8A5
:10B9A8000030ADF806009B6820780DF1060103EB26
:10B9B8004000022203F08DFC05E0532803D1002348
:10B9C8002B70FDF7B9FE13482978FFF76DFF652244
:10B9D800207800231049FCF73FF905200B21FCF7DC
:10B9E800ADF921780D4801310222FCF71DFABDE8B6
:10B9F800FE8300BF581400207314002002020020A8
:10BA08000802002010020020B51400202014002095
:10BA18007D14002045F90108CB140020F301002013
:10BA280073B59A4B9A4D1A7812F0010F05D12A78FE
:10BA380012F0380204BF2A706A701A78934E42F0E6
:10BA480001021A702B78924C13F038023ED19149BA
:10BA58000978552904D113F0070F2FD0DA1D0AE011
:10BA680044290CD103F0070201323D3992FBF1F170
:10BA7800C800411A521A62F3020323701EE05329C8
:10BA88000AD1C3F3C201013161F3C503237063789E
:10BA980062F34303637011E023290FD1FCF762FAC4
:10BAA80033787D4A43F0060333701378013BDBB2E9
:10BAB80013707A4A52F82320794B1A60002079498A
:10BAC800FCF78CF91C20FFF785FEDDE0082A2ED153
:10BAD80075490020FCF782F90620FFF76DFE0C205F
:10BAE800FFF778FE1521182201A8FFF73DFE694BE4
:10BAF8001B78552B06D1637803F0FE03C3F342028B
:10BB0800013A07E0442B0BD1637803F0FE03C3F33B
:10BB18004202013202F0030262F343036370B3E0AE
:10BB2800532B28D0232B40F0AF802378A6E0102A8F
:10BB380051D15D490020FCF751F90620FFF73CFE82
:10BB48000C20FFF747FE1521182201A8FFF70CFE6D
:10BB58006178564801F00101FFF7A6FE4D4B1878B1
:10BB6800232801D02A2804D16378DA4362F300033A
:10BB7800D4E7532804D12378C3F3C202013280E00A
:10BB8800A0F13003DBB2092B01D943287CD16B78B3
:10BB980002AA03F001033B21D41883F001024B43AE
:10BBA800172606FB023214F8041CFDF7E5FD04F81D
:10BBB800040C6B780E22C3F342035343287803F531
:10BBC800EC433C3300F0070003EB400001A90C3ABA
:10BBD80003F07FFB58E0182A4DD133490020FCF7C9
:10BBE800FDF80620FFF7E8FD0C20FFF7F3FDFFF74F
:10BBF80007FE284B1B78552B07D1237813F0C00F6D
:10BC080042D0C3F38112013A06E0442B07D12378CE
:10BC18009A09012A38DC013262F3871333E0232BB7
:10BC280004D12378C3F3C202023A2AE0532B2BD162
:10BC3800FCF798F933781E4A43F006033370164B25
:10BC48001648197840F82120013119702378C3F378
:10BC5800C201013161F3C503C3F381112370104B95
:10BC680011B1012904D101E01C3202E0114A00E0BF
:10BC7800114A1A6008E0114A00211170C3F3C20288
:10BC8800013A62F3C50323707CBD00BFB5140020E0
:10BC98007814002020140020A3140020A4140020ED
:10BCA80058140020215602084256020848F9010893
:10BCB8004CF9010884F90108A0F901087D14002055
:10BCC80073B5494B494D1A7812F0010F04D12A78FF
:10BCD80012F0030208BF2A701A78434E42F001029C
:10BCE8001A702B78414C13F003022ED1404A127877
:10BCF800552A03D1C3F38202013A04E0442A06D14B
:10BD0800C3F38202013262F38403237017E0532ADB
:10BD180003D15A1C62F30103F7E7232A0FD1FCF77A
:10BD280021F93378334A43F0060333701378013B23
:10BD3800DBB21370304A52F82320304B1A6001A846
:10BD480010211B22FFF776FD4CE0012A4AD101A8F9
:10BD580010211A32FFF76EFD254B1878232804D1DD
:10BD68002378C3F34112013205E02A2807D123784A
:10BD7800C3F34112013A62F3461323702CE05328AF
:10BD880004D12378DA1C62F30103F6E7A0F130034B
:10BD9800DBB2092B01D943281ED12B7802AAC3F3A1
:10BDA8004113D4180C215A1C03F001034B4302F031
:10BDB80001021F2614F8041C06FB0232FDF7DCFC06
:10BDC80004F8040C287801A900F01C0000F50A40CA
:10BDD8002430042203F07DFA29780948C1F341117F
:10BDE800FFF762FD7CBD00BFB51400203C140020A5
:10BDF80020140020A3140020A414002058140020AC
:10BE0800BCF90108064B1B7803F08003DBB233B1A1
:10BE1800435C04482021C0180322F4F7BBBA7047DA
:10BE2800A8210020F20100204328F8B504460D4659
:10BE3800174606D1104B00261A786FF3C3021A7002
:10BE480000E00E462046FCF785F890B10A4B303CDE
:10BE58001A780A2602F00801C9B2002918BF00257D
:10BE680006FB05466FF3C30236B21A70BE42A8BF7E
:10BE78003E4630B2F8BD00BFB51400202DE9F341AD
:10BE88006E4F6F4E3B7843F001033B70347844B9F2
:10BE98004AF28E1003F012FA6A4B6B49186020467A
:10BEA80017E0012C02D10020684912E0022C02D1CF
:10BEB800002067490DE0032C02D10020654908E005
:10BEC800042C02D10020644903E0052C03D1634906
:10BED8000020FBF783FF3178D9B9614B1B78312BF0
:10BEE80001D1013101E0302B05D1564B4AF28E10B9
:10BEF800196003F0D9F95B4B1A785B4B02F08002AA
:10BF0800D2B20AB1202202E04E4A12683032DA7701
:10BF18006EE001290BD002290CD003290DD0042989
:10BF28000ED04AF28A15052918BF00250AE04AF200
:10BF38007A1507E04AF27E1504E04AF2821501E01C
:10BF48004AF286152946042201A803F0C8F9474B8E
:10BF5800474A03F1100153F8040B8B4242F8040BD3
:10BF6800F9D1032243489DF80410FBF75DFF032233
:10BF780041489DF80510FBF757FF03223F489DF8FD
:10BF88000610FBF751FF3E4803229DF80710FBF708
:10BF98004BFF334B3B4C1878232804D12378022BD2
:10BFA80022D8013304E02A2804D12378E3B1013BE5
:10BFB800237019E0A0F13003DBB2092B01D9432823
:10BFC80012D194F8008002AA904418F8041CFF22A9
:10BFD800FFF72AFF08F8040C207802AA131813F8B0
:10BFE800041C281803F060F927482178FFF70AFF96
:10BFF8001B4B1B78532B1FD1224B00221A7033780E
:10C008000133DBB2062B337004D0012B14D10D4B56
:10C018001B688BB1FDF790FB002333703B781B4AFC
:10C0280043F006033B701378013BDBB21370184AE8
:10C0380052F82320174B1A60BDE8FC81B514002084
:10C04800731400208C140020659002088E91020859
:10C05800AF910208D0910208F191020812920208E9
:10C0680020140020A8210020F2010020BDAD020804
:10C078000202002003020020070200200B02002019
:10C088000F0200207D140020C0F90108A31400202D
:10C09800A41400205814002070B5174C0D464A22ED
:10C0A800002106462046F4F775F9FF2D0AD1B100A4
:10C0B80001F5D64120463E31042203F010F92378D9
:10C0C8009BB970BDFE2D01D1173E02E0FD2D02D1B6
:10C0D8000136267009E0B60006F5D6403E30401914
:10C0E80003F0ECF8C0B2207020B10348BDE87040FE
:10C0F80011F084BF70BD00BF641600202DE9F04127
:10C1080011F0ACFF60B110208F49FBF767FE8F4B31
:10C118001B78432B40F0EE81BDE8F04111F0C0BF21
:10C1280011F0AEFF002826D0894C23786BB110207F
:10C138008849FBF753FE88482D211030F4F7A8F9F9
:10C14800002800F0D781217810E010208349FBF700
:10C1580045FE81482D211030F4F79AF9044600284D
:10C1680000F0C88111F0A4FF014620468222BDE8F4
:10C17800F041FBF759BE7A4C43F6CC2223689B6802
:10C18800934250D0774E744D307803EB800003F023
:10C1980095F8032201467448FBF746FE2368986821
:10C1A80046F6A24398422BD0203B984228D03378B9
:10C1B800013000EB830003F081F80322014605F10A
:10C1C8001500FBF731FE236830789B68023303EBD8
:10C1D800800003F073F80322014605F11900FBF70C
:10C1E80023FE236830789B68033303EB800003F059
:10C1F80065F80322014605F11D00FBF715FE0EE068
:10C208002D2103225948F4F7C5F82D210322584857
:10C21800F4F7C0F857482D210322F4F7BBF8202380
:10C228002B772B762B75544B1B7813F0010F00F0EE
:10C23800BD80236843F6CC229B68444D934261D06D
:10C248004E4E484F32783878D31803EB800003F00D
:10C2580035F84B4B0146186028789846A0F1300213
:10C26800D2B2092A01D943280FD109B2BA22FDF75F
:10C2780083FA236832789B680146C8F8000038784A
:10C28800D31803EB800003F00FF82B782A2B04D186
:10C29800337813B1394A013B13702B78232B0ED115
:10C2A8003378022B0BD8226846F6824192688A427C
:10C2B80005D020318A4202D0304A013313702B78DE
:10C2C800552B01D0442B0FD1236831789B68A3F5F7
:10C2D800D643B3F13E0248BFA3F13B023B7803EBE0
:10C2E800A202D0B2FFF7D8FE264B1B7803F08003DA
:10C2F800DBB23BB13278184B03EB820320225A742D
:10C308009A74DA742B78532B06D023689A6843F60C
:10C31800CC239A4240F0EE80FBF724FE236846F6D1
:10C328003E329B68934203D10E4B0220197806E0F7
:10C3380046F6A242934227D10A4B002019780131D0
:10C34800BDE8F04108F038BD7A7E020820140020CC
:10C3580004100020517D0208F20100209B7E020893
:10C368005814002073140020030200200702002044
:10C378000B0200200F020020B51400207D140020BD
:10C388008C140020A821002046F68242934204D152
:10C39800594B012019780918D2E746F63E429342D4
:10C3A80040F0A880544B03201978C8E7236849F265
:10C3B800EE429B6893423ED14F4E10204F49FBF707
:10C3C8000DFD31784E4D01EB011101F51441EE31AF
:10C3D8001022284602F083FF2B4605F110012A4659
:10C3E8001078474F78B94749FBF7F8FC3846E721FA
:10C3F800F4F74EF878B13178401B38180131032230
:10C40800FBF712FD07E013F8010B10B9203003F811
:10C41800010C8B42E4D13C4D2B782A2B03D1307888
:10C42800FD21FFF739FE2B78432B63D13078236841
:10C438000130C0B259E043F6CC229342324E1AD0B2
:10C4480010203249FBF7CAFC33782A2B52D1304BE3
:10C458001B689B68A3F5D643B3F13E0248BFA3F11E
:10C468003B02254BFF211B7803EBA202D0B2BDE8AB
:10C47800F041FFF711BE33781F4D552B04D12B78AF
:10C48800142B01D1033B2B703378442B05D12B7827
:10C49800122B02D1184B15221A702B78DFF87480F2
:10C4A8005901C918414401F5725100207931FBF74F
:10C4B80095FC08F56E51102071312F78FBF78EFC32
:10C4C8003378112F8CBF032700272A2B05D1287812
:10C4D800FE21C01BC0B2FFF7DFFD3378432B09D123
:10C4E8002B78173BDF1B2368F8B2997CBDE8F04135
:10C4F80011F09CBDBDE8F08173140020597E02083C
:10C50800F20100204F64020820140020177E020860
:10C51800581400206842020810B50E4B1B78452BB2
:10C5280017D10D4B1A7842F006021A700B4A13788D
:10C53800012B0ED80A490B4C086844F82300013334
:10C54800137083680B60FBF743FBBDE81040FBF7F3
:10C5580009BD10BD20140020B5140020A31400202C
:10C5680058140020A414002010B50C4B0446214692
:10C57800D8790BF020F868B1094B1B5D543BDBB24E
:10C58800012B09D820460AF00DFFD0F1010038BF71
:10C59800002010BD022010BD022010BD8014002014
:10C5A800A122002008B50AF0F5FFC0B208BD0000BE
:10C5B8002DE9F047634B644C1A78994612F0010F45
:10C5C800624D65D02078FFF7CFFF614A2B181178AC
:10C5D800604F93F8A031604E44293870336090461C
:10C5E8000AD12D2B08D038B995F8A11101233B7039
:10C5F80031602078FFF7D6FF98F80030552B10D11E
:10C6080033682D2B0DD03B785BB1013B514ADBB22F
:10C618001370EB1893F8A0114F4B20781960FFF7AF
:10C62800C1FF98F80030232B19D14C4B20781B6898
:10C638009B7C013B984212DA434B0130C0B2187020
:10C64800FFF792FF3870281890F8A0313360444BF8
:10C658009B7803F00203DBB20BB1FBF763FB98F89E
:10C6680000302A2B14D1207890B1374B0138C0B252
:10C678001870FFF779FF3870281890F8A0313360E8
:10C68800374B9B7803F00203DBB20BB1FBF74AFB95
:10C69800344EFDF751F8237832789A4288BF3370C8
:10C6A80032780F32934202DD2E4A0F3B1370DFF8C7
:10C6B800C480002730783818C0B2FFF755FF281813
:10C6C80090F8A0310137102F08F8013F07D0254B0B
:10C6D8001A78224BBA181B689B7C9A42EADB99F8B5
:10C6E800003013F0010F13D01F4B1A781F4B02F0C4
:10C6F8008002D2B22AB1227831781032521A5F21E0
:10C7080005E0227831781032521A13490968995491
:10C7180013498B7803F00203DBB253B12078073159
:10C72800652246F63E43FBF797FA05200B21FBF7F7
:10C7380005FB21780E4801310222BDE8F047FBF7DE
:10C7480073BB00BFB51400207D14002024F8010835
:10C75800201400203A1400208C14002058140020C3
:10C76800C414002075140020A8210020F201002024
:10C77800F3010020010200202DE9F0410746104690
:10C788000D461446F4F756F8C3B28046B3B1AB422F
:10C7980014D80B4E20212A46F019F3F7FBFD20464A
:10C7A800F4F748F8C8EB05056D08EDB2EF19024635
:10C7B8002146F019BDE8F041F3F744BDBDE8F0812A
:10C7C800F2010020F0B5134B1A1894781F4604B3F1
:10C7D8000E7800233A1892781A4112F0010F4FF0A0
:10C7E80001020DD0A6420D7803D09A4042EA050511
:10C7F80004E09A40C2F10F0202EA05050D7005E057
:10C808009A400D78C2F10F022A400A700133042BB6
:10C81800E0D1F0BD801400203122002301781941B5
:10C8280011F0010F02D00449C9188A750133013289
:10C83800042BD2B2F2D17047F2010020034670B542
:10C848000846684A31B11278532A40F0C980533AF1
:10C858001A7070BD1278302A24D163491C780A787E
:10C8680022400FD00A78024112F0010F06D00122AF
:10C8780082401C78C2F10F0222401A70013004284D
:10C88800F0D10CE00878104110F0010F04D001201D
:10C8980090401C78204318700132042AF2D1534882
:10C8A80000211AE0A2F13100C0B2032825D84E4A6F
:10C8B8001278024112F0010F00F092801C7854FAAD
:10C8C80000F212F0010F4FF001020BD08240C2F1CA
:10C8D8000F0202EA040445481C701322BDE87040A8
:10C8E800F3F758BD82404149441C4C741C782243DC
:10C8F8001A70102246F682436EE0132A0BD0552A8E
:10C9080017D13B4A3B491278122000FB0212527899
:10C9180012F0200F64D00024344D194620466C7460
:10C92800FFF750FF304B9B78002B59D02046294603
:10C938004FE0142A0BD02A2A16D12D4A2D491278F5
:10C94800122000FB0212527812F0200F48D0274C18
:10C958000022194662740120FFF734FF224BDB786E
:10C96800002B3DD0012033E0152A0BD0232A16D105
:10C978001F4A20491278122000FB0212527812F046
:10C98800200F2DD0194C0022194662740220FFF79F
:10C9980019FF154B1B79002B22D0022018E0162A0C
:10C9A8000BD0442A1CD1124A12491278122000FBDB
:10C9B8000212527812F0200F12D00C4C00221946A5
:10C9C80062740320FFF7FEFE074B5B7943B1032037
:10C9D8002146102246F6A243BDE87040FBF73CB959
:10C9E80070BD00BF201400208014002022140020F5
:10C9F80076140020552200202DE9F04F87B09DF8CD
:10CA080040508046072D0E4605929A4637D100249D
:10CA180027463378234113F0010F2CD0012523B288
:10CA28004FF000080293512029462A462B460095CC
:10CA3800CDF8048002F0B6FC1B204146621943463B
:10CA4800CDF80080F5F78CFB37B9112039463A4606
:10CA58002B460097F5F784FB534B204613F8242008
:10CA680001276FF3000203F824201199F6F7A4F9BF
:10CA78002046F6F76DFB0134042CCAD1F7E1012DED
:10CA880003780CD10BB90B7823B3FF230093002153
:10CA9800464B01911B780C200133029316E0022DBE
:10CAA80009D10BB90B78ABB10021FF230093019199
:10CAB800029134200AE0062D0CD10BB90B784BB14A
:10CAC8000021FF23009301910291652004220B4667
:10CAD80002F068FCBAF1010F98F800302BD13BB195
:10CAE800334B0020D979024653460090F5F738FBBE
:10CAF80033783BB12E4B0120D979002203460092AE
:10CB0800F5F72EFB0020F6F749F998F80030002BCE
:10CB18005BD0284B1978002957D1274B1B78002B5D
:10CB280053D0FF2300933A2001220B460191029132
:10CB380002F038FC49E063B1052D4FF0000102D145
:10CB480000910F2001E000910B200A460123F5F720
:10CB580007FB337883B1052D4FF0000106D1102073
:10CB68000A4601230091F5F7FBFA12E00C200A4669
:10CB780001230091F5F7F4FA022D25D0032D01D1F8
:10CB88000E4B02E0042D02D10D4B1F781DE0052D40
:10CB980001D10C4BF9E7012D01D1044BF5E7062D26
:10CBA8000CBFFF27002710E031120020721200206E
:10CBB800801400202B1200201F0E002018160020C1
:10CBC800E32800208C230020FF2798F80030002B52
:10CBD80000F09D80914C237803F02003DBB26BB109
:10CBE8008F4B197811F0010108D1FF2300932820F9
:10CBF80001220B460191029102F0D4FB237803F045
:10CC08001003DBB273B1864B197801F00201C9B287
:10CC180041B9FF230093292001220B46019102917B
:10CC280002F0C0FBE37813F0010F0ED07C4B1978AB
:10CC380001F00401C9B241B9FF2300932A2001225F
:10CC48000B460191029102F0ADFBE37803F0020379
:10CC5800DBB273B1724B197801F00801C9B241B95E
:10CC6800FF2300932B2001220B460191029102F031
:10CC780099FBE37803F00403DBB273B1684B1978CE
:10CC880001F01001C9B241B9FF2300932C20012201
:10CC98000B460191029102F085FBE37803F008034B
:10CCA800DBB273B15E4B197801F02001C9B241B90A
:10CCB800FF2300932D2001220B460191029102F0DF
:10CCC80071FB0CF015FD70B1554B197801F040015E
:10CCD800C9B241B9FF230093492001220B460191B3
:10CCE800029102F05FFBE37803F04003DBB273B11B
:10CCF8004B4B197801F08001C9B241B9FF23009369
:10CD08004E2001220B460191029102F04BFB119B30
:10CD1800444A1978444B51B198F800101170327890
:10CD28001A7033780BB1542005E0522003E01170DB
:10CD3800327853201A7002F0AFFE119B00241A7843
:10CD48003A4B1A7098F80030234113F0010F2DD098
:10CD58002146059810F0DCFB0122014628B923B2D0
:10CD6800019000920293104605E0002123B2009240
:10CD78000191029324200B4602F014FBBAF1010F33
:10CD880005D12B4B8020DA790521013208E0022DEC
:10CD980007F1010202D18020072101E0802006214D
:10CDA8002346F6F7EFFC2046F6F7A6F93378234139
:10CDB80013F0010F57D000214FF0010B23B202935B
:10CDC80002205A460B46CDF800B0019102F0EAFA6B
:10CDD800DA45DFF868900CD119F8243013EA0B0310
:10CDE80034D1134A0520D1790093594404EB0B023E
:10CDF8002AE019F8243013F0010327D1022D1FD19E
:10CE08000C4B1B7803F02403042B04BF0A4B83F854
:10CE180000B000230093072014E000BFA8210020E1
:10CE28002D13002051120020521200203813002028
:10CE3800801400203C130020180E0020311200201E
:10CE480000930620791C621CF5F78AF9119920468F
:10CE5800F5F7B2FF2046F6F77BF919F824306FF39F
:10CE6800000309F824300134042C7FF46BAF07B0B9
:10CE7800BDE8F08F2DE9F74F16469A4633780446F9
:10CE88000F469DF830909DF834B09DF83820DFF8B3
:10CE98007C8043B102EA03033370097898F80020D4
:10CEA8008A18D31A0370164B00251D70217843F693
:10CEB800ED2002F0F9F9494646F2A75002F0F4F9DC
:10CEC800104B31465D7052464B463846CDF800B09F
:10CED8000194FFF791FD2046F8F70AFD23780A48E8
:10CEE8000A4988F80030F6F7E1F88AF800503570FA
:10CEF8003D70257003B0BDE8F04F02F0DDBC00BF07
:10CF0800B41400201F0E00202E1300202B12002026
:10CF18002DE9F04180460E46174646F26865002422
:10CF28003846214610F0F4FA88B1294602220B4807
:10CF380002F0D5F90948414610F08EFA074810F07A
:10CF4800BAFA20B90123A34032781343337001346D
:10CF58000835042CE4D1BDE8F08100BF3613002069
:10CF68002DE9F04387B08046894604A847F252016C
:10CF7800082202F0B4F900244046214610F0C8FA0D
:10CF880038B301260223A719002100933BB20025DC
:10CF9800029323200B460422019602F003FA394635
:10CFA80032462B4611200095F5F7DAF80420214681
:10CFB8002A4633460095F5F7D3F8B9F1000F08D0A3
:10CFC80004A8214610F0A4FA18B10548214610F02B
:10CFD80089FA01340C2CCFD107B0BDE8F08300BF2B
:10CFE8004612002010B50A4B0A4C1B8801460A4815
:10CFF800238010F05DFA2146074810F02DFA064804
:10D0080010F059FAD0F1010038BF002010BD00BF60
:10D01800381A002032130020361300202DE9F04F73
:10D02800764B774EF0221A7033788BB00B2B40F08A
:10D038008280DFF81C822021EC3A7248F3F7AAF9C3
:10D0480098F80270012F06D96F4900200BB0BDE88F
:10D05800F04FFAF7C3BE6D4D19D16D4B6D4A6E494D
:10D068006E4800246E4E1C7014700C70047088F8A2
:10D0780002400097019436780296FFF7FBFEFAF714
:10D0880071FF2C600BB0BDE8F04FFAF73FBE624964
:10D098006448F6F70BF8644B644F1B88644A3B807E
:10D0A800644B127819782B68532A9B7C09D05A1E36
:10D0B80048BF9A1DD71001374F4307F5CA47A8370D
:10D0C8003AE05D49574810F0C7F95648FFF78AFF1C
:10D0D800044618B1052388F80230BCE1022246F262
:10D0E800A851504802F0FBF84E49544810F0E0F9B6
:10D0F800022246F60A21384602F0F1F83946494834
:10D1080010F0CBF947480121FFF72AFF454840496D
:10D11800414AFFF7FDFE01230093414B01941B7820
:10D128003E4802933C493B4A394BFFF7A3FEFAF7C6
:10D1380019FF2C608FE10027414B344D1A78414C80
:10D1480012F0010F00F0A480394B1A789846432A50
:10D1580021D133780B2B1ED13248217810F0D8F921
:10D16800C8B13248217810F0D3F9A0B920780FFA65
:10D1780087F909EBD00002F0A1F82378012103F028
:10D1880007029140304A80EA0101116009EBD3009F
:10D19800C9B202F089F898F80030232B10D12A6818
:10D1A8002378927C013A93420ADA264A01331370B3
:10D1B800264B9B7803F00203DBB20BB1FAF7B2FD02
:10D1C80098F800302A2B0CD1237853B11D4A013B23
:10D1D80013701E4B9B7803F00203DBB20BB1FAF716
:10D1E800A1FD98F80030552B3ED129682278897C1A
:10D1F800144B08398A422DDA08322CE0C114002079
:10D20800B4140020020200201565020858140020FA
:10D2180021140020B6140020C21400205C14002041
:10D228008014002039130020381A0020281200200A
:10D2380020140020731400204A1200204F120020EE
:10D24800B51400207D1400208C140020C414002084
:10D258001F0E002000221A70804B9B7803F00203F7
:10D26800DBB20BB1FAF75EFD98F80030442B0FD112
:10D2780022787B4B072A9CBF2A68927C083A1A704E
:10D28800764B9B7803F00203DBB20BB1FAF74AFD49
:10D29800FCF752FA734A237811789046994288BF6E
:10D2A800137012780F32934202DD6E4A0F3B1370EF
:10D2B8002B684FF0000B93F81290CDF81CB0B9F121
:10D2C8000F0F9ABFC9F120095FFA89F94FF01009C9
:10D2D8003B4630784FFA8BF20B2805D198F80010AE
:10D2E8005218D210604904E098F8001052185F49AB
:10D2F800D2108F5C98F800104FFA8BF251180B2857
:10D3080001F0070A13D118B200EBE1000692059369
:10D3180001F0D4FF5349069A0978C0B20790511812
:10D328005348C910415C059B07EA0101099131780E
:10D33800089198F8001052183CE0DDF81CC04CFA2F
:10D348000AF111F0010F4B490CD108980B280BD1A9
:10D3580049484FEAE20C10F80C0040FA0AF010F0C5
:10D36800010F01D12A2013E0DDF824C04CFA0AF09D
:10D3780010F0010F04D008980B2801D14D3007E0B8
:10D3880047FA0AF000F0010000280CBFA520DB20B6
:10D398000AF1010A5FFA8AFA01F809000BF1010B98
:10D3A80009F101090132BAF1080F5FFA8BFB5FFA44
:10D3B80089F903D0B9F1200FBFD10CE0B9F1200FE2
:10D3C80009D098F800204FFA8BF189182A68927CC6
:10D3D8009142FFF67EAF29490B7813F0010F17D061
:10D3E8002B68274A9B7C12780F2B02F0800298BF8B
:10D3F800C3F11003D2B294BFDBB2002342B122784A
:10D4080098F800101032521A1A49CB185F21995413
:10D41800124EB37803F00203DBB253B12078F11D4A
:10D42800652246F63E33FAF717FC05200B21FAF77A
:10D4380085FC2B689B7C0B2B0DD9B37803F002037A
:10D44800DBB243B121780F48013102220BB0BDE8AD
:10D45800F04FFAF7E9BC0BB0BDE8F08FC414002018
:10D468007D140020751400204A1200206412002048
:10D4780028120020F201002039130020B5140020E2
:10D48800A8210020F301002010B50A4CA37C4BB161
:10D4980000200949FAF7A2FC084B1B78432B01D15D
:10D4A800433BA374A07C20B90549BDE81040FAF7B6
:10D4B80095BC10BD2214002091640208201400209D
:10D4C80070640208034B1A7801321A700123037042
:10D4D800704700BFB41400200A4A10B50024147025
:10D4E800094A0A4B14700A4A9C701470094A5C7005
:10D4F8001470094A1470094A1470FAF733FD084B7E
:10D508001C6010BD80140020211400201F0E002074
:10D51800B6140020C21400205C140020B4140020AB
:10D52800581400202DE9F041002386B08DF81730FB
:10D53800884B1B78012B00F0EA81874C874D2378B4
:10D5480043B12B78002B40F0A680FAF70BFD082397
:10D558002B70A0E02A78072A00F29D80804A127872
:10D56800232A13D12B70FAF7FDFC7E497E4A0B78EB
:10D5780053B17E48013B0478DBB244F006040470E2
:10D588000B707B4951F8233013605FE2774B1A78B0
:10D5980012F0010F04D101210A438DF817101A70F7
:10D5A800F5F744FA28B92B781BB90DF11700FFF7E6
:10D5B80089FFF5F749FA30B92B78012B03D10DF122
:10D5C8001700FFF77FFFF5F74DFA30B92B78022BDC
:10D5D80003D10DF11700FFF775FFF5F74FFA30B9D2
:10D5E8002B78032B03D10DF11700FFF76BFFF5F72D
:10D5F80053FA48B9F5F76CFA30B92B78042B03D1F4
:10D608000DF11700FFF75EFFF5F7A0FA30B92B7898
:10D61800052B03D10DF11700FFF754FFF5F78AFA30
:10D6280030B92B78062B03D10DF11700FFF74AFF0D
:10D63800F5F740FA30B92B78072B03D10DF1170015
:10D64800FFF740FF9DF817302BB32B78072B1FD817
:10D65800DFE803F004070C0F1215181B00204549DA
:10D6680001E045490020FAF7B9FB14E000204349DE
:10D67800F9E700204249F6E700204249F3E7002095
:10D688004149F0E700204149EDE700204049EAE739
:10D69800FAF768FCDAE12B78304F082B40F0A280CB
:10D6A800324B2F4F1978984611F00101394E23D18A
:10D6B80013223046F2F76EFE0123B374364A2378FC
:10D6C800137003B9B374B37C13B1344B00221A70CE
:10D6D800FFF7DAFE3048B17CFFF7B0F898F8003071
:10D6E80003F0FD0343F0010388F800302C4B1A784F
:10D6F80012B13A7000221A703B78002B5ED0FFF707
:10D70800C3FE2548B17CFFF799F8234B1A78984651
:10D7180022B1002010211F4AFFF72EF8237838780D
:10D7280098F800401F4924EA030252380A70C0B230
:10D738001D4A23EA0403012813703FD8002C37D16F
:10D74800002B35D001230093184B01941B78124805
:10D7580002931FE1C11400202B120020B4140020F2
:10D7680020140020A314002058140020B514002011
:10D77800A4140020D2680208B1680208F3680208FD
:10D7880014690208356902085669020877690208AF
:10D7980098690208221400205C140020180E00204A
:10D7A80077140020C2140020B61400208014002032
:10D7B800814B04229A702B7801332B707F48FFF736
:10D7C8002BF8737C002B00F041817D4A127802F01F
:10D7D8008002D2B2002A00F039817A4AD318202276
:10D7E8005A7533E1092B31D1774806F08FFBC6B261
:10D7F800714C2EB3A378042B02D10020734903E0A7
:10D80800022B04D172490020FAF7E8FA02E00BB9BA
:10D818000433A370314602226A48FAF705FB6D4BC0
:10D828001E78232E73D03046FAF794FB002800F0B8
:10D838000D81312E40F00A812B7801332B7002E0E4
:10D848003B7801333B700823A370FFE00A2B40F0BC
:10D85800FD805D48002106F031FBC4B2002C4CD09D
:10D86800554F7B783E466BB95B4BD879F7F7A6FFE7
:10D8780010B90323FB704AE0BE2010F031FC7B781E
:10D8880001337B70B3784C4A092B02D900205349E5
:10D8980015E010D1504B00241C709470504B514A25
:10D8A8004949464801251C7014700C700470009595
:10D8B800019402946FE0082B04D14B490020FAF739
:10D8C8008DFA11E0062B02D100204849F7E7042B16
:10D8D80002D100204649F2E7022B02D10020454937
:10D8E800EDE70BB908339370B378082B0BD835489C
:10D8F80021460222FAF798FA05E001230093364BF5
:10D9080001941B7842E0334F3C78232C02D1FFF777
:10D91800E3FD9BE02046FAF71DFB002800F0968007
:10D92800303CE4B2631EDBB2012B3C703AD8022CC7
:10D93800294D26D1E879F7F741FF002839D02E483C
:10D94800FFF750FB002834D1224646F2A8512B4855
:10D9580001F0C5FC284929480FF089FD22462749CE
:10D9680046F2A85001F0B5FC244925480FF0A0FD67
:10D9780021480121FFF7F4FA1F481949124AFFF715
:10D98800C7FA01230024009301942B780B480E4911
:10D99800144A0293124BFFF76DFAFAF7E3FA194BA0
:10D9A8001C6053E0032C51D10B4BD879F7F706FFD5
:10D9B80050BB0C23B37049E01F0E00205C140020FC
:10D9C800A8210020F2010020C21400205765020897
:10D9D80078650208201400208014002015650208CC
:10D9E80021140020B6140020B2640208D36402088F
:10D9F800F464020836650208391300202812002052
:10DA08004F120020581400200024124821460FF01D
:10DA18007FFD28B1E02010F063FB204610F098FB52
:10DA280001340C2CF1D1022246F60A200A4901F0F1
:10DA380050FC0023B3702B78084A01332B70084B35
:10DA48001A60084B1A7842F006021A7006B0BDE850
:10DA5800F08100BF391300204F120020C8F90108D7
:10DA680058140020B51400201FB5044611B1002039
:10DA78000B4901E008460B49FAF7B0F92178102262
:10DA88000139C9B201EB011101F5C04122316846E3
:10DA980001F025FC102001466A46FEF76DFE1FBD09
:10DAA80078440208BA4402080B4B1B78442B06D072
:10DAB800552B037801D013B17047013B01E003787F
:10DAC8000133037003780BB9203302E0212B01D115
:10DAD800203B0370FFF7C8BF201400202DE9F74F43
:10DAE800DFF8C881DFF8D4A198F80030554643F034
:10DAF800010388F800309AF80130624C23F07F0364
:10DB08009B46D3B100206049FAF768F95F482A219B
:10DB1800F2F7BEFC18B121788222FAF785F922784B
:10DB2800002A40F0AB802B6862F3CF332B60584B50
:10DB38001A7842F003021A70A0E0DFF854912370BB
:10DB480099F800304E4603F00202D2B20192514FCA
:10DB5800002A40D013F0010813D058464E49FAF76E
:10DB68003DF93B78232B20D14C4B4D4A4D481A6048
:10DB78000121FFF779FF337803F0FE036BF34103CC
:10DB880012E040464849FAF729F93B78232B0CD193
:10DB9800424B434A43481A600121FFF765FF337837
:10DBA80068F3000368F3410333703B782A2B65D18F
:10DBB800337803F0FE036FF3410333702B6843F4AB
:10DBC80000432B600F232370364B187803B0BDE851
:10DBD800F04F0BF04DB80AF08FFF054600282DD006
:10DBE80001213048FFF760FF3B78532B12D133787F
:10DBF800019A03F0FD0362F300033370DAF8003092
:10DC080043F40043CAF800300F232370254B1878DB
:10DC18000BF02EF83B78232B30D13378002203F019
:10DC2800FD036FF3000333701E4B1A70FAF79AF96D
:10DC38001E4A137843F00603137015E01C49FAF7DF
:10DC4800CDF83B78232B19D199F8003065F34103BF
:10DC580065F3000389F80030FAF784F998F8003082
:10DC680043F0060388F80030124A1378013BDBB210
:10DC78001370114A52F82320084B1A6003B0BDE80C
:10DC8800F08F00BFEE290020FC440208F2010020BA
:10DC980014230020201400201D45020858140020D9
:10DCA800E4F901087D1400203E450208B51400205F
:10DCB8005F450208A3140020A4140020A821002016
:10DCC8002DE9FF412C4D2D4C2B7843F001032B708F
:10DCD800217801F00401C9B211B92948FFF7E4FE1F
:10DCE800284E3378232B21D12378274F13F00408AB
:10DCF8000AD0224A6FF382031370244B20483B60FA
:10DD08000021FFF7B1FE11E0FAF72CF92B78204A31
:10DD180043F006032B701378013BDBB213701D4AE6
:10DD280052F823303B60164B83F800803378532B2E
:10DD38001FD12378052243F004032370104B1649A2
:10DD48001C78013CE4B204EB840000F5C840623062
:10DD580001F0BFFA00201149FAF740F8FF2300212B
:10DD680000930134162004220B460191029401F01D
:10DD780019FBBDE8FF8100BFB51400201423002063
:10DD88007D140020201400205814002000FA0108F7
:10DD9800A3140020A41400201CFA0108DB44020884
:10DDA8002DE9F041984B04469A7812F0010F00F0E3
:10DDB80017811B88002B40F01381944D95F8203073
:10DDC8000B2B40F2D780012C14D1914B1B7803F018
:10DDD8000203DBB2002B00F0C48095F820208B4BA7
:10DDE8000C2A03D1013283F82020FBE0142283F8A7
:10DDF8002020B6E0022C03D1142385F82030B0E0AF
:10DE0800844E337803F02002D2B28AB195F82020EC
:10DE18000C2A0DD1032C0BD07F4B804A03F1100143
:10DE280053F8040B8B4242F8040BF9D10D2395E00B
:10DE380003F01003DBB28BB195F820300D2B0DD118
:10DE4800032C0BD0764B754A03F1100153F8040BE1
:10DE58008B4242F8040BF9D10E237FE0F37813F0DC
:10DE6800010F0FD095F820200E2A0BD16D4B6B4A6D
:10DE780003F1100153F8040B8B4242F8040BF9D15B
:10DE88000F236BE003F00202D2B27AB195F820209A
:10DE98000F2A0BD1644B614A03F1100153F8040BAC
:10DEA8008B4242F8040BF9D1102357E003F0040227
:10DEB800D2B27AB195F82020102A0BD15B4B574A81
:10DEC80003F1100153F8040B8B4242F8040BF9D10B
:10DED800112343E003F00803DBB28BB195F820303F
:10DEE800112B0DD1032C0BD0514B4C4A03F11001CF
:10DEF80053F8040B8B4242F8040BF9D112232DE09E
:10DF08000BF0F6FBA0B14B4B1B788BB195F820308A
:10DF1800122B0DD1032C0BD0474B404A03F11001B3
:10DF280053F8040B8B4242F8040BF9D1132315E084
:10DF3800F37803F04003DBB29BB195F82030132B44
:10DF48000FD1032C0DD03D4B344A03F1100153F887
:10DF5800040B8B4242F8040BF9D1142385F82030C6
:10DF680078E095F820300133DBB2132B85F82030A8
:10DF78007FF629AF95F82060132E04D9234B00268D
:10DF880083F8206001E00136F6B206F10C07FFB213
:10DF980012E02B4831460FF0BBFA08B1032C04D12C
:10DFA800284B9B5D23B1032C02D185F820600FE03C
:10DFB8000136F6B2BE4203D00B2EEAD90C2E07D199
:10DFC800214B1E221A700C2385F82030BDE8F08101
:10DFD80095F820001149652246F63E33F9F73CFED4
:10DFE800012C37D1194B0D4A03F1100153F8040BDA
:10DFF8008B4242F8040BF9D1044B93F820300B2BD9
:10E008003CD9002012493EE0C4140020F20100204F
:10E018002C120020A8210020B04B0208CB140020AD
:10E02800D14B0208F24B0208134C0208344C020888
:10E03800554C0208ED240020764C0208B84C020822
:10E0480064120020541200207E1400209C9B0208B9
:10E058006E4B0208104BD87800F02000C0B220B1F7
:10E06800022C06D000200D490DE0032C01D10C49EB
:10E0780009E00C4B93F820300B2B02D800200A49FA
:10E0880001E00A490020F9F7A9FE10200146BDE881
:10E09800F041F9F753BE00BFA821002089420208C9
:10E0A8008F4B0208F20100202C4B0208974C020803
:10E0B80010B5F9F757FF084B1B7803F00403DBB2E0
:10E0C8002BB106490020BDE81040F9F787BE0220B1
:10E0D800BDE81040FFF764BE2C1200205E4902081C
:10E0E80070B5214B06461B78204CF3B9257819E00A
:10E0F8001F4829460FF00CFA78B123689D4202D9CF
:10E10800FF2E02D007E0FF2E02D19D4208D202E086
:10E1180036B91DB913B9256012E00EB9013500E012
:10E12800AD19EDB20B2DE3D90AE0013B20211148CE
:10E1380010222360F2F72EF900200F49F9F74EFE5E
:10E14800F9F7E4FD46F63E3320780C496522F9F7E5
:10E1580083FD084D216805F1100001310222F9F70D
:10E1680063FE2D23AB7470BD731400208C14002043
:10E178005E140020F201002006800208CB14002063
:10E18800F8B5534BF02253481A700378044613F03D
:10E198000E0518D1504A43F00203156000F8013B00
:10E1A8000FF052F92C464D4BE35C1BB14C4821460D
:10E1B8000FF098F901340C2CF5D14A4B1A7842F03B
:10E1C80001021A70F8BD13F00C0543D12E464448DD
:10E1D80029460FF09DF908B10136F6B201350C2D2C
:10E1E800F5D11EB9237843F0040331E000253E48F9
:10E1F8002946EFB20FF08CF968B1384BEB5C53B19C
:10E208003A4B01371F700020FFF76AFF237843F06D
:10E218000803237002E001350C2DE8D1344D3A2172
:10E228002846F2F735F938B1401BC0B2013028183A
:10E2380031460222F9F7F8FD2E4B1B78532B46D1B5
:10E248002A4B00201870FFF74BFF237843F0080390
:10E258002370F8BD6FF34103037003F00403DBB2CE
:10E26800244D23B100202449F9F7B8FD0DE02B789F
:10E27800552B01D1FF2002E0442B02D10120FFF7EA
:10E288002FFF13200D21F9F759FD2B78232B1ED1D1
:10E29800227802F00204D4B90E4902F0FB0264F3BA
:10E2A800C3020A700C4A1460F9F75CFE0D4B1A7829
:10E2B80042F006021A70114A1378013BDBB2137060
:10E2C8000F4A52F823200F4B1A60084B1C70F8BDF8
:10E2D800C11400205D1400208C140020EC190020CB
:10E2E8005E140020B51400202D12002073140020A5
:10E2F800F201002020140020878C0208A3140020BB
:10E30800A414002058140020024800210922F2F722
:10E3180041B800BF9114002070B50A46002405E0FA
:10E328001B19811A2A2501345D54E4B20E4D0F4B96
:10E33800295D09B19442F3D1801A001918182021D7
:10E34800121BF2F727F80A4B1E785EB1432E04D150
:10E358000CB1013CE4B200232B553046F9F7FAFD25
:10E3680000B12E5570BD00BF91140020F2010020AD
:10E378002014002038B5184C184DA07800F0100073
:10E38800C0B250B91649F9F729FDFFF7BDFF236858
:10E3980043F4801323600F232B702A782AB923684B
:10E3A800FF2062F31453236038BD0E48C5792DB998
:10E3B8001C200821FFF7B0FF284638BD23680A490A
:10E3C8006FF3145308222360F2F764FA00280CBF95
:10E3D8000120FF2038BD00BFA8210020C314002061
:10E3E800C149020891140020ADAC0208F0B5634D94
:10E3F80085B06E7806F01006F6B2002E3ED1604B5E
:10E408001A78604B013A53F822305F4A934204D19C
:10E418005E4B1A7842F0020207E002F11C018B42BF
:10E4280008D15A4B1A7842F00402022161F3C7025C
:10E438001A7019E03832934216D1FFF79BFF002873
:10E4480000F09A800128514C06D12378022243F02B
:10E45800010362F3C70306E030464D49F9F7BEFCF5
:10E46800237866F3C70323704A4B1A7842F00102F7
:10E478001A702B6843F480532B607DE0434E337849
:10E4880013F0F80406D04449002005B0BDE8F04078
:10E49800F9F7A4BC13F0070F4FD003F00202D7B26C
:10E4A80087B1214612200CF045FAFF230093432040
:10E4B8002146042223460194029400F073FF00943D
:10E4C800162031E003F00404E4B2A4B1394638461A
:10E4D8000CF030FA0BF0A8FC07F002FD0AF034FB50
:10E4E800FF2300934420394604223B4601970297B4
:10E4F80000F058FF1DE013F0010F1AD0012143F678
:10E50800FA400CF017FA2046F7F7BAF9234B4520E2
:10E518001C80FF2300932146042223460194029481
:10E5280000F040FF00941520214601222346F3F70E
:10E5380017FE00201A49F9F751FC337803F0FA0363
:10E548006FF341033370174B1B78232B14D12B68BF
:10E558006FF30C332B60F9F705FD0E4B1A7842F078
:10E5680006021A70064A1378013BDBB21370054A9B
:10E5780052F823200C4B1A6005B0F0BDA8210020EA
:10E58800A3140020A414002020FA010872270020F8
:10E59800E2490208B514002002900208381400204D
:10E5A800E18F020820140020581400201FB50446EB
:10E5B800F7F724FAA8B14B2001F06EFAFF23009375
:10E5C8000121FF3B0193392004220B4601340294B8
:10E5D80000F0E8FE064B01205A7842F004025A7017
:10E5E80004E0044B1888003818BF012004B010BD9F
:10E5F80004230020042A0020F0B51E4E0024337A9C
:10E608000546013385B00F4633721020214601229A
:10E6180023460094F3F7A4FD45B9FF230093019521
:10E6280002974F20294604222B4609E0012D09D1E3
:10E63800FF23009301940297502021460422234689
:10E6480000F0B0FE337A052B11D1FA3301210024F2
:10E65800009327200B4604220194029400F0A2FEA6
:10E66800044B1C7205B0BDE8F04001F0E7B905B0F5
:10E67800F0BD00BF801400202DE9F04F9D4B87B0FE
:10E688001A78804699461AB1012A40F0DB812AE0BF
:10E69800994B1A68994B9A4200F0D681F6F76CFEAE
:10E6A800974B5B7803F02003DBB223B901F0ECF958
:10E6B80008B907F015FC934B1A686FF310421A60FB
:10E6C800914B1878F9F746FC002800F0BD81FFF758
:10E6D8001BFE8E4B3C221A70F9F77AFA99F8003033
:10E6E800013389F80030894B1C787CB9884B08F1D4
:10E6F80001011A78204664F3C30264F304121A7005
:10E70800C9B2FFF779FF89F800409DE1814D404685
:10E7180007F006FCF9F706FB00207F49F9F75EFBD6
:10E728007E4F2B78AA46FB1813F8313C23B91B20DF
:10E738000621FFF7F1FD87E1754A0B21137804A83C
:10E74800C3F3C004C3F3001603F0F7036FF3041315
:10E758001370002389F80030062200F0C0FD2A78E3
:10E76800394604A8303AF1F73BFD074620B10027A7
:10E778004FF012093D4629E049F2DB4000F09EFDCA
:10E788000028F4D0664D2F72F6F74EFF0446002895
:10E7980040F05A81634A584B21461A60FF23009380
:10E7A8000190029004220820234600F0FBFD01227C
:10E7B80023460E2021460094F3F7D2FC5A4B1A78D0
:10E7C80042F004021A700123AB713DE1494606226A
:10E7D80004A800F084FD9AF8002004A84F49303AB4
:10E7E800F1F7FEFC002840F01E812846FFF7DEFE08
:10E7F800002840F02981DFF828B101218BF80800B2
:10E808002846F6F71FFF8146F6F70EFFDA4600287E
:10E8180040F0B28048464549F1F7C0FEB0B901F072
:10E828004BF8354B14B916B9414A23E036B1414A81
:10E838001A60414B1A786FF3410205E03F4A1A60AB
:10E848003D4B1A7866F341021A70D4E048463C49B9
:10E85800F1F7A4FE20B148463A49F1F79FFE58B9AE
:10E86800002C40F0F180002E40F0EE8001F024F8FA
:10E87800354A214B1A60BEE048463449F1F78EFE0E
:10E8880050B949F2D940012100F00EFD1D4A136824
:10E8980043F400531360E3E748462D49F1F77EFE41
:10E8A80038B9002C40F0D080002E40F0CD80294AA5
:10E8B800DFE748462849F1F771FE38B9002C40F0E7
:10E8C800C380002E40F0C080244AD2E7484624493D
:10E8D800F1F764FE002840F08E8000F0EDFF002C78
:10E8E80040D0164A044B1A60134B1A786FF3410252
:10E8F800A9E000BF571400205814002074FA01083A
:10E9080012230020A821002020140020C314002076
:10E91800901400203F14002068420208911400203F
:10E928008014002090FA0108FD170020D7AD0208D6
:10E93800C0FC010848FE0108B514002064FE010867
:10E94800A9AD020894AF020880FE0108CDAD020807
:10E95800CFAD0208B8FE010866AF02080CFF010837
:10E96800D1AD0208002E6FD0394A3A4B1A603A4BA3
:10E978001A7864F3410266E048463849F1F70EFE1A
:10E98800064620B900F098FF002C5DD01BE04846F1
:10E998003349F1F703FE002856D048463149F1F7CC
:10E9A800FDFD38B9002C4FD12F4A2A4B8BF8075060
:10E9B8001A6049E048462D49F1F7F0FD064650B97E
:10E9C800A4B100F079FF2A4A224B1A60224B1A7828
:10E9D80066F3410237E048462649F1F7DFFD20B1EA
:10E9E80048462549F1F7DAFD00B96CBB234A194BB3
:10E9F8001A6000F061FF07F56A506E308AF8075018
:10EA080000F05CFC8AF800009AF8070000F5D44092
:10EA1800123000F053FC8AF801001948F6F748FF55
:10EA2800202D11D107E00135EDB20137202D09F174
:10EA380007097FF4CBAE08F101010020C9B2FFF746
:10EA4800DBFD01E000221A7007B0BDE8F08F00BFBF
:10EA580048FE010858140020B5140020D1AD020862
:10EA6800CFAD020866AF02080CFF0108D7AD020857
:10EA780064FE0108A9AD0208CDAD020828FF01080F
:10EA88008014002038B51C491C4A0B6810789C7B00
:10EA98008442144603D99D8915F0200F18D09A890D
:10EAA80012F0800F01D105E01C3B9A8912F0400F4B
:10EAB800FAD000E01C330B60002323700B689B899D
:10EAC80013F0200F06D00E4BDA790C4B1A7001E0C8
:10EAD800013010700B4A002313700B4A13700B4A55
:10EAE800136843F480731360F9F772F8084B1A78C7
:10EAF80042F006021A7038BD581400207314002022
:10EB0800801400203B14002035140020A821002088
:10EB1800B514002010B51D4B1D4A1978184639B197
:10EB28001468A48914F0200F02D1013919701AE071
:10EB38001368998911F0400F01D106E01C339989B7
:10EB480011F0800FFAD0136002E011491C3B0B60F2
:10EB580013689A7B02709B8913F0200F03D00D4B2A
:10EB6800DA790A4B1A700C4A002313700B4A137097
:10EB78000B4A136843F480731360F9F729F8094BBB
:10EB88001A7842F006021A7010BD00BF73140020F4
:10EB980058140020801400203B1400203514002055
:10EBA800A8210020B5140020084B094A1B6893428D
:10EBB80003D002F57C72934205D1064B18780038D1
:10EBC80018BF012070470020704700BF581400206C
:10EBD80074FA01082B120020074B084A1B6893425D
:10EBE80002D03832934205D1054B1878003818BF47
:10EBF8000120704700207047581400200CFF0108BE
:10EC08002B1200202DE9F04F8B4B8C4D1970A0F181
:10EC18001103DBB2012B87B00E46287020D81228CA
:10EC280004D1874B1A8842F480521A80854B0024FD
:10EC38005A78214642F010025A70FF2302220093AC
:10EC48003D20FE3B0194029400F0ACFB4D2000F007
:10EC580023FF12202021012223460094F3F780FA93
:10EC68002B78522B0DD1F3F7BDFF28B9F3F7AEFF80
:10EC780010B9F3F7CFFF20B1734B1A7842F00802AE
:10EC88001A70724B724C1B78002B2DD12168714A77
:10EC9800914229D0704A23601370704A70481178E5
:10ECA800037063F3C30163F3000163F30711117089
:10ECB8006C4A117863F3010111706B4A117863F3A0
:10ECC800C5011170694A1370694A117863F34101EB
:10ECD80063F3000163F382011170664A116863F3FC
:10ECE8000C311160644A13702368002B40F057817F
:10ECF800604F7B7803F02003DBB273B15F4B93F86E
:10ED08000080B8F1000F08D149F2D940414600F01F
:10ED1800CBFA3B6868F34D333B60594B187810F0D9
:10ED28001E0002D00020574907E0574B93F8038094
:10ED38009946B8F1000F05D0544907B0BDE8F04F27
:10ED4800F9F74CB8524F97F801B0BA46BBF1000F2B
:10ED58002BD0BBF1070F14D9F8F7D8FF4D49B87875
:10ED6800652246F63E43F8F777FF3878072310F018
:10ED780003007B700EBF484940464849F9F72EF812
:10ED88000CE0BBF1020F09D8454B5B7823B1F8F7CB
:10ED9800BDFF87F8018069E202237B7010200146DD
:10EDA80007B0BDE8F04FF8F7C9BF3E4FBB795BB17C
:10EDB80087F806B000F0DAFB8E20594601225B4640
:10EDC800CDF800B0F3F7CCF90020F3F7E7FF234ABA
:10EDD80021491378344843F00603137000230B705D
:10EDE800324923600B70324989F8003003701233BE
:10EDF80003FB061C9CF802C093461CF0100F8846C3
:10EE080004D130460593FFF737FC059B03FB0683C7
:10EE18005B7813F0100F04D02A78133AD2B2032A81
:10EE28004AD913F0200F7DD02B78442B44D041D8F9
:10EE3800232B41D02A2B3EE07614002020140020FA
:10EE48003C130020042300204C120020C114002091
:10EE580058140020C8F90108A3140020B514002094
:10EE68007D1400203C140020781400207F1400201A
:10EE780090140020A8210020C01400202B1200208C
:10EE8800ED290020CB4202081F0E0020B9690208B4
:10EE98007A140020CB140020D3430208B24302089E
:10EEA800C41400208014002077140020731400205C
:10EEB80055220020552B35D17A4B1B78002B31D1A8
:10EEC800794B93F80080B8F1000F2BD143F6DB2083
:10EED80000F0F4F9012825D11F23FB7189F80000FF
:10EEE80043F60D3000F0EAF93870F87900F5D440AF
:10EEF800123000F0E3F978706C48F6F7D9FC9BF80B
:10EF08000030304668F341038BF8003007F008F80A
:10EF1800F9F728F8664B67482360674BC3F8008009
:10EF28002B7803702B78432B0AD15F4B1B783BB9A6
:10EF3800013389F80030614B3046236006F0F0FF5A
:10EF480028781738C3B2072B00F290815C4908F083
:10EF580079FB9AF800105B4B60F301018AF8001006
:10EF680001F00301022900F081810122032041B14F
:10EF7800009001929B7868309B180293002103321D
:10EF880006E0009001929B786C20013302930422E2
:10EF98000B4600F007FAFF238AF8013066E1474A7A
:10EFA800934253D12878A0F14303DAB2122A25D824
:10EFB800454A5BB29A4021D5432840F05781394BE6
:10EFC8001B78002B40F0528100F080FC3F4B40B191
:10EFD8001A7803201109013191FBF0F000EB400091
:10EFE80007E01A7807201109013191FBF0F0C400FD
:10EFF800201A091A61F307121A7037E1F8F7AAFF05
:10F00800002823D0314F3A7812F0F00308D163F387
:10F0180007123A7023602E4B1A7842F008020EE06D
:10F02800102B13D100F052FC80B13B786FF307131B
:10F038003B7000232360264B1A7842F010023046BA
:10F048001A7007B0BDE8F04FFFF716BB214B1E2121
:10F058001A781E4E61F346021A70337813F0010FC6
:10F06800134B3DD022689A420CD0A3F5AC639A4268
:10F0780008D0FFF799FD28B9FFF7AEFD10B9AA30FF
:10F08800F3F78CFE2268144B9A4202D10020F3F762
:10F0980085FE2B78522B40F0AE80104B53221A700D
:10F0A800A9E000BF2B120020571400208014002074
:10F0B80028FF010877140020A414002074FA01081E
:10F0C8007C1400207A140020002000C0B514002011
:10F0D800901400203215002060FF01082014002041
:10F0E80022689A420CD0A3F5AC639A4208D0FFF785
:10F0F8005BFD28B9FFF770FD10B9AA30F3F74EFE93
:10F108002B78552B16D1FFF705FD3378594F43F06F
:10F1180006033370584B9B7803F00203DBB24BB104
:10F12800F8F7F4FD23681868FCF752F83B786FF39A
:10F1380041033B702B78442B16D1FFF7A3FC33789F
:10F148004C4F43F0060333704B4B9B7803F002039C
:10F15800DBB24BB1F8F7DAFD23681868FCF738F82A
:10F168003B786FF341033B702B78522B09D13378EE
:10F17800002243F001033370404B1A70404B453274
:10F188001A70404B00271F702B78232B33D13E4B2E
:10F198001F703E4B1F70F8F7B9FD33783C4943F0B8
:10F1A800060333700B78334AFBB13A4A013B1770B8
:10F1B800394ADBB20B7052F82330384A23609B6817
:10F1C800934202D107F0F8FC15E002F59A718B42E0
:10F1D80004D10120014605F027FB0CE002F5D272AC
:10F1E800934208D12E4B1F7005E0117863F3071185
:10F1F800117023603AE02B4B1B7813B10020F3F712
:10F20800CDFD23681F7B17F00F0702D1FDF784F9A6
:10F218001BE0012F02D1FAF739FC16E0022F02D1C8
:10F22800FAF762FF11E0082F05D84FF09C53BB4056
:10F2380001D5FBF727FC042F03D123689B69984766
:10F2480003E0052F01D1FBF7E5F9337803F002035A
:10F25800DBB21BB123681868FBF7BAFF33786FF38A
:10F26800410333702B780BB1064A137007B0BDE821
:10F27800F08F00BFB5140020C41400207D140020B6
:10F28800201400203D1400207F140020C01400200A
:10F29800A314002073140020A41400207CFF01088C
:10F2A800611400201F0E002007B502AB03F8011DF2
:10F2B80019460122002303F0C3FF0EBD07B5002342
:10F2C80002A901F8013D012204F022F89DF8070087
:10F2D8000EBD08B5002303F0B3FF002008BD0346A8
:10F2E80010B508461446194604F012F8E0B210BDED
:10F2F80010B50346002484540846194604F008F85B
:10F30800204610BD37B50546002400E0144601220A
:10F3180060190DF1070103F0FBFF9DF80730621C2F
:10F32800203BDBB25A2BF1D920463EBDF8B500246C
:10F338001949022211F8340001EBC40140000431DC
:10F3480000F571500134FFF7C4FF292CF0D143F6C2
:10F35800B630124904220025FFF7BBFF48F6D8272C
:10F368002C4615E007EB460004EB440100B259189F
:10F378000222FFF7AEFF0136F6B2094B5A1992780E
:10F38800B242EFD8013480370335142CBFB201D014
:10F398000026F2E7F8BD00BF04250208ABAD02085D
:10F3A8004C2602082DE9F347044615468A460222F0
:10F3B80043F6F8410DF106001E46BDF930909DF860
:10F3C80028809DF82C70FFF78AFF2F4B2F499A78D9
:10F3D800BDF906008A705A7800EBC000CA701A7925
:10F3E80000F572500A715A797A304A719A791B7805
:10F3F80045EAC6158A710C7081F80190CB710D72BF
:10F4080000B20922FFF765FF1EB1214B1A880132AD
:10F418001A80BDF8063001339BB2B3F57A7FADF898
:10F42800063002D30023ADF8063002220DF10601A2
:10F4380043F6F840FFF74DFFBDF80600154B18805E
:10F4480000B200EBC00000F5725000F17A0582307E
:10F4580000B2FFF733FF10F0800F03D00C4B1A886F
:10F46800013A1A8028B20021FFF71EFF0A4B03F861
:10F47800148003EB44046770BAF1000F02D0012036
:10F48800F6F7FEF9BDE8FC87782700209A140020DB
:10F4980038140020A01D0020591B00202DE9F74337
:10F4A800314B1D78303DEDB2C5F10606F6B23EB3DC
:10F4B80005F11207202413E008F101080FFA89F07A
:10F4C80000215FFA88F8FFF7EFFE09F10109B0455E
:10F4D8001FFA89F9F0D1013C0737E4B2BFB21CB179
:10F4E800B9464FF00008E7E70B35013428B2002190
:10F4F800E4B20135FFF7D8FEB442ADB2F5D131E040
:10F50800122425B2684629460622FFF7E8FE9DF830
:10F51800003043B19DF805302BB99DF803308DF8C4
:10F5280004308DF805300734062228466946A4B20F
:10F53800FFF7CFFEF22CE4D168460B210622FFF735
:10F54800CEFE9DF8003043B19DF805302BB99DF8EB
:10F5580003308DF804308DF805300B2069460622FB
:10F56800FFF7B7FEBDE8FE833F14002010B507F093
:10F5780023FB09F091FB04F0A7FB04F0CFFAF3F7A3
:10F5880035FE9C48F6F7AEF943F6D120FFF796FE14
:10F59800994B9A4C187043F6D020FFF78FFE984B82
:10F5A800187043F6DC20FFF789FE964B187043F677
:10F5B800E130FFF783FE944B187043F6E230FFF713
:10F5C8007DFE924B187043F6DA20FFF777FE904BDA
:10F5D800187043F6D920FFF771FE8E4B187043F66A
:10F5E800CF20FFF76BFE8C4B187043F6CC20FFF74B
:10F5F80065FE8A4B187043F6D220FFF75FFE884BF2
:10F60800187043F6DF20FFF759FE864B187043F653
:10F61800E820FFF753FE844B187043F6DD20FFF710
:10F628004DFE237801280CBF43F001036FF300035C
:10F63800237043F6E020FFF741FE237801280CBF32
:10F6480043F080036FF3C713237043F6E720FFF7F7
:10F6580035FE764B01281A6843F6EA200CBF42F0C3
:10F6680000526FF35D721A60FFF728FE6378012875
:10F678000CBF43F001036FF3000363706C4843F65B
:10F688006E210822FFF72BFE6A4B00241C705C7069
:10F698006748235C312B03D1103021460DF022FF3F
:10F6A8000134082CF4D1224643F6F6116048FFF7DE
:10F6B80016FE224643F63A215F48FFF710FE47F24E
:10F6C800740104225D48FFF70AFE47F2780104221C
:10F6D8005B48FFF704FE0AF023FEF6F7D3FB43F678
:10F6E800E120FFF7EBFD574C237860F3000323700C
:10F6F80043F6E220FFF7E2FD237860F3410323702D
:10F7080043F6E420FFF7DAFD237860F3C3032370A0
:10F7180043F6E620FFF7D2FD237860F34513237004
:10F7280043F6E920FFF7CAFD237860F386132370B8
:10F7380043F6E520FFF7C2FD237860F30413237036
:10F7480043F6EB20FFF7BAFD237860F3C713237065
:10F7580043F6E320FFF7B2FD237860F382032370BA
:10F768003948FFF7ABFD394B18703948FFF7A6FD4C
:10F77800384B18703848FFF7A1FD384B18703848D7
:10F78800FFF79CFD374B18703748FFF797FD374B4D
:10F7980018703748FFF792FD364B18703648FFF758
:10F7A8008DFD364B18703648FFF788FD354B1870BD
:10F7B8003548FFF783FD354B1870FFF76FFE344867
:10F7C800FFF77CFD334B18703348FFF777FD334B59
:10F7D80018703348FFF772FD324B18703248FFF744
:10F7E8006DFD324B18703248FFF768FD314B1870C9
:10F7F80010BD00BF531400201A0E0020321500203F
:10F80800190E00201C0E0020141200200A100020DF
:10F81800062A002000000020341300203E14002097
:10F828001B0E00201B220020EA210020A821002016
:10F83800A1220020B1220020A9220020B621002008
:10F84800CC2100202D130020CE8AFFFFED240020BC
:10F85800CF8AFFFF1A240020D08AFFFFEA24002065
:10F86800D18AFFFFEB240020D28AFFFF1C2400204E
:10F87800D48AFFFF93230020D58AFFFFEC150020D0
:10F88800DC94FFFF57130020DA94FFFF3F14002099
:10F8980014A2FFFF932100208FA1FFFF331C00203B
:10F8A80091A1FFFF9E1D002090A1FFFF991D002040
:10F8B800858AFFFF38180020034B1E211A7861F350
:10F8C80046021A70704700BF32150020024B1878A4
:10F8D80000F00100704700BF32150020014B187876
:10F8E800C00970473215002008B5FFF7F7FF38B98F
:10F8F800044B1B7813F07E0F0CBF0020012008BDBD
:10F90800012008BD32150020F8B546F6AA74204635
:10F91800FFF7D4FC2D2803DD20462D21FFF7C4FC7A
:10F92800A4F55856123E3046FFF7C8FC414FC0B206
:10F9380007EBC0000579C5F30015A5B90DE03D4BEF
:10F948003D4953F83500F0F729FE20B930462946DD
:10F95800FFF7AAFC07E00135EDB207EBC5031B79F9
:10F9680013F0080FEBD0013446F6B6739C42CED1A3
:10F9780043F6C4242046FFF7A1FC2D2803DD2046CA
:10F988002D21FFF791FC013443F6C8239C42F1D1A5
:10F99800012143F6E120FFF787FC012143F6E2202D
:10F9A800FFF782FC012143F6E420FFF77DFC0121EB
:10F9B80043F6E620FFF778FC012143F6E920FFF73C
:10F9C80073FC012143F6E520FFF76EFC012143F6A5
:10F9D800E320FFF769FC012143F6EB20FFF764FC05
:10F9E800002143F6E020FFF75FFC002143F6EA2000
:10F9F800FFF75AFC002143F6EC20FFF755FC0121E4
:10FA080043F6DC20FFF750FC002149F2DB40FFF70A
:10FA18004BFC48F644200121FFF746FC47F252040C
:10FA28002046FF21FFF740FC013447F25A039C426D
:10FA3800F6D1F8BD08040020529A020810B506F065
:10FA48002FFA09F0EDF8074B4FF416721A800121CE
:10FA580047F26200FFF728FC4C20BDE8104000F098
:10FA68001BB800BF042A002010B506F039FA09F0C7
:10FA78006BF8044B002147F262001980BDE8104082
:10FA8800FFF712BC042A0020024B1888003818BF60
:10FA980001207047042A0020542873B5044663D80F
:10FAA8003D4BDB7803F02003DBB2002B72D10B282F
:10FAB80001D80EF03BFB394D35F81460002E69D1A2
:10FAC800E10001F5D8416846B2310822FFF707FC8A
:10FAD800334821460DF01CFD50B1F3B2072B07D077
:10FAE8000B2C05D80122B240D243D2B22D4B27E0CD
:10FAF8001DF806300122542B08D0562B03D0532B67
:10FB0800284B1AD100E0284BB24007E0B240254B01
:10FB1800D2B2195D42EA01011955234B195D0A4316
:10FB28001A55FFF7D3FE98B1204B1B7883B10B2CE5
:10FB38000ED81E3325F814300AE0B240D243D2B2B0
:10FB4800195D02EA01011955174B195D0A401A554A
:10FB58000136082EBCD1134B1A5D134B1B5D1343A2
:10FB680018D125F8143015E0C10001F5D8416846D0
:10FB7800B2310822FFF7B3FB00231DF803202D2A1A
:10FB880005D001219940074A105D01431155013301
:10FB9800082BF2D17CBD00BFA8210020361500201B
:10FBA800361A00204C170020B116002054130020EC
:10FBB8001FB500F017FD10B900F028FD48B100216D
:10FBC800FF2300930B2004220B4601910291FFF7BB
:10FBD800E9FBAD220023D9B24D2909D0012A07D962
:10FBE8000D48002119540D4819540D4820F81310D8
:10FBF80001330132552BD2B2EDD1074B002183F8E6
:10FC08005510084B08481970084B0822197005B0A0
:10FC18005DF804EBF0F7BEBB4C170020B1160020CE
:10FC2800361500204D1600202C1600203415002013
:10FC380059B1064B0C2202FB0030437AC918837A6B
:10FC4800417208300BB93C3383707047581A002052
:10FC5800032811D9094B1B5C022B0DD10438C0B203
:10FC6800C308012100F0070011FA00F0044A01332B
:10FC7800D15C41EA0000D054704700BFEC19002065
:10FC8800FF210020044B0C2202FB00330C3A5A726D
:10FC98009A72FFF7DDBF00BF581A002010B504465E
:10FCA800FFF7F0FF034B0C2202FB0434FF236372BF
:10FCB80010BD00BF581A002070B5104D0024104820
:10FCC8002146E6B20DF024FC90B96B7A83B10D4A57
:10FCD800A318A25C1B7E022A0AD0413BDAB2122A80
:10FCE80006D8094A5BB29A4002D53046FFF7CAFFE8
:10FCF80001340C350C2CE2D170BD00BF581A00201D
:10FD08002E130020EC1900200020008810B50A4BA3
:10FD18000C2203EBD00393F84810084B02FB003386
:10FD28001C7A3CB900F0070051FA00F010F0010FFE
:10FD380018BF1A7210BD00BFEC190020581A002015
:10FD4800044B0C2202FB00331A7AFF2A01D1FF3A36
:10FD58001A727047581A0020104B1B7813F0010FC5
:10FD680002D10F4B187818B10E4B03F190020CE03A
:10FD78000C4B03F19002197A0C330139C9B2FD29F1
:10FD880098BF01209342F6D17047197A09B1FF2133
:10FD980019720C339342F8D1002070473C130020AD
:10FDA80054130020581A002030B504461048007833
:10FDB80000F00200C0B2C8B10C2060430D4D285CB1
:10FDC800904201D1994207D0984201D1914203D083
:10FDD800052A0BD1052B09D10C2303FB0455064832
:10FDE80021462B72BDE830400DF087BB30BD00BF07
:10FDF8005D140020581A00205E1400201FB5044628
:10FE0800214614480DF084FB002821D0012202234A
:10FE180000210093A31802935C200B460192FFF780
:10FE2800C1FA21460B480DF068FB21460A480DF03F
:10FE380064FB214609480DF055FB074BE40804F51F
:10FE4800CA40195DA83004B0BDE81040FFF72CBACD
:10FE580004B010BD461200204F1200202E130020BF
:10FE68002DE9F7438E480DF0EFFADFF858828D4EF2
:10FE78000024E5B2284603F0CDFF18F8019F074695
:10FE880018F80C3C13B1022B3ED10FE02846FFF7BF
:10FE9800F9FE214684480DF030FB214683480DF0D9
:10FEA8002CFB214682480DF028FBC9E0284649462C
:10FEB800F5F76EF810B12846FFF7EEFD737AFF2BC1
:10FEC80001D1FF3B7372737A4B4501D2F37A9BB130
:10FED800734821460DF006FBF37A002B40F0B08002
:10FEE800204604F0BDFA052128460A460B46FFF7CE
:10FEF8005BFF2846FFF7C6FEF37A002B40F0A08090
:10FF08002846FFF77BFF9BE090B92846FFF7BAFE2B
:10FF1800214663480DF0E6FA28463946F3F758FCBF
:10FF2800002800F086803378002B00F082803AE0C9
:10FF3800022814D15A4821460DF0D4FA3378012BFF
:10FF480001D0737A1BB928460121FFF771FE2846B4
:10FF58004946F5F71DF800286BD0284626E0032807
:10FF68000FD12846FFF78EFE21464D480DF0BAFA0C
:10FF780028460121F3F72CFC00285AD03378032BAC
:10FF880010E0042815D12846FFF77CFE2146444896
:10FF98000DF0A8FA28460221F3F71AFC002848D0E9
:10FFA8003378042B45D0052B43D04520FFF774FD4B
:10FFB8003FE001283DD1737A4B4502D32846FFF72D
:10FFC80061FE214638480DF098FA214637480DF071
:10FFD80094FA214636480DF090FA2846FFF7B0FE0D
:10FFE8003378012B25D0052B23D02846FFF706FFB1
:08FFF80033780BB1032B07D194
:020000040801F1
:100000002E4821460DF088FAB8B12046012108E0BB
:10001000042B09D12A4821460DF07EFA68B120460A
:100020000221F2F797FA08E0264821460DF074FA0B
:1000300018B120460021F2F7BFF9284639460122BF
:100040000223FFF7B5FE3770214617480DF064FA1A
:10005000013401462846F5F7E1FB0C360C2C7FF401
:100060000CAF194D09F014FF2C68D4B943F6D32016
:10007000FFF728F9C6B29EB14320FFF711FD2146D4
:100080000122234608200094F2F76EF801230E2087
:10009000214622460094F2F767F84FF461635E430D
:1000A0002E60BDE8FE8300BF4A170020581A0020CA
:1000B000E0190020E2190020E41900202D12002090
:1000C0005213002040130020D0170020F719002001
:1000D000324AF8B59042054601D000231FE0304B6C
:1000E0001C78005D002808BF002401E00134E4B260
:1000F0008C4207D2105D0028F8D02A4830F814004E
:100100000028F3D18C4201D1002242E02649087830
:1001100008B9125D0A701C700B780EE00133DCB276
:100120008C4207D2EA5C002AF8D01E4A32F813202B
:10013000002AF3D18C422DD02B5D002613F0010F45
:1001400005D10136F6B2082E01D05B08F6E7174F4D
:1001500000213E702122164806EB0616F0F71EF924
:1001600006F51671124801312022FFF7BCF83878E5
:1001700000F046F978B93B78012212FA03F3295DC1
:1001800021EA03032B553978074B8A40197821EA75
:1001900002021A70FF242046F8BD00BFB1160020ED
:1001A000230E0020361500203415002051160020A3
:1001B000F215002070B50E46C11EC9B201230024FD
:1001C00007E002FB03440A2253430138A4B2C0B241
:1001D000DBB230B1325C303AD5B2092D01D8884259
:1001E000EFD1451C202106221648F0F7D7F8092C3C
:1001F000EDB204D9632C8CBF0023012309E0022354
:1002000007E011490135C918013381F8A320DBB299
:10021000EDB2052B09D8725DA2F13001C9B20929EE
:10022000EFD92C2AEDD02E2AEBD046F60920FFF785
:1002300049F8844204DA5520BDE87040FFF730BC2D
:1002400070BD00BFE318002040180020F0B587B053
:100250000446F0F7F3FA47F26301C5B2102201A891
:10026000FFF741F89DF804300BB1202B03D1234B4D
:100270001E78022E08D9204601A9F0F717FD07467F
:10028000002838D001A80BE01D4B06EB0616F61827
:1002900020463146F0F70AFD074600282BD03046AD
:1002A000F0F7CCFA3F1837B33F1B1DE0E35D2C2B72
:1002B00001D02E2B17D1E31913F8012C303AD2B20A
:1002C000092A10D85B78303BDBB2092B0BD80D4BD9
:1002D0001B7803F00803DBB263B1013FF8B221469B
:1002E000FFF768FF06E00137FFB26B1E9F42DDDBC0
:1002F000002700E00127384607B0F0BD410E00207E
:10030000C04102084018002008B50449F0F74AF936
:10031000D0F1010038BF002008BD00BFB517002094
:10032000044A00231370044A1370044A1370044AE9
:1003300013707047F1240020E9170020E81700200F
:100340000617002038B51C4B1C4A19781C4B19B1F4
:1003500000201870107038BD12789AB9194A1078B8
:1003600070B1194A117801F04004E4B244B91C7824
:10037000844205D141F040011E2060F30501117057
:1003800000221A701C7894B10F4B1D7805F04005BF
:10039000EDB22DB943F6D520FEF794FF844208D183
:1003A0000A4B01201A7860F301021A7038BD20460A
:1003B00038BD284638BD00BFE917002006170020C9
:1003C000F1240020EC150020EC2400201E24002045
:1003D00010B5F7F79FFA084B00211A68074822F07A
:1003E00002026FF382021A601122EFF7D7FFBDE815
:1003F000104002F0D5BD00BFA8210020A3170020A7
:10040000F8B5344D07462B78A3F13002D2B2092A51
:100410000CD92B2B0AD0002404E02E4B20221A5595
:100420000134E4B22B5D202B02D106E0002404E06D
:10043000002BF2D101E00134E4B22E5D202EFAD07F
:10044000254800211122EFF7A9FF002E3DD0A6F18B
:100450003003DBB2092B02D8204A00200DE02B2EFE
:10046000FAD00020F8BD013002F8013FC0B22023CD
:100470002B5501341028E4B20FD02B5D33B1A3F11A
:100480003001C9B20929EED92B2BECD028B9F8BD1F
:10049000104B20221A550134E4B22B5D202B04D0DE
:1004A000002BF5D101E00134E4B22B5D202BFAD012
:1004B0000B4C0023072F237009D807F566505830DE
:1004C000FEF700FF20700120F8BD3046F8BD012086
:1004D000F8BD00BFF2150020A3170020A2170020CE
:1004E000E015002038B540F2592500240C48294673
:1004F0002022FEF701FF2046FFF782FF40B10948A6
:10050000FFF702FF20B1012010FA04F4E0B238BD79
:100510000134E4B21135082CE8D1002038BD00BF09
:10052000F2150020A317002070B52A4B2A4C1B7827
:1005300023B12A4B00201870207070BD2378ABB90E
:10054000264D2B78012B00D100BF013BDBB2012BE4
:100550000AD802F01DFD01462148F0F711F9FFF716
:10056000C1FF08B107F03CF800232B701D4B5878F1
:1005700000F00200C0B200282AD01A6843F6D52045
:100580006FF349221A60FEF79DFE144DC6B22B7818
:100590000BB902F0DDFC06239EB123702B780133EA
:1005A000DBB2B3422B7012D10F4B1A786FF30102FA
:1005B0001A7002F0EDFC01460948F0F7E1F801205D
:1005C00070BD23702B78304601332B7070BD002036
:1005D00070BD00BFF1240020E8170020E9170020BB
:1005E000B51700200C1800201E2400200023074A05
:1005F000184632F8021F11B90549595C0843013306
:10060000572BF6D1003818BF012070473415002051
:100610004C1700200023074A184632F8021F11B970
:100620000549595C08430133552BF6D1003818BFF2
:100630000120704734150020B116002038B50C4653
:100640001546F0F7FBF8C0B207E0054B1A181B5D22
:100650001219013C02F8013CE4B2AC42F5D838BDB5
:1006600036280020F8B506460C46084617460021F5
:1006700010221D46EFF792FE3278174B002013F838
:10068000011F914206D12146102246F6A243F7F7F8
:10069000E7FA12E001300428F1D1002331211A4693
:1006A0003078184110F0010F02D0A1540132D2B2BB
:1006B00001330131042BC9B2F2D139462A46204612
:1006C000FFF7BCFF06460548214640193246EFF7C2
:1006D000BDFD3046F8BD00BF521400203628002072
:1006E00030B50378A121594301F5387185B0013146
:1006F000A0221248FEF700FE1048F0F79FF80024F1
:10070000C5B217E00D4B1B5D242B01D10C4806E050
:10071000262B01D10B4802E0402B09D10A482A467A
:1007200023466946FFF79EFF4519EDB2041900E024
:100730000134E4B2AC42E5D305B030BD3628002028
:1007400038130020521200205112002070B5234AA5
:1007500003780546D3181B7E542B05D12048214928
:10076000F0F70EF8002405E0462B1D480CBF1E498B
:100770001E49F5E72878800000F5D6403E30201865
:10078000FEF7A0FDC6B246B31548F0F757F8C0B261
:100790009F281BD8013EF6B21D2E114B4FEA0611C1
:1007A00008D8891901F514411818EE311122FEF705
:1007B0009AFD0BE00E4A89198918181801F11003E7
:1007C00051F8042B994240F8042BF9D10448094907
:1007D0000134EFF73DFE042CCCD170BDEC190020A4
:1007E00036280020627B0208837B0208417B0208D6
:1007F000BF990208CBAD020838B52C4D2B782C469A
:10080000012B16D002D3022B4BD138E057212848B8
:10081000FFF75EFC274BFF28187045D02648274974
:10082000EFF7AEFF264B1A78264B1A702B78013360
:100830002B70214801F096FB002836D01D48037824
:100840000B2B02D8FFF782FF10E0A3F15202D2B2C5
:10085000022A02D8FFF744FF08E0A121594301F51D
:10086000387119480131A022FEF746FD1648174994
:10087000EFF7EEFD237800200133237038BD01F03F
:1008800091FB90B10F4901200978002310FA01F182
:100890002B70084B064A1B78D45C24EA0101D15422
:1008A00038BD0020287038BD012038BD240E00203E
:1008B0004C170020AF1600203C160020A317002084
:1008C000511600204E16002036280020D3AD020815
:1008D00008B502F083FA18B9074B05225A7008BD13
:1008E000F6F7E6FF232804D1034B07225A7023387A
:1008F00008BD012008BD00BF240E002038B501242A
:10090000844000210A480B22EFF748FDE4B200259D
:10091000084BEB5C1C4207D0074B33F815301BB972
:10092000034829460CF0E2FD0135552DF0D138BDC4
:10093000E1150020B11600203615002070B5012504
:1009400085400024EDB20A4821460CF0E5FD20B1B7
:10095000084BE25C22EA0502E2540134552CF2D144
:10096000034800210B22BDE87040EFF717BD00BF20
:10097000E1150020B116002010B50B4A137813F0D2
:1009800001000FD0094903F0FE030978084800244C
:1009900013F0040F4454137003D0FFF70DF9012036
:1009A00010BD012010BD00BF46170020EE1500202D
:1009B0002C16002070B586B0F6F77AFF002800F0FC
:1009C0009A804E4B4E491A7888540132D2B2072A87
:1009D0001A7001D907221A704A4E1A783378303BC0
:1009E0009A42C0F28580454B00221A7043F6E4100B
:1009F000FEF768FCC4B214B91224002509E0FFF721
:100A000071FD10EA0401F7D108223D48EFF7C6FC5A
:100A100070E00021072204A8EFF7C0FC062221465F
:100A200004A8FEF760FC327804A8303A3449EFF7A6
:100A300035FF10F0FF0F38D12846FDF7BBFD01460A
:100A4000002857D104A80722EFF7A8FC2846F4F79E
:100A5000B9FE20B92846F4F7CBFE00284AD02A4C2C
:100A6000002108222648EFF799FC0021FF2325707A
:100A70000422009301350B461C2001910295FEF7DC
:100A800095FC2078214D00F56A506E30FEF71AFC77
:100A90002870207800F5D4401230FEF713FC6870FF
:100AA0002846F4F709FF022025E00135EDB20734AE
:100AB000202DAED10021072204A8EFF76FFC0622FB
:100AC00040F2522104A8FEF70EFC0E4B0C491A7896
:100AD00004A8303AEFF7E2FE002104460822084855
:100AE000EFF75CFC14F0FF0F14BF0120052002E0BB
:100AF000032000E0012006B070BD00BFD517002024
:100B0000341600203F140020181600208014002006
:100B1000044B054A1B784FF4147101FB032318188A
:100B20000DF070BA3E140020A0A90208024800216E
:100B30004A22EFF733BC00BF6416002010B504460C
:100B40000548EFF77BFE80B2492801D9013880B211
:100B5000014B1C5410BD00BF641600202DE9F0416C
:100B6000FFF7E4FFA92646F6423500241748214640
:100B70000CF0D2FCD8B1E3B20B2B15D8144BE31810
:100B80001B7E542B01D1FB2000E02520FFF7D6FF70
:100B90002F1F3846FEF796FBC0B240B10137FFF772
:100BA000CDFFAF42F5D102E03046FFF7C7FF013479
:100BB00001360435552CF6B2D8D1FC20FFF7BEFF24
:100BC0000448BDE8F0410DF01DBA00BFE11500205A
:100BD000EC19002064160020F0B5734C85B06378E2
:100BE000072B00F27881DFE813F008003700570088
:100BF0008500C70007013001690155216B48FFF7E7
:100C000067FA6B4BFF28187000F06A8169496A48DF
:100C1000EFF7B6FD694B6A4A1D78012313FA05F018
:100C20001178684E40EA01011170674A674F1178E8
:100C30006370674A735D3D70117023B943F6E0102D
:100C4000FEF740FB7055634B9B7803F02003DBB24B
:100C500013B13B780122F2545C4B1878FFF74EFE3B
:100C60005D480B210CF035FCF8B95C4B1B78002B70
:100C700040F03681504802F071F8002800F03381CE
:100C80004D495748EFF77CFD022343F6E3106370AC
:100C9000FEF718FB534B18704C4B1878FFF72EFEDD
:100CA0004D480B210CF015FC08B1062379E002F049
:100CB00095F8E0B102F0BCF8484D10B1494B1B78F3
:100CC0002B702B780BB901F025F902F0E1F8002820
:100CD00000F0098103236370F6F71CFE43F6E2106F
:100CE000FEF7F0FA404B187002232B70FAE006234F
:100CF0006370F5E0FFF7ECFD002800F0F480374B5F
:100D00001B78002B40F0EE80304B1878FFF7F6FD93
:100D1000364B1D7815F0030523D104F0ADFF0028F4
:100D200000F0E18004F08AFF002800F0DC800AF087
:100D300095FE002840F0D2802D4B93F8292093F89F
:100D40002A1042EA012193F82B2041EA024102468F
:100D500061F31702D3F82100D3F82510032304F020
:100D60004DFF244B1A7842F014026FF345121A70AB
:100D7000FFF7F4FE042314E0FFF7AAFD002800F0BB
:100D8000B2800DF06FF9002840F0AC80164B1A7855
:100D90000AB1013A1A701B7873B3104B02221A7011
:100DA000032363709EE000BF240E0020B1160020D4
:100DB000AE160020A3170020531600205116002065
:100DC0004D1600202C160020E0150020EE15002006
:100DD00046170020A8210020E1150020F115002071
:100DE000B517002047170020D41700201E2400202C
:100DF0004C0C0020F82E00203C4D0DF055F92A78BF
:100E0000012111FA02F23A4B3A4E197821EA020214
:100E10001A70337803F00503042B01D1FEF7CCFEE2
:100E2000337813F0010002D12A783349885403F053
:100E30000303022B04D1314B1A7842F010021A70CE
:100E400001F0CCFF08B90623637043F6E110FEF70A
:100E500039FA264F2A4B284A18703B78D15C09B1E1
:100E60000139D154012515FA03F62649D25C0878D8
:100E700020EA06000870CAB91D4E3178194111F0F8
:100E8000010F10D05B19FF210091019202932946B6
:100E90002B463B200332FEF789FA3B789D4033789E
:100EA00023EA050535703878FFF748FD00236370A5
:100EB00001F0EEFFA0B901F02DF811E00DF0F4F80B
:100EC00005236370FFF758FD60B90C4B1A7842F0A8
:100ED00008021A7007E00020607004E0284602E073
:100EE000012000E0002005B0F0BD00BFEE1500209D
:100EF0004D160020461700202C1600204917002010
:100F0000F11500203415002008B5064B4FF414717C
:100F10001A78054B01FB02314A2209180348EFF702
:100F200095F908BD3E140020A0A90208641600200F
:100F300070B53B4C2378032B66D8DFE803F0020A38
:100F40001946384B03221A7001232370364B033A9B
:100F50001A70344B1B78002B59D0344B1A7842F05E
:100F600001021A7023780022013323702E4B1A706D
:100F70000DF078F810B12E4B0A221A702B4D2B78F9
:100F800013F0010F0CD00DF06DF8064640B9FFF7D5
:100F9000BFFD2B780A2266F300032B70244B1A70D6
:100FA000FFF708FD032805D10DF07EF82378013303
:100FB00023702EE01E4B187800282AD1194B1A787E
:100FC000013A1A700123237070BDFFF7F3FC184B30
:100FD00005461B780BB1012808D14A20FFF798FD80
:100FE000104B1A78013A1A7001232370022D12D087
:100FF000052D12D1FFF79AFDBF20FFF79FFD0D4889
:101000000DF000F8FEF7D8FD0020207070BD012023
:1010100070BD002070BD284670BD002070BD00BFAF
:10102000F015002050160020D51700204917002089
:10103000D6170020641600200A4A13783BB1013B02
:10104000DBB21370084A52F82320084B1A60084B91
:1010500008481A7800216FF300021A704A22EFF74D
:101060009DB900BFB0160020D8170020141600202C
:10107000E42E0020641600202DE9F041384D394F50
:101080002B7823B90CF0EEFF08B103233B703B78BB
:10109000002B5FD1344C207800285FD00CF0E2FFA9
:1010A00000285AD12B78FF2B07D12D4B1870FFF752
:1010B000C3FF2C4A032313702370DFF8C0802B4E2C
:1010C00098F8003033B340460CF09CFF00214A22D0
:1010D0004046EFF763F9264A33681146934205D03C
:1010E000244A934202D0FF232B7033E025781E4A16
:1010F0000120002D32D08B4204D1107001380CF049
:10110000DDFA1BE01B498B4218D1107000200CF057
:101110009BFC13E02B78142253433268DFF84080A5
:10112000D118097971B9144B1B781BB19420FFF7C2
:10113000EFFC01E005233B7000232B702378013B7B
:10114000237007E0D058FFF7E3FC98F80030013334
:1011500088F800300120BDE8F0810120BDE8F08171
:10116000B4170020D61700204517002014160020C1
:10117000D80E0020500F0020B0160020641600206A
:1011800030B50F4A0F4913780D680F4C8068022B59
:1011900044F82350086001D8013313700B4B984278
:1011A00004D10020BDE830400CF088BA084B9842CA
:1011B00004D10020BDE830400CF046BC30BD00BF7B
:1011C000B016002014160020D8170020D80E0020DA
:1011D000500F002010B5154B1B681979022903D157
:1011E00013490870184617E012498B4203D1BDE835
:1011F00010400CF071BB10498B4203D1BDE8104088
:101200000CF0B6BC142101FB00321379012B02D083
:10121000032B0AD104E01046BDE81040FFF7B0BF31
:10122000034913690878117B984710BD14160020F4
:1012300048170020D80E0020500F00201D4BF7B596
:101240001B68002504E01A7B1433954238BF15460D
:101250001A79002AF7D16846F6F770FB044608B100
:10126000F6F758FB0DF1FF361FE0134B03221A70FF
:10127000124A00231370124A16F8017F13700CF003
:1012800013FF232F02D1FFF7D7FE10E0303FFFB24C
:1012900037B1AF4204D8013FF8B2FFF79BFF06E039
:1012A000013CDE20E4B2FFF72FFE002CDDD101204F
:1012B000FEBD00BF1416002045170020D6170020E1
:1012C000B417002010B5104B00241A7821466FF394
:1012D00000021A700D4B0E4A1C700E4B0E481A601D
:1012E0000822EFF75BF8FFF721FC0C4BFF221C7084
:1012F0000B4B1C700B4B1A700B4BFC3A1C700B4BBE
:101300001A700B4B1C7010BDE42E002049170020F2
:1013100010AD02081416002034160020D517002046
:10132000D6170020B4170020F01500204517002024
:10133000B016002070B5364CA378042B60D8DFE8D7
:1013400003F00320334E57000123A370314B1B7869
:1013500003F00802D2B212B12D4A0221917003F0BB
:101360001003DBB203252C4E2BB1FFF7ABFF00209F
:10137000A570307070BDFFF7A5FF284B1D700A23C4
:101380003370254D287800282CD0F6F791FA2328C1
:1013900039D1FFF7F1FA20B10020052360702B70DE
:1013A00070BD02232870A370FFF7C2FD012803D18E
:1013B0000423A370013870BD022826D1FFF7B6FBC5
:1013C000154B00251D700323A370154B1878F4F7F7
:1013D0000FFAD8B1134A144B28461A6070BDFFF7B4
:1013E0004BFE10B90423A37070BDFFF727FF0AE07E
:1013F00000F090FD0CF058FE0023A370012070BD9A
:101400000020A07070BD002070BD002070BD00BF26
:10141000240E002049170020D61700205016002067
:101420001816002060AD0208141600202DE9F041C6
:10143000884D894C2B6826466FF3DB632B6023783D
:101440006FF34513237001F0CFFD58B1834B1B7828
:1014500043B10220072106F017FA237843F0200356
:10146000237010E001F0A4FD90B17D4B1B787BB997
:101470007A4B1B7863B10220012106F005FA33781C
:1014800043F0200333702B6843F000632B6010E0BF
:1014900008F032F910B10220012108E0297801F0AA
:1014A0001001C9B211B10220014600E0022006F08D
:1014B000EBF96C4C2378082B00F21C83DFE813F067
:1014C00009001E002B0136015A017A01E6010902CA
:1014D0000A030BF079FB08F0C5F8FEF779FFFEF779
:1014E0001FFF614B00229A70012323705F48802107
:1014F0000CF0FFFF04F0C8FB0CF0E4FDFF205C4E95
:10150000014608F027F9337803F00A02082A06D0CA
:1015100003F00502042A02D013F0300F0DD0554B12
:101520001B7803F00203DBB20BB104F0ADFB3378A0
:1015300003F0D3036FF304133370AB7803F00203AB
:10154000DBB24BB1082323704B484C4B3C221A7042
:10155000BDE8F0410CF056BD494E337803F040032E
:10156000DBB223B908F0E0F8002800F0C382FEF7F0
:10157000E9FE10B9FEF7D8FF70B101F0A1FC414BB4
:101580001A7842F008021A70374B00229A7005232D
:1015900023703D4B02321A706B7803F00203DBB20A
:1015A0005BB1337803F04003DBB233B1374B1A78C9
:1015B0006FF301021A70062308E0FFF717F840B135
:1015C000337803F04003DBB21BB102232370BDE884
:1015D000F081F1F77DF82E4DFF28287029D02D4B92
:1015E0001B78002B40F08682012212FA00F02A4B71
:1015F0001A781043187043F6DF30FDF763FE274B6F
:101600001870274807F0CCFF204B1B7803F003032A
:10161000022B00F06F822978224801EB011101F5BD
:101620006C5107232E3110222370BDE8F041FDF7E5
:1016300063BEFEF7EFFF002838D01B4807F0B0FF6D
:10164000124B1B7803F00303022B00F05382032399
:10165000BCE700BFA8210020042300203818002088
:10166000F32900202B160020240E0020001001403A
:10167000F82E002095210020071700200A2A0020BC
:101680000C18002049170020ED1500201E24002012
:10169000EF15002052160020111200204F160020D6
:1016A000EA240020A31700201A240020984B994C0C
:1016B0005A7860F386125A70257805F01003DBB271
:1016C000002B00F01782337803F04003DBB2002BCD
:1016D00000F01082904B1B7833B963F3041563F369
:1016E00001052570BDE8F08115F00C0540F002827F
:1016F0002946062204F1A300EEF750FEA01C29465D
:10170000A122EEF74BFEF0236370237843F004032D
:1017100065F304135AE70221FF2008F01BF8FFF7D6
:101720006BF8002800F0E68100234FE77B4B1B7825
:1017300023B17B4B5B78012B3FF448AF794B1B788F
:1017400003F00303012B02D10220FF2101E0FF205F
:10175000022107F0FFFFFFF73FFA002800F0CA81DF
:1017600001F096FB002800F08E806D4B00229A70ED
:10177000042323706B4B1B7803F00303012B02D16E
:101780000220FF2101E0FF20022107F0E3FF01F02A
:101790007FFB20B1FFF7CEFD002800F0AB8101F008
:1017A00077FB08B900F0B6FB00232370BDE8F041D9
:1017B0000CF07ABC5B4D2B7803F00303012B02D1B4
:1017C0000220FF2101E0FF20022107F0C3FF04F007
:1017D00053FA002800F08E8104F030FA002800F05F
:1017E00089810AF03BF9002840F084812D784E4928
:1017F00005F00305012D19D191F82A2091F829301F
:1018000043EA022391F82B2043EA024300F07F428F
:101810001A43D1F821000D23D1F8251004F0EEF978
:10182000424880212A460CF064FE13E091F82A20F9
:1018300091F8293043EA022391F82B2043EA02432E
:1018400000F07F421A43D1F821000323D1F825107C
:1018500004F0D4F9364B1A7842F014026FF34512B3
:101860001A702F4B00229A7001F012FB30B1314BED
:101870001B78002B40F03E810433A7E601F038FBD3
:10188000002840F037812070BDE8F0810221FF2060
:1018900007F060FF284801F061FA01F041FB10B940
:1018A000264B05221A7001F03BFB20B901F096FA95
:1018B000002840F01F81214B1E78002E40F01A8135
:1018C0002B6866F349232B6000F024FB2670BDE8EB
:1018D000F081144E337803F00303012B02D1022070
:1018E000FF2101E0FF20022107F034FF144B1F7895
:1018F00067BB144D01222878134B8240197821EAE6
:1019000002021A70F0F716FF2F702770BDE8F08101
:10191000182400204018002038180020F11500205D
:10192000240E00201E2400204C0C0020001001403A
:10193000F82E0020ED1500201A16002019160020A0
:10194000A3170020EF150020111200206A4B1A780F
:10195000984602F02002D2B29ABB337813F0030FFC
:101960002FD104F089F9002800F0C48004F066F952
:10197000002800F0BF800AF071F80746002840F008
:10198000B9805E4B93F8292093F82A1042EA01218E
:1019900093F82B2041EA0241024661F31702D3F883
:1019A0002100D3F82510082304F028F998F8003016
:1019B00067F3041367F38203DBB243F0200388F874
:1019C00000304F4801F0CAF901F04AFA002866D108
:1019D0004C4B9B7803F01003DBB21BB9337813F048
:1019E000030F0BD0484B5B7803F00803DBB2002BEE
:1019F00055D1337803F00303012B50D101F048FA9D
:101A0000002846D098F800303B4D03F02003DBB2AD
:101A1000002B35D1337803F00303012B30D104F0D0
:101A20002BF9002866D004F009F9002862D00AF0EA
:101A300015F8064600285DD1334B5B7803F00203AE
:101A4000DBB2EBB12D4B93F8292093F82A1042EA30
:101A5000012193F82B2041EA0241024661F317026B
:101A6000D3F82100D3F82510102304F0C7F82B7801
:101A700066F3041366F38203DBB243F020032B709A
:101A8000224B1878F0F774FE002833D000F042FAA9
:101A900019E001F0CDF928B11D4B1A7800E00022C1
:101AA0001C4B1A701B4B1B7823BB184E3078F0F779
:101AB000B5FF00F02FFAAB7803F04003DBB213B1AF
:101AC0003078F0F737FE00232370134B0F221A7083
:101AD000BDE8F081FF20014607F03CFE0F4B1B786C
:101AE00023B1054B1B7813F0010F03D10CF0EAFA78
:101AF00001232370BDE8F081F82E00204C0C00205B
:101B0000A31700200C18002018240020EF15002037
:101B10004F16002044170020521600200A2A0020E9
:101B2000034B9878A0F10303584240EB0300704741
:101B3000240E002010B50446EEF780FE2146C2B206
:101B40000948EEF751FB094B18B964221A700130AD
:101B500010BD1A780AB1013A1A70187810B9044BFE
:101B6000187010BD002010BD0D190020391800207C
:101B70000719002038B5002412E0242B0ED1601C78
:101B800028180A490322EEF72FFB38B9281943F623
:101B90007F210422FDF7A7FB0334E4B20134E4B251
:101BA000034D2B5D002BE8D138BD00BFD5AD020839
:101BB0000D1900202DE9F0474C4C4D4D23684D4840
:101BC00043F0040323602968A2460431EEF7D8FDF0
:101BD000FFF7D0FF47484FF4FA710BF0F7F945488B
:101BE00000210BF02DFA2E46074600286DD02868FC
:101BF0004430FFF79FFF8046002848D1C8200BF0F3
